:0410000062EF09F0A2
:101008005D82FACF4BF0FBCF4CF0E9CF4DF0EACF41
:101018004EF0E1CF4FF0E2CF50F0D9CF51F0DACF18
:1010280052F0F3CF53F0F4CF54F0F6CF55F0F7CF9A
:1010380056F0F8CF57F0F5CF58F05DC059F05EC0C4
:101048005AF05FC05BF060C05CF0A6AAACD0A69A6C
:101058002ACF28F023BA83D0240E2818D8A40CD07D
:1010680082D0C951010D780EF324D96E040EF420F4
:10107800DA6E28C0DFFF7BD00101C951010D780E5F
:10108800F324D96E040EF420DA6E28C0DFFFC92BD2
:101098002A0E2818D8A419D0520E04017B19D8A4F6
:1010A80014D04D0E7C19D8A410D0430E7D19D8A4A5
:1010B8000CD0000E0101C96F2780C72B010E020159
:1010C8002E27000E2F2330233123540E04017B19C1
:1010D800D8A412D0580E7C19D8A40ED0540E7D195D
:1010E800D8A40AD0000E0101C96F000E04017B6F5D
:1010F800000E7C6F000E7D6F500E7919D8A412D0A7
:10110800410E7A19D8A40ED0490E7B19D8A40AD05A
:10111800000E0101C96F000E04017B6F000E7C6F89
:10112800000E7D6F500E7919D8A412D0510E7A197D
:10113800D8A40ED0540E7B19D8A40AD0000E0101F1
:10114800C96F000E04017B6F000E7C6F000E7D6F6F
:101158007F0E0101C9658CD0000EC96F89D0240E9D
:101168002818D8A406D0000E0101C96F7AD7C92B58
:101178007FD07F0E0101C96502D0000EC96FC95129
:10118800010D780EF324D96E040EF420DA6E28C00F
:10119800DFFFC92B240E04017819D8A404D00A0E45
:1011A8002818D8B42386A6A020D0A6909E908F9207
:1011B8000101C2B71AD0C287C283CECF36F2CFCFD1
:1011C80037F20201386B396B000ECF6E010ECE6E0E
:1011D8000101C291C293C28BB790010E0F01066F35
:1011E8007D0E056FB890B78004859EA00ED09E90A6
:1011F800000ECF6E000ECE6E0101CA2B100ECA195A
:10120800D8A403D0C281000ECA6FB8A00BD0B89082
:10121800010E0F01066F7D0E056FB79004958F8242
:101228000101C2979EA222D09E920101C8A104D0BA
:10123800010ECC6E1E0E03D0010ECC6EE10ECB6EED
:10124800B82B030EB819D8A411D0B62BB52BBC8176
:10125800A34BA42B02016D4B6E2B010E3E27000EF3
:101268003F2340234123000E0101B86FBDEC4BF032
:101278005CC060F05BC05FF05AC05EF059C05DF0C2
:1012880058C0F5FF57C0F8FF56C0F7FF55C0F6FF26
:1012980054C0F4FF53C0F3FF52C0DAFF51C0D9FF66
:1012A80050C0E2FF4FC0E1FF4EC0EAFF4DC0E9FF6A
:1012B8004CC0FBFF4BC0FAFF5D92110041EF64F098
:1012C8000024392C35383533323831302C33343723
:1012D80033353732302C362C313136382C313936DB
:1012E800332C333332302C313237382C33313832D7
:1012F8002C313534382C333534372C313931382CBE
:10130800323230302C313435352C313834332C31BD
:101318003730322C65766974612E7061722C302CEE
:101328002A00010000000A00000064000000E80331
:10133800000010270000A086010040420F008096A0
:10134800980000E1F50500CA9A3B24322C352C3070
:101358002C352C302C352C302C352C302C352C3091
:101368002C352C302C352C302C352C302C2A0024C4
:1013780031302C322C323030302C2A003134333199
:101388002C31383034313600504D544B3136312CF5
:10139800302A0024362C332C332C312C2A002435C7
:1013A8002C322C322C322C2A0024342C312C312C87
:1013B800312C2A000E0B0510141516170F1F244781
:1013C80050454E440D0A002431312C36302C2A0069
:1013D8002431322C322C2A005B444154415D0024D4
:1013E800382C322C2A0024372C332C2A0024332C76
:1013F800302C2A003F157E144A143335000714098F
:10140800024300020100C032090400000102020187
:101418000005240010010424020205240600010529
:1014280024010001070581030800020904010002E4
:101438000A0000000705020240000007058202407A
:1014480000003403430044004300200052005300CE
:101458002D00320033003200200045006D00750079
:101468006C006100740069006F006E002000440089
:1014780065006D006F0034034D0069006300720061
:101488006F00740065007800200046006900720053
:1014980065004C006F0067000000000000000000BD
:1014A80000000000000000000000504D544B333194
:1014B800342C302C312C302C302C302C302C302C3F
:1014C800302C302C302C302C302C302C302C302C34
:1014D800302C302C302C302A0024312C70696C6F61
:1014E800746F2C70697374612C2A00120100020257
:1014F800000008FF0FFF0F000101020001504D54CA
:101508004B3235312C35373630302A00504D544B5C
:101518003232302C3130302A0024302C462C3130F5
:1015280030302C2A00504149523030322A00504184
:1015380049523030332A00040309040D0A24677025
:10154800636C724552524F52210054454D50205001
:101558004152002467657261772C00286E756C6CA7
:101568002900244750454E4400247365636E660085
:10157800246770636C6D00246770636F6E00246766
:1015880070636C7200246770636C7400256C64006F
:07159800256400257300002B
:1015A000000E58EC71F0320E17EC72F0EAEC46F0D7
:1015B0008F8E0101C483020E0201606F000E5F6F07
:1015C0002FEC58F003EC6EF0000E756E000E0E015D
:1015D000106F000E2D6E7CEC71F0000E0101CC6FCF
:1015E000320EFC6F86B429D0000E1E6E1F0E1E64D4
:1015F00001D004D042EC4EF01E2AF8D797EC66F0EA
:101600001E6E150E1E18D8B408D0160E1E18D8B4AB
:1016100004D0170E1E18D8A408D01D901D821D944A
:10162000080E0101CC6F000E1E6E238A23942392B4
:101630001D9254EC45F0239A01D08F9E000E156E3A
:10164000100E166E000E176E000E186EE1EC70F0A4
:1016500000C5E8FF240AD8A41ED001C5E8FF530A3C
:10166000D8A419D002C5E8FF450AD8A414D003C5F0
:10167000E8FF550AD8A40FD004C5E8FF500AD8A443
:101680000AD005C5E8FF4C0AD8A405D043EC40F0C9
:10169000F29E0EEF00F059EC6CF043EC40F0CFEC12
:1016A00053F0050E1E6E25928D808D8217EF11F07E
:1016B000090E1E18D8A480D00E01E8A702D0010E92
:1016C00001D0000EFF0A0201F86FF847F847F8470B
:1016D0000E01E8510201F819F70BF8190E01E86F35
:1016E000E8A502D0010E01D0000EFF0A0201F86F3A
:1016F000F847F8470E01E8510201F819FB0BF819F9
:101700000E01E86FE8A302D0010E01D0000EFF0A1F
:101710000201F86FF8470E01E8510201F819FD0BBC
:10172000F8190E01E86FE5A702D0010E01D0000EF6
:10173000FF0A0201F86FF847F847F8470E01E55134
:101740000201F819F70BF8190E01E56FE5A902D0AF
:10175000010E01D0000EFF0A0201F86FF83B0E01E6
:10176000E5510201F819EF0BF8190E01E56FE5A339
:1017700002D0010E01D0000EFF0A0201F86FF847F7
:101780000E01E5510201F819FD0BF8190E01E56F84
:10179000E5A502D0010E01D0000EFF0A0201F86F8C
:1017A000F847F8470E01E5510201F819FB0BF8194B
:1017B0000E01E56F2790268203013C518CEC6EF000
:1017C000B9EF17F0000E1E6E1E50CCEC6BF0B9EFA7
:1017D00017F01E50CCEC6BF00E01E887E885E8832B
:1017E000E587E589E583E5851E50D8B4E8971E04B2
:1017F000D8B4E895020E1E18D8B4E893030E1E184C
:10180000D8B4E597040E1E18D8B4E599050E1E1835
:10181000D8B4E593060E1E18D8B4E595070E1E1829
:10182000D8A409D0E887E885E883E587E589E583DA
:10183000E5858D908D82080E1E18D8A409D0E897F2
:10184000E895E893E597E599E593E5958D808D9288
:101850001E2A0A0E1E18D8A4B9EF17F0000E1E6E2D
:10186000B9EF17F0010E1E6E4BEC72F01E50CCEC6F
:101870006BF0B9EF17F0020E1E6E33EC72F01E50D3
:10188000CCEC6BF0B9EF17F0090E1E18D8A4B9EF25
:1018900017F00E01E8A702D0010E01D0000EFF0ADA
:1018A0000201F86FF847F847F8470E01E8510201C6
:1018B000F819F70BF8190E01E86FE8A502D0010E30
:1018C00001D0000EFF0A0201F86FF847F8470E0139
:1018D000E8510201F819FB0BF8190E01E86FE8A3B3
:1018E00002D0010E01D0000EFF0A0201F86FF84786
:1018F0000E01E8510201F819FD0BF8190E01E86F0D
:10190000E5A702D0010E01D0000EFF0A0201F86F18
:10191000F847F847F8470E01E5510201F819F70BAF
:10192000F8190E01E56FE5A902D0010E01D0000EF5
:10193000FF0A0201F86FF83B0E01E5510201F819A8
:10194000EF0BF8190E01E56FE5A302D0010E01D0EF
:10195000000EFF0A0201F86FF8470E01E55102017F
:10196000F819FD0BF8190E01E56FE5A502D0010E7F
:1019700001D0000EFF0A0201F86FF847F8470E0188
:10198000E5510201F819FB0BF8190E01E56F2790DC
:10199000268288EC70F0B9EF17F02784B9EF17F0C2
:1019A00056EC5EF0B9EF17F053EC33F0000AD8B400
:1019B000B9EF17F0020AD8B47BD6010AD8B4A4EF65
:1019C00017F0160AD8B4FED6030AD8B402D7010A13
:1019D000D8B448D70F0AD8B44ED7010AD8B4E0D744
:1019E000070AD8B451D73A0AB9EF17F00201B65135
:1019F00004E1330EB55DD8A034D001014E5102018F
:101A0000AD5D01014F510201AE590101505102017A
:101A1000AF59010151510201B059D8B008D0ADC23F
:101A20004EF1AEC24FF1AFC250F1B0C251F101015F
:101A300052510201B15D010153510201B25901013C
:101A400054510201B359010155510201B459D8B0A2
:101A500008D0B1C252F1B2C253F1B3C254F1B4C210
:101A600055F10E01E8A702D0010E01D0000EFF0AC9
:101A70000201F86FF847F847F8470E01E8510201F4
:101A8000F819F70BF8190E01E86FF5EC70F0B9EFE3
:101A900017F0180E01014E27FC0E4F23FF0E5023A6
:101AA000FF0E5123180E5227FC0E5323FF0E542312
:101AB000FF0E552321EE52F0DECFF8F2DDCFF9F222
:101AC0000201F81FF91FF84BF92BB151F82503015A
:101AD000536F0201B251F9210301546F21EE4EF010
:101AE000DECFF8F2DDCFF9F20201F81FF91FF84B53
:101AF000F92BAD51F8250401506F0201AE51F921C7
:101B00000401516F010E01014C6F27840E01E8970B
:101B1000E885E8832486279A010E01011FD356EC3D
:101B20005EF0B9EF17F053EC33F0000AD8B4B9EF18
:101B300017F0020AD8B45AD7010AD8B4A4EF17F0A4
:101B40000F0AD8B4B9EF17F0190AD8B4B9EF17F0E3
:101B5000030AD8B4B9EF17F0010AD8B4B9EF17F0F7
:101B60000F0AD8B4B9EF17F0010AD8B4D8D73D0A94
:101B7000D8B4B9EF17F0150AD8B48BD7B9EF17F06E
:101B80000E01E8A702D0010E01D0000EFF0A0201EB
:101B9000F86FF847F847F8470E01E8510201F819C5
:101BA000F70BF8190E01E86F010E0201976F020E94
:101BB0009F6F26B025A203D05EEC41F0269071EC19
:101BC00042F006EC66F0B9EF17F06FEC67F026B064
:101BD00025A2B9EF17F00E01E8935EEC41F02690D4
:101BE0000E01E883B9EF17F026B025A2B9EF17F080
:101BF0000E01E895320E17EC72F00E01E8855EECEE
:101C000041F0B9EF17F07B0E8CEC6EF035EC6AF01A
:101C100083EC3CF0B6EC67F046EC69F008D3FBECE3
:101C20006BF035EC6AF043EC40F0B6EC67F0800EF8
:101C300002019D199E11D8B4B9EF17F0020EFFEC06
:101C40004FF0B9EF17F0020E0101CC6F2784FBECC7
:101C50006BF0B9EF17F0180E8CEC6EF056EC5EF0EE
:101C6000B9EF17F053EC33F0000AD8B4B9EF17F01E
:101C7000020AD8B4B9EF17F0010AD8B4E4D70F0AB2
:101C8000D8B4B9EF17F0030AD8B49FD71E0AD8B456
:101C9000ABD7040AD8B4B7D7030AD8B4C0D7010A5F
:101CA000D8B4B9EF17F00F0AD8B4B9EF17F0010A9A
:101CB000D8B4D1D7040AD8B463D7B9EF17F056EC2B
:101CC0005EF0B9EF17F020502118D8A432D0295077
:101CD000D8A418D0010E296E78C160F079C161F0E6
:101CE0007AC162F07BC163F074C164F075C165F0C4
:101CF00076C166F077C167F0000E0001686FC3EC33
:101D000069F017D0000E296E78C160F079C161F0DA
:101D10007AC162F07BC163F074C164F075C165F093
:101D200076C166F077C167F0010E0001686FC3EC01
:101D300069F0F5EC70F0B9EF17F035EC6AF0A5EC4E
:101D400062F00101B46F4CC1B3F1B451D8B413D0F7
:101D50004FEC66F0000E296E20C021F00E01D98FE5
:101D6000010EFFEC4FF00E01E885E883E8878D90C7
:101D70008D92B9EF17F088EC70F088EC70F088EC79
:101D800070F088EC70F008EF13F0010E216401D0C0
:101D90002106215023EC51F0B9EF17F00101B451A5
:101DA000215CD8A0212A215023EC51F0B9EF17F083
:101DB0004FEC66F0000E296E20C021F0B9EF17F04D
:101DC000060EA5EF17F0FBEC6BF08FEC72F0A4EFB2
:101DD00017F053EC33F0000AD8B4B9EF17F0010A4A
:101DE000D8B4ABD7030AD8B4ACD0010AD8B4EBD777
:101DF000160AD8B4CAD7030AD8B4D0D7010AD8B4BF
:101E0000D7D70F0AD8B4DCD7010AD8B458D7040AF8
:101E1000D8B459D73F0AD8B4FBD32FEF13F056EC00
:101E20005EF0B9EF17F00101A751A811D8A408D0AE
:101E3000000EA86F010EA76F21508CEC6EF009D038
:101E4000000E0101A86F000EA76F0001FA514AECC5
:101E50006EF0F5EC70F0B9EF17F035EC6AF0000EAB
:101E6000296E000E0101A86F000EA76F010E000180
:101E7000FA6F2950D8A406D0010EEB6FFA515BEC33
:101E800048F0D5D1000E0001EB6FFA515BEC48F041
:101E9000CED10001FA05D8A4FA072950D8A407D05A
:101EA000010EEB6FFA515BEC48F0B9EF17F0000E42
:101EB0000001EB6FFA515BEC48F0B9EF17F001014C
:101EC000B3510001FA5DD8A0FA2B2950D8A407D04D
:101ED000010EEB6FFA515BEC48F0B9EF17F0000E12
:101EE0000001EB6FFA515BEC48F0B9EF17F02950A5
:101EF000D8A40AD0010E296E000E0001EB6FFA5132
:101F00005BEC48F0B9EF17F0000E296E010E0001EE
:101F1000EB6FFA515BEC48F0B9EF17F0050E0101D9
:101F2000CC6F215023EC51F0000E296EB9EF17F061
:101F3000FBEC6BF0A4EF17F0CC6F2FD588EC70F0B2
:101F400067D30101C5B3B9EF17F0000EF5D753EC15
:101F500033F0000AD8B4B9EF17F0010AD8B47DD72E
:101F6000030AD8B4EED7010AD8B4E2D7160AD8B417
:101F700090D7030AD8B4A3D7010AD8B4B8D70F0AA8
:101F8000D8B4CCD7010AD8B44AD7070AD8B44BD7AB
:101F90003C0AD8B4D3D763D356EC5EF0B9EF17F050
:101FA0008FEC72F00E01E887E885E8838D908D92C2
:101FB000020E0201706F580E6F6F279625942498B9
:101FC00046EC69F0B9EF17F025B027A616D00E0140
:101FD000E887E8A502D0010E01D0000EFF0A020139
:101FE000F86FF847F8470E01E8510201F819FB0BAA
:101FF000F8190E01E86FE88314D00E01E887E88530
:10200000E8A302D0010E01D0000EFF0A0201F86F12
:10201000F8470E01E8510201F819FD0BF8190E01FD
:10202000E86FF5EC70F0DFD2D98FB9EF17F072ECF2
:1020300065F0E806D8A4B9EF17F027840E01E897F9
:10204000E885E8832486279A01014C51D8B44FD003
:102050004EC1F8F24FC1F9F250C1FAF251C1FBF290
:102060000201F81FF91FFA1FFB1FF82B000EF923BE
:10207000FA23FB23AD51F82500016C6F0201AE512C
:10208000F92100016D6F0201AF51FA2100016E6F5D
:102090000201B051FB2100016F6F000E6AEC4AF0A3
:1020A0006CC07EF06DC07FF06EC080F06FC081F0BC
:1020B000CDEC6EF07EC0ABF07FC0ACF080C0ADF078
:1020C00081C0AEF0000E0001AF6F600EB06FEA0E7F
:1020D000B16F460EB26F92EC50F00001D8B007D04D
:1020E000010E0101CC6F010EB96FB9EF17F0000EB0
:1020F00001014C6FFF0E4E6FE70E4F6F760E506F63
:10210000480E516FFF0E526FE70E536F760E546FED
:10211000480E556F010E4D6F030EBF19D8A402D0A3
:10212000020E4D6F0E01E897E885E88335EC6AF002
:10213000DDEC6DF0F00ECFEC71F0F00ECFEC71F045
:10214000F00ECFEC71F0B6EC67F0000E02016C6F90
:10215000000E6B6F000E0101B96F010ECC6FB9EF6D
:1021600017F0FBEC6BF0A4EF17F035EC6AF0A5EC80
:1021700062F00101B46FB451D8B402D0050EDCD6C0
:102180000E01D98F88EC70F088EC70F088EC70F05C
:1021900088EC70F0B6EC67F00E01E887E885E8831C
:1021A0008D908D9246EC69F0B9EF17F02488B9EF65
:1021B00017F02784D6D153EC33F0000AD8B4B9EF26
:1021C00017F0010AD8B4ECD6030AD8B430D7010A04
:1021D000D8B4C7D70F0AD8B4F7D6010AD8B4BBD140
:1021E0001A0AD8B4C2D70F0AD8B4E0D7010AD8B4B3
:1021F000D3D6B9EF17F056EC5EF0B9EF17F08FECCD
:1022000072F00E01E89735EC6AF083EC3CF0B6EC26
:1022100067F0259A01014C51D8A427EC6FF00E010C
:10222000E887E885E8838D908D9246EC69F00E0191
:10223000FBD6278AB9EF17F06FEC67F026B025A21E
:10224000B9EF17F08F88120E17EC72F05EEC41F0C8
:102250008F9826A2B9EF17F071EC44F0B9EF17F0A0
:1022600026B025A2B9EF17F01DA002D00E01E89705
:10227000120E17EC72F05EEC41F026B271EC44F0F5
:102280001DA0B9EF17F00E01E887B9EF17F0F5ECD4
:1022900070F01DB0B9EF17F027A225BA18D00101D0
:1022A000B905D8A414D00E01E8A702D0010E01D0C0
:1022B000000EFF0A0201F86FF847F847F8470E01D1
:1022C000E8510201F819F70BF8190E01E86F010146
:1022D000C5B325AA02D080EC43F00101C5A325BAFD
:1022E00002D0A4EC63F00101C5A3B9EF17F0E9EC4B
:1022F00061F006EC66F0B9EF17F025A217D026A022
:1023000005D05EEC41F026B271EC44F071EC42F085
:1023100027A225AA0BD01DB009D048EC62F0D7EC5B
:102320004EF06BEC4FF0000EFFEC4FF001014C5102
:10233000D8B453D0B751D8B402D0B7074ED0E2ECDE
:1023400017F00101BB29D8B448D00A0EB76F25BADF
:102350000FD0BB51D8A441D0258A65EC4CF01EC2E9
:102360002AF21FC22BF220C22CF221C22DF235D04C
:102370002AC2F8F22BC2F9F22CC2FAF22DC2FBF2F9
:102380000201F81FF91FFA1FFB1FF82B000EF9239B
:10239000FA23FB231E51F825266F1F51F921276FC1
:1023A0002051FA21286F2151FB21296F1EC22AF2E8
:1023B0001FC22BF220C22CF221C22DF226C2EBF05A
:1023C00027C2ECF028C2EDF029C2EEF091EC26F025
:1023D0000009D8A402D00101CD830101B951D8A4CC
:1023E00051D00201B65104E1330EB55DD8A036D00C
:1023F00001014E510201AD5D01014F510201AE5983
:10240000010150510201AF59010151510201B0596E
:10241000D8B008D0ADC24EF1AEC24FF1AFC250F14C
:10242000B0C251F1010152510201B15D010153519C
:102430000201B259010154510201B3590101555130
:102440000201B459D8B008D0B1C252F1B2C253F1AE
:10245000B3C254F1B4C255F16B4B6C2B0E01E8A71B
:1024600002D0010E01D0000EFF0A0201F86FF847FA
:10247000F847F8470E01E8510201F819F70BF8196F
:102480000E01E86F0101C5B3B9EF17F0E9EC61F097
:1024900006EC66F0B9EF17F00101B951D8A4B9EF15
:1024A00017F0180E4E27FC0E4F23FF0E5023FF0E81
:1024B0005123180E5227FC0E5323FF0E5423FF0EF8
:1024C000552321EE52F0DECFF8F2DDCFF9F2020112
:1024D000F81FF91FF84BF92BB151F8250301536F81
:1024E0000201B251F9210301546F21EE4EF0DECF0B
:1024F000F8F2DDCFF9F20201F81FF91FF84BF92BC2
:10250000AD51F8250401506F0201AE51F9210401CB
:10251000516F010E01014C6F010EB96F0E01E8976A
:10252000E895E8935DEC31F00E01E887E885E883F3
:1025300027EC6FF0B9EF17F0FBEC6BF083EC72F067
:10254000A4EF17F0050E0101CC6FFBEC6BF083ECF0
:1025500072F0CDEF0CF0010E0101B06F030ECC6FE5
:1025600028D60E01E89517D153EC33F0000AD8B401
:10257000B9EF17F0010AD8B442D6030AD8B4BDD6D1
:10258000010AD8B4D9D70F0AD8B481D6010AD8B471
:10259000E2D7020AD8B450D61E0AD8B461D6040ACB
:1025A000D8B4B9EF17F0030AD8B4B9EF17F0010A9D
:1025B000D8B4C8D70F0AD8B43CD6010AD8B41BD6B1
:1025C000280AD8B469D7B9EF17F056EC5EF0B9EF26
:1025D00017F00101C5B3B9EF17F0CD91F5EC70F02C
:1025E0008FEC72F015D00E01D9AF1ED50E01D99F18
:1025F000B9EF17F0050E0101CC6F27848FEC72F054
:10260000B9EF17F00101CD91F5EC70F08FEC72F09D
:10261000000EA5EF17F0FBEC6BF083EC72F08FEC83
:1026200072F0A4EF17F053EC33F0000AD8B4B9EF0E
:1026300017F0010AD8B4B9EF17F0030AD8B4C9D714
:10264000010AD8B4E8D70F0AD8B4CDD71B0AD8B43A
:10265000D1D70E0AD8B4B9D73B0AD8B4D3D7060A13
:10266000B9EF17F00E01E8973BEC72F0B9EF17F0F5
:102670000E01E885E88788EC70F0FF00B9EF17F0ED
:102680005FEC6FF00E01E8952A50D8A407D07F0EBA
:102690000001606F150E616F3BEC6DF071EC70F036
:1026A00090D35FEC6FF00E01E895FBEC67F089D3F7
:1026B0005FEC6FF00E01E895000E0001766F050EDD
:1026C000776F5B0E786F150E796F16EC3FF02A501E
:1026D000D8A40AD0000E0001606F050E616F90EC67
:1026E0006DF002D03BEC72F02A50D8A4FBD7C3ECBB
:1026F00068F067D35FEC6FF00E01E89551EC54F091
:10270000000E0001676F050E686F85EC69F00E0121
:10271000E885FFD75FEC6FF00E01E895E893E88756
:1027200051EC54F041EC70F0780ECFEC71F0780E73
:10273000CFEC71F0780ECFEC71F0780ECFEC71F039
:10274000780ECFEC71F0780ECFEC71F0780ECFEC04
:1027500071F0780ECFEC71F0780ECFEC71F0780E4E
:10276000CFEC71F0780ECFEC71F0000E156E000E0C
:10277000166E000E176E000E186E000E0001666FCA
:10278000050E676F020E696F000E686F6CEC6AF0E1
:102790000E01E885E883E897ECD35FEC6FF00E015B
:1027A000E8950101CDA102D0010EC16F240EE8CF42
:1027B00000F5670EE8CF01F5650EE8CF02F5760E5D
:1027C000E8CF03F5650EE8CF04F5720EE8CF05F506
:1027D0002C0EE8CF06F525EE07F0EDC2DFFF25EE63
:1027E00008F0EEC2DFFF2C0EE8CF09F5020EF66E00
:1027F000140EF76E000EF86E0800F5CFF8F2F8C26E
:102800000AF5030EF66E140EF76E000EF86E080051
:10281000F5CFF8F2F8C20BF52C0EE8CF0CF525EE4B
:102820000DF0EAC2DFFF25EE0EF0EBC2DFFF2C0E4B
:10283000E8CF0FF5C1C16DF000016E6B100E6F6F28
:10284000050E706F3EEC68F02C0EE8CF13F52A0EE3
:10285000E8CF14F5000EE8CF15F52A50D8A407D01C
:10286000000E0001606F050E616F90EC6DF071EC71
:1028700070F0A7D25FEC6FF00E01E895FBEC62F010
:102880000101BE6F240EE8CF00F5670EE8CF01F519
:10289000650EE8CF02F5630EE8CF03F56C0EE8CFC6
:1028A00004F56F0EE8CF05F52C0EE8CF06F5BEC196
:1028B0006DF000016E6B070E6F6F050E706F3EECD2
:1028C00068F02C0EE8CF0AF5000EE8CF0BF52A5081
:1028D000D8A407D0000E0001606F050E616F90EC68
:1028E0006DF071EC70F06DD25FEC6FF00E01E89559
:1028F00014EC4BF06CC098F16DC099F16EC09AF178
:102900006FC09BF1240EE8CF00F5670EE8CF01F50C
:10291000650EE8CF02F56D0EE8CF03F5650EE8CF42
:1029200004F56D0EE8CF05F52C0EE8CF06F5000E88
:10293000010198250001606FE00E0101992100015D
:10294000616FFF0E01019A210001626FFF0E01010C
:102950009B210001636F100E646F270E656F000EE0
:10296000666F000E676F81EC68F0000160516D6F5B
:102970006E6B070E6F6F050E706F3EEC68F0300ED9
:10298000E8CF0AF5300EE8CF0BF5300EE8CF0CF5A6
:10299000300EE8CF0DF52C0EE8CF0EF5000EE8CF87
:1029A0000FF52A50D8A407D0000E0001606F050E65
:1029B000616F90EC6DF071EC70F003D25FEC6FF032
:1029C0000E01E895A5EC62F00101BE6F240EE8CF80
:1029D00000F5670EE8CF01F5650EE8CF02F5630E4E
:1029E000E8CF03F5740EE8CF04F5650EE8CF05F5E2
:1029F0002C0EE8CF06F5BEC16DF000016E6B070E20
:102A00006F6F050E706F3EEC68F02C0EE8CF0AF584
:102A1000000EE8CF0BF52A50D8A407D0000E000115
:102A2000606F050E616F90EC6DF071EC70F0C9D1C4
:102A30005FEC6FF00E01E8953DEC52F06CC098F140
:102A40006DC099F16EC09AF16FC09BF1240EE8CF72
:102A500000F5670EE8CF01F5650EE8CF02F56D0EC3
:102A6000E8CF03F5650EE8CF04F5740EE8CF05F561
:102A70002C0EE8CF06F5000E010198250001606FCD
:102A8000100E010199210001616FE00E01019A21F0
:102A90000001626FFF0E01019B210001636F0A0EAE
:102AA000646F000E656F000E666F000E676F81EC3D
:102AB00068F0000160516D6F6E6B070E6F6F050E51
:102AC000706F3EEC68F0300EE8CF0AF52C0EE8CFC0
:102AD0000BF5000EE8CF0CF52A50D8A407D0000E55
:102AE0000001606F050E616F90EC6DF071EC70F09D
:102AF00068D15FEC6FF00E01E895000E00016C6F7D
:102B0000070E6D6FD5EC6AF0DFEC66F0F00ECFECDF
:102B100071F0000E0001676F070E686F85EC69F0B9
:102B200043EC40F014EC4BF06CC015F06DC016F0A7
:102B30006EC017F06FC018F0200E16181510171081
:102B40001810D8B40DD02A50D8A40AD0450E0001D0
:102B5000606F150E616F3BEC6DF002D03BEC72F0D4
:102B60002A50D8A4FBD7000E156E200E166E000E4C
:102B7000176E000E186E2A50D8A407D0860E0001DA
:102B8000606F150E616F3BEC6DF071EC70F019D158
:102B90005FEC6FF00E01E895C0EC5EF0DDEC6DF0DF
:102BA000F00ECFEC71F0F00ECFEC71F0F00ECFEC38
:102BB00071F02050D8B42ED03DEC52F06CC09CF196
:102BC0006DC09DF16EC09EF16FC09FF1000E0001BF
:102BD000FC6F330EFC6501D01AD0FC51040D000EC1
:102BE000F324D96E030EF420DA6EFC51040DC50EE9
:102BF000F324E16E030EF420E26EDECFE6FFDECFBB
:102C0000E6FFDECFE6FFDECFE6FFFC2BE2D725882E
:102C100071EC44F043EC40F014EC4BF06CC015F058
:102C20006DC016F06EC017F06FC018F05FEC6FF05B
:102C30002A50D8A407D0780E0001606F150E616F7E
:102C40003BEC6DF071EC70F0BCD05FEC6FF00E01FE
:102C5000E895DDEC6DF0F00ECFEC71F0F00ECFECFE
:102C600071F0F00ECFEC71F0F00ECFEC71F0F00ED1
:102C7000CFEC71F0F00ECFEC71F043EC40F014ECBF
:102C80004BF06CC015F06DC016F06EC017F06FC041
:102C900018F05FEC6FF02A50D8A407D08D0E000119
:102CA000606F150E616F3BEC6DF071EC70F089D0C8
:102CB0005FEC6FF00E01E89541EC70F0F00ECFEC98
:102CC00071F0F00ECFEC71F0F00ECFEC71F0F00E71
:102CD000CFEC71F0F00ECFEC71F0F00ECFEC71F0A4
:102CE00014EC4BF06CC015F06DC016F06EC017F010
:102CF0006FC018F0200E1618151017101810D8B441
:102D00000DD02A50D8A40AD0450E0001606F150ED0
:102D1000616F3BEC6DF002D03BEC72F02A50D8A40E
:102D2000FBD7000E156E200E166E000E176E000EED
:102D3000186E2A50D8A407D0860E0001606F150EB9
:102D4000616F3BEC6DF071EC70F03BD05FEC6FF0BD
:102D50000E01E895C80ECFEC71F0C80ECFEC71F003
:102D6000C80ECFEC71F0C80ECFEC71F0E2EC6CF055
:102D7000140ECFEC71F071EC70F023D05FEC6FF0BB
:102D80000E01E89551EC54F0000E0001676F050E3E
:102D9000686F85EC69F043EC40F05FEC6FF002D0B7
:102DA0003BEC72F02A50D8A4FBD72A50D8A407D005
:102DB000710E0001606F150E616F3BEC6DF071ECF0
:102DC00070F00E01E885D5D00E01D98F010EFFEC11
:102DD0004FF00E01E897E885E883FA0ECFEC71F02A
:102DE000AEEC6FF088EC70F088EC70F088EC70F06E
:102DF00088EC70F00E01E88788EC70F088EC70F0D9
:102E000088EC70F088EC70F00E01E89788EC70F0B8
:102E100088EC70F088EC70F088EC70F00E01E887B8
:102E200088EC70F088EC70F088EC70F088EC70F052
:102E30000E01E89788EC70F088EC70F088EC70F088
:102E400088EC70F05FEC6FF088EC70F00101CD91D0
:102E500046EC69F00E01E885E89735EC6AF089D018
:102E600053EC33F0000AD8B432EF13F0010AD8B4AF
:102E7000ABD7050AD8B404D4010AD8B412D4030AD3
:102E8000D8B464D7010AD8B479D70F0AD8B4F2D429
:102E9000010AD8B438EF13F0030AD8B42AD6010ACD
:102EA000D8B422D51B0AD8B403D4020AD8B422D489
:102EB000010AD8B4FDD6070AD8B46FD40E0AD8B424
:102EC00067D6050AD8B4C1D63F0AD8B4B1D5010A2D
:102ED000D8B474D5020AD8B41DD44BD056EC5EF0E9
:102EE00048D00E01E887E893E887010EFFEC4FF029
:102EF00040D00E01E8A302D0010E01D0000EFF0A5F
:102F00000201F86FF8470E01E8510201F819FD0BB4
:102F1000F8190E01E86F0201ACA103D00101CD85C3
:102F200002D00101CD950E01E8A303D00101CD83AC
:102F300002D00101CD93F5EC70F00101B0518CECA1
:102F40006EF017D0FBEC6BF0020E01019CEF0FF05E
:102F500053EC33F0000AD8B40CD0010AD8B4C1D76E
:102F6000020AD8B4EFD70F0AD8B4C3D7150AD8B419
:102F7000B5D70101CC51000AD8B4DBEF10F0010A3B
:102F8000D8B4B4EF12F0030AD8B46AD7010AD8B49F
:102F9000DFD7070AD8B432EF0EF0010AD8B4E9EF50
:102FA0000EF0030AD8B4A7EF0FF0010AD8B413EF5C
:102FB00013F00F0AD8B4D4EF0CF0010AD8B493EF91
:102FC0000DF0D7D70101BB69BA69000E946F500E9E
:102FD000956FC30E966F470E976F000E0001FC6F42
:102FE00080D1FC51020D530EF324D96E030EF42050
:102FF000DA6EDECFEBF0DDCFECF0EBC06CF0ECC0C6
:103000006DF06E6B6F6B000E6AEC4AF06CC07AF07C
:103010006DC07BF06EC07CF06FC07DF011EC70F085
:103020007AC09BF07BC09CF07CC09DF07DC09EF080
:1030300068C16CF069C16DF000016E6B6F6B000EC2
:103040006AEC4AF06CC097F06DC098F06EC099F0D1
:103050006FC09AF0A8EC36F097C082F098C083F069
:1030600099C084F09AC085F00001FC51020D530E06
:10307000F324D96E030EF420DA6EDECFEDF0DDCF4F
:10308000EEF0EDC06CF0EEC06DF06E6B6F6B000E8D
:103090006AEC4AF06CC07AF06DC07BF06EC07CF0D8
:1030A0006FC07DF011EC70F07AC09BF07BC09CF09B
:1030B0007CC09DF07DC09EF068C16CF069C16DF070
:1030C00000016E6B6F6B000E6AEC4AF06CC097F0FB
:1030D0006DC098F06EC099F06FC09AF0A8EC36F011
:1030E00097C07EF098C07FF099C080F09AC081F0C0
:1030F000FFEC34F07EC0F4F17FC0F5F180C0F6F152
:1031000081C0F7F10001FC51020D500EF324D96E7D
:10311000040EF420DA6EDECFEBF0DDCFECF0EBC086
:103120006CF0ECC06DF06E6B6F6B000E6AEC4AF0E9
:103130006CC07AF06DC07BF06EC07CF06FC07DF02B
:1031400011EC70F07AC09BF07BC09CF07CC09DF0CD
:103150007DC09EF06EC16CF06FC16DF000016E6BB2
:103160006F6B000E6AEC4AF06CC097F06DC098F07F
:103170006EC099F06FC09AF0A8EC36F097C082F05C
:1031800098C083F099C084F09AC085F00001FC518A
:10319000020D500EF324D96E040EF420DA6EDECF49
:1031A000EDF0DDCFEEF0EDC06CF0EEC06DF06E6BCB
:1031B0006F6B000E6AEC4AF06CC07AF06DC07BF069
:1031C0006EC07CF06FC07DF011EC70F07AC09BF0A7
:1031D0007BC09CF07CC09DF07DC09EF06EC16CF009
:1031E0006FC16DF000016E6B6F6B000E6AEC4AF000
:1031F0006CC097F06DC098F06EC099F06FC09AF0F7
:10320000A8EC36F097C07EF098C07FF099C080F0AF
:103210009AC081F0FFEC34F07EC0F8F17FC0F9F184
:1032200080C0FAF181C0FBF1F4C197F0F5C198F0CC
:10323000F6C199F0F7C19AF0F8C19BF0F9C19CF082
:10324000FAC19DF0FBC19EF0A8EC36F097C0ABF040
:1032500098C0ACF099C0ADF09AC0AEF0C4EC39F0B3
:103260000001FC51040D000EF324D96E040EF4206D
:10327000DA6EABC0DEFFACC0DEFFADC0DEFFAEC0BD
:10328000DEFFFC51040D000EF324D96E040EF42071
:10329000DA6EDECFABF0DECFACF0DECFADF0DECF5E
:1032A000AEF094C1AFF095C1B0F096C1B1F097C146
:1032B000B2F092EC50F00001D8B012D0FC51040DE5
:1032C000000EF324D96E040EF420DA6EDECF94F1F2
:1032D000DECF95F1DECF96F1DECF97F1FCC0BAF1EB
:1032E000FC2B01014C510001FC5DD8A07AD60101F4
:1032F000BA51020D530EF324D96E030EF420DA6E88
:10330000DECFEBF0DDCFECF0EBC06CF0ECC06DF09D
:1033100000016E6B6F6B000E6AEC4AF06CC07AF0C5
:103320006DC07BF06EC07CF06FC07DF011EC70F072
:103330007AC09BF07BC09CF07CC09DF07DC09EF06D
:1033400068C16CF069C16DF000016E6B6F6B000EAF
:103350006AEC4AF06CC097F06DC098F06EC099F0BE
:103360006FC09AF0A8EC36F097C082F098C083F056
:1033700099C084F09AC085F00101BA51020D530E34
:10338000F324D96E030EF420DA6EDECFEDF0DDCF3C
:10339000EEF0EDC06CF0EEC06DF000016E6B6F6B87
:1033A000000E6AEC4AF06CC07AF06DC07BF06EC023
:1033B0007CF06FC07DF011EC70F07AC09BF07BC0A8
:1033C0009CF07CC09DF07DC09EF068C16CF069C12E
:1033D0006DF000016E6B6F6B000E6AEC4AF06CC012
:1033E00097F06DC098F06EC099F06FC09AF0A8EC9D
:1033F00036F097C07EF098C07FF099C080F09AC0F8
:1034000081F0FFEC34F07EC0F4F17FC0F5F180C0B4
:10341000F6F181C0F7F10101BA51020D500EF3240B
:10342000D96E040EF420DA6EDECFEBF0DDCFECF0D7
:10343000EBC06CF0ECC06DF000016E6B6F6B000EBA
:103440006AEC4AF06CC07AF06DC07BF06EC07CF024
:103450006FC07DF011EC70F07AC09BF07BC09CF0E7
:103460007CC09DF07DC09EF06EC16CF06FC16DF0B0
:1034700000016E6B6F6B000E6AEC4AF06CC097F047
:103480006DC098F06EC099F06FC09AF0A8EC36F05D
:1034900097C082F098C083F099C084F09AC085F0FC
:1034A0000101BA51020D500EF324D96E040EF4201E
:1034B000DA6EDECFEDF0DDCFEEF0EDC06CF0EEC0F9
:1034C0006DF000016E6B6F6B000E6AEC4AF06CC021
:1034D0007AF06DC07BF06EC07CF06FC07DF011ECB7
:1034E00070F07AC09BF07BC09CF07CC09DF07DC0EA
:1034F0009EF06EC16CF06FC16DF000016E6B6F6B72
:10350000000E6AEC4AF06CC097F06DC098F06EC087
:1035100099F06FC09AF0A8EC36F097C07EF098C092
:103520007FF099C080F09AC081F0FFEC34F07EC04B
:10353000F8F17FC0F9F180C0FAF181C0FBF1F4C16C
:1035400097F0F5C198F0F6C199F0F7C19AF0F8C17B
:103550009BF0F9C19CF0FAC19DF0FBC19EF0A8EC74
:1035600036F097C0ABF098C0ACF099C0ADF09AC0FF
:10357000AEF0C4EC39F0ABC040F1ACC041F1ADC02D
:1035800042F1AEC043F15DC26CF05EC26DF000016D
:103590006E6B6F6B000E6AEC4AF06CC0ABF06DC0E6
:1035A000ACF06EC0ADF06FC0AEF044C1AFF045C13D
:1035B000B0F046C1B1F047C1B2F092EC50F000015A
:1035C000D8A0120044C1ABF045C1ACF046C1ADF08B
:1035D00047C1AEF040C1AFF041C1B0F042C1B1F05F
:1035E00043C1B2F092EC50F00001D8B0120044C1D7
:1035F000ABF045C1ACF046C1ADF047C1AEF048C13B
:10360000AFF049C1B0F04AC1B1F04BC1B2F092EC99
:1036100050F00001D8B0120048C1ABF049C1ACF085
:103620004AC1ADF04BC1AEF040C1AFF041C1B0F006
:1036300042C1B1F043C1B2F092EC50F00001D8A009
:1036400060D368C16CF069C16DF06E6B6F6B000E7A
:103650006AEC4AF06CC07AF06DC07BF06EC07CF012
:103660006FC07DF011EC70F07AC09BF07BC09CF0D5
:103670007CC09DF07DC09EF06AC16CF06BC16DF0A6
:1036800000016E6B6F6B000E6AEC4AF06CC097F035
:103690006DC098F06EC099F06FC09AF0A8EC36F04B
:1036A00097C082F098C083F099C084F09AC085F0EA
:1036B00068C16CF069C16DF000016E6B6F6B000E3C
:1036C0006AEC4AF06CC07AF06DC07BF06EC07CF0A2
:1036D0006FC07DF011EC70F07AC09BF07BC09CF065
:1036E0007CC09DF07DC09EF06AC16CF06BC16DF036
:1036F00000016E6B6F6B000E6AEC4AF06CC097F0C5
:103700006DC098F06EC099F06FC09AF0A8EC36F0DA
:1037100097C07EF098C07FF099C080F09AC081F089
:10372000FFEC34F07EC0F4F17FC0F5F180C0F6F11B
:1037300081C0F7F16EC16CF06FC16DF000016E6B6E
:103740006F6B000E6AEC4AF06CC07AF06DC07BF0D3
:103750006EC07CF06FC07DF011EC70F07AC09BF011
:103760007BC09CF07CC09DF07DC09EF070C16CF071
:1037700071C16DF000016E6B6F6B000E6AEC4AF068
:103780006CC097F06DC098F06EC099F06FC09AF061
:10379000A8EC36F097C082F098C083F099C084F00E
:1037A0009AC085F06EC16CF06FC16DF000016E6B58
:1037B0006F6B000E6AEC4AF06CC07AF06DC07BF063
:1037C0006EC07CF06FC07DF011EC70F07AC09BF0A1
:1037D0007BC09CF07CC09DF07DC09EF070C16CF001
:1037E00071C16DF000016E6B6F6B000E6AEC4AF0F8
:1037F0006CC097F06DC098F06EC099F06FC09AF0F1
:10380000A8EC36F097C07EF098C07FF099C080F0A9
:103810009AC081F0FFEC34F07EC0F8F17FC0F9F17E
:1038200080C0FAF181C0FBF1F4C197F0F5C198F0C6
:10383000F6C199F0F7C19AF0F8C19BF0F9C19CF07C
:10384000FAC19DF0FBC19EF0A8EC36F097C0ABF03A
:1038500098C0ACF099C0ADF09AC0AEF0C4EC39F0AD
:10386000ABC090F1ACC091F1ADC092F1AEC093F19C
:1038700040C19BF041C19CF042C19DF043C19EF00C
:1038800044C17AF045C17BF046C17CF047C17DF070
:1038900011EC70F07AC097F07BC098F07CC099F082
:1038A0007DC09AF0A8EC36F097C0F4F198C0F5F11D
:1038B00099C0F6F19AC0F7F144C19BF045C19CF064
:1038C00046C19DF047C19EF090C17AF091C17BF056
:1038D00092C17CF093C17DF011EC70F07AC097F04A
:1038E0007BC098F07CC099F07DC09AF0A8EC36F0CF
:1038F00097C0F8F198C0F9F199C0FAF19AC0FBF1BC
:1039000044C19BF045C19CF046C19DF047C19EF06B
:1039100040C17AF041C17BF042C17CF043C17DF0EF
:1039200011EC70F07AC097F07BC098F07CC099F0F1
:103930007DC09AF0A8EC36F097C0E0F198C0E1F1B4
:1039400099C0E2F19AC0E3F190C19BF091C19CF063
:1039500092C19DF093C19EF0F4C197F0F5C198F02B
:10396000F6C199F0F7C19AF0A8EC36F097C082F052
:1039700098C083F099C084F09AC085F040C19BF054
:1039800041C19CF042C19DF043C19EF0F8C197F047
:10399000F9C198F0FAC199F0FBC19AF0A8EC36F0A1
:1039A00097C07EF098C07FF099C080F09AC081F0F7
:1039B000FFEC34F07EC0E4F17FC0E5F180C0E6F1B9
:1039C00081C0E7F140C19BF041C19CF042C19DF034
:1039D00043C19EF044C197F045C198F046C199F0AB
:1039E00047C19AF0A8EC36F097C0E8F198C0E9F129
:1039F00099C0EAF19AC0EBF1E4C182F0E5C183F02D
:103A0000E6C184F0E7C185F090C19BF091C19CF0C4
:103A100092C19DF093C19EF0E0C197F0E1C198F092
:103A2000E2C199F0E3C19AF0A8EC36F097C07EF0BD
:103A300098C07FF099C080F09AC081F0FFEC34F01C
:103A40007EC0ECF17FC0EDF180C0EEF181C0EFF1FE
:103A5000ECC182F0EDC183F0EEC184F0EFC185F0DE
:103A600090C19BF091C19CF092C19DF093C19EF0DA
:103A7000E8C197F0E9C198F0EAC199F0EBC19AF07A
:103A8000A8EC36F097C07EF098C07FF099C080F027
:103A90009AC081F0FFEC34F07EC0ABF07FC0ACF098
:103AA00080C0ADF081C0AEF0C4EC39F0ABC0C8F05E
:103AB000ACC0C9F0ADC0CAF0AEC0CBF0000E000182
:103AC000CC6F000ECD6F000ECE6F400ECF6F28EC86
:103AD0003BF0C8C08CF1C9C08DF1CAC08EF1CBC01B
:103AE0008FF18CC1C8F08DC1C9F08EC1CAF08FC1F1
:103AF000CBF090C1CCF091C1CDF092C1CEF093C18A
:103B0000CFF028EC3BF0C8C08CF1C9C08DF1CAC021
:103B10008EF1CBC08FF144C182F045C183F046C124
:103B200084F047C185F044C17EF045C17FF046C1B5
:103B300080F047C181F0FFEC34F07EC097F07FC089
:103B400098F080C099F081C09AF08CC182F08DC14C
:103B500083F08EC184F08FC185F08CC17EF08DC161
:103B60007FF08EC180F08FC181F0FFEC34F07EC019
:103B70007AF07FC07BF080C07CF081C07DF011ECDA
:103B800070F07AC09BF07BC09CF07CC09DF07DC043
:103B90009EF0A8EC36F097C0ABF098C0ACF099C09E
:103BA000ADF09AC0AEF0C4EC39F0ABC094F1ACC04B
:103BB00095F1ADC096F1AEC097F144C19BF045C1FF
:103BC0009CF046C19DF047C19EF08CC17AF08DC13A
:103BD0007BF08EC17CF08FC17DF011EC70F07AC06B
:103BE00097F07BC098F07CC099F07DC09AF0A8EC6B
:103BF00036F097C0F0F198C0F1F199C0F2F19AC097
:103C0000F3F1F0C17EF0F1C17FF0F2C180F0F3C1B9
:103C100081F0CDEC6EF07EC0ABF07FC0ACF080C028
:103C2000ADF081C0AEF06F0E0001AF6F120EB06F3D
:103C3000830EB16F3A0EB26F92EC50F00001D8B023
:103C400009D0000E0101946F000E956F000E966F63
:103C5000000E976FBAC1BBF190C1CCF091C1CDF00D
:103C600092C1CEF093C1CFF0000E0001826F000E22
:103C7000836FC80E846F420E856F94C17EF095C12C
:103C80007FF096C180F097C181F0FFEC34F07EC0E8
:103C9000C8F07FC0C9F080C0CAF081C0CBF028EC6A
:103CA0003BF0C8C09BF0C9C09CF0CAC09DF0CBC01F
:103CB0009EF004C26CF005C26DF006C26EF007C241
:103CC0006FF0000E6AEC4AF06CC097F06DC098F08F
:103CD0006EC099F06FC09AF0A8EC36F097C0E1F092
:103CE00098C0E2F099C0E3F09AC0E4F0A0EC5CF078
:103CF000E1C01EF2E2C01FF2E3C020F2E4C021F2F4
:103D0000120048C1ABF049C1ACF04AC1ADF04BC1A3
:103D1000AEF040C1AFF041C1B0F042C1B1F043C11B
:103D2000B2F092EC50F00001D8B012006CC16CF00F
:103D30006DC16DF06E6B6F6B000E6AEC4AF06CC07B
:103D40007AF06DC07BF06EC07CF06FC07DF011EC3E
:103D500070F07AC09BF07BC09CF07CC09DF07DC071
:103D60009EF06AC16CF06BC16DF000016E6B6F6B01
:103D7000000E6AEC4AF06CC097F06DC098F06EC00F
:103D800099F06FC09AF0A8EC36F097C082F098C016
:103D900083F099C084F09AC085F06CC16CF06DC15D
:103DA0006DF000016E6B6F6B000E6AEC4AF06CC038
:103DB0007AF06DC07BF06EC07CF06FC07DF011ECCE
:103DC00070F07AC09BF07BC09CF07CC09DF07DC001
:103DD0009EF06AC16CF06BC16DF000016E6B6F6B91
:103DE000000E6AEC4AF06CC097F06DC098F06EC09F
:103DF00099F06FC09AF0A8EC36F097C07EF098C0AA
:103E00007FF099C080F09AC081F0FFEC34F07EC062
:103E1000F4F17FC0F5F180C0F6F181C0F7F172C115
:103E20006CF073C16DF000016E6B6F6B000E6AEC8D
:103E30004AF06CC07AF06DC07BF06EC07CF06FC051
:103E40007DF011EC70F07AC09BF07BC09CF07CC0E0
:103E50009DF07DC09EF070C16CF071C16DF00001ED
:103E60006E6B6F6B000E6AEC4AF06CC097F06DC021
:103E700098F06EC099F06FC09AF0A8EC36F097C039
:103E800082F098C083F099C084F09AC085F072C126
:103E90006CF073C16DF000016E6B6F6B000E6AEC1D
:103EA0004AF06CC07AF06DC07BF06EC07CF06FC0E1
:103EB0007DF011EC70F07AC09BF07BC09CF07CC070
:103EC0009DF07DC09EF070C16CF071C16DF000017D
:103ED0006E6B6F6B000E6AEC4AF06CC097F06DC0B1
:103EE00098F06EC099F06FC09AF0A8EC36F097C0C9
:103EF0007EF098C07FF099C080F09AC081F0FFEC0E
:103F000034F07EC0F8F17FC0F9F180C0FAF181C0D1
:103F1000FBF1F4C197F0F5C198F0F6C199F0F7C143
:103F20009AF0F8C19BF0F9C19CF0FAC19DF0FBC179
:103F30009EF0A8EC36F097C0ABF098C0ACF099C0FA
:103F4000ADF09AC0AEF0C4EC39F0ABC090F1ACC0AB
:103F500091F1ADC092F1AEC093F148C19BF049C15F
:103F60009CF04AC19DF04BC19EF044C17AF045C11E
:103F70007BF046C17CF047C17DF011EC70F07AC057
:103F800097F07BC098F07CC099F07DC09AF0A8ECC7
:103F900036F097C0F4F198C0F5F199C0F6F19AC0E7
:103FA000F7F148C19BF049C19CF04AC19DF04BC15B
:103FB0009EF090C17AF091C17BF092C17CF093C1E8
:103FC0007DF011EC70F07AC097F07BC098F07CC067
:103FD00099F07DC09AF0A8EC36F097C0F8F198C03F
:103FE000F9F199C0FAF19AC0FBF144C19BF045C1C7
:103FF0009CF046C19DF047C19EF048C17AF049C18E
:104000007BF04AC17CF04BC17DF011EC70F07AC0BE
:1040100097F07BC098F07CC099F07DC09AF0A8EC36
:1040200036F097C0E0F198C0E1F199C0E2F19AC092
:10403000E3F190C19BF091C19CF092C19DF093C1BE
:104040009EF0F4C197F0F5C198F0F6C199F0F7C170
:104050009AF0A8EC36F097C082F098C083F099C02F
:1040600084F09AC085F044C19BF045C19CF046C1E4
:104070009DF047C19EF0F8C197F0F9C198F0FAC1E0
:1040800099F0FBC19AF0A8EC36F097C07EF098C08A
:104090007FF099C080F09AC081F0FFEC34F07EC0D0
:1040A000E4F17FC0E5F180C0E6F181C0E7F144C1F1
:1040B0009BF045C19CF046C19DF047C19EF048C1B0
:1040C00097F049C198F04AC199F04BC19AF0A8EC19
:1040D00036F097C0E8F198C0E9F199C0EAF19AC0CA
:1040E000EBF1E4C182F0E5C183F0E6C184F0E7C101
:1040F00085F090C19BF091C19CF092C19DF093C15D
:104100009EF0E0C197F0E1C198F0E2C199F0E3C1FF
:104110009AF0A8EC36F097C07EF098C07FF099C076
:1041200080F09AC081F0FFEC34F07EC0ECF17FC0EB
:10413000EDF180C0EEF181C0EFF1ECC182F0EDC194
:1041400083F0EEC184F0EFC185F090C19BF091C186
:104150009CF092C19DF093C19EF0E8C197F0E9C137
:1041600098F0EAC199F0EBC19AF0A8EC36F097C04C
:104170007EF098C07FF099C080F09AC081F0FFEC8B
:1041800034F07EC0ABF07FC0ACF080C0ADF081C039
:10419000AEF0C4EC39F0ABC0C8F0ACC0C9F0ADC0F3
:1041A000CAF0AEC0CBF0000E0001CC6F000ECD6F98
:1041B000000ECE6F400ECF6F28EC3BF0C8C08CF1E4
:1041C000C9C08DF1CAC08EF1CBC08FF18CC1C8F0CF
:1041D0008DC1C9F08EC1CAF08FC1CBF090C1CCF0B7
:1041E00091C1CDF092C1CEF093C1CFF028EC3BF05D
:1041F000C8C08CF1C9C08DF1CAC08EF1CBC08FF19F
:1042000044C182F045C183F046C184F047C185F0C6
:1042100044C17EF045C17FF046C180F047C181F0C6
:10422000FFEC34F07EC097F07FC098F080C099F02A
:1042300081C09AF08CC182F08DC183F08EC184F070
:104240008FC185F08CC17EF08DC17FF08EC180F072
:104250008FC181F0FFEC34F07EC07AF07FC07BF03C
:1042600080C07CF081C07DF011EC70F07AC09BF0D2
:104270007BC09CF07CC09DF07DC09EF0A8EC36F029
:1042800097C0ABF098C0ACF099C0ADF09AC0AEF05A
:10429000C4EC39F0ABC094F1ACC095F1ADC096F16F
:1042A000AEC097F144C19BF045C19CF046C19DF062
:1042B00047C19EF08CC17AF08DC17BF08EC17CF03D
:1042C0008FC17DF011EC70F07AC097F07BC098F050
:1042D0007CC099F07DC09AF0A8EC36F097C0F0F160
:1042E00098C0F1F199C0F2F19AC0F3F1F0C17EF0FB
:1042F000F1C17FF0F2C180F0F3C181F0CDEC6EF03E
:104300007EC0ABF07FC0ACF080C0ADF081C0AEF03D
:104310006F0E0001AF6F120EB06F830EB16F3A0EC9
:10432000B26F92EC50F00001D8B009D0000E01013C
:10433000946F000E956F000E966F000E976FBAC1C6
:10434000BBF190C1CCF091C1CDF092C1CEF093C140
:10435000CFF0000E0001826F000E836FC80E846FD5
:10436000420E856F94C17EF095C17FF096C180F0BA
:1043700097C181F0FFEC34F07EC0C8F07FC0C9F077
:1043800080C0CAF081C0CBF028EC3BF0C8C07AF006
:10439000C9C07BF0CAC07CF0CBC07DF011EC70F0DE
:1043A0007AC09BF07BC09CF07CC09DF07DC09EF0ED
:1043B00004C26CF005C26DF006C26EF007C26FF069
:1043C000000E6AEC4AF06CC097F06DC098F06EC0B9
:1043D00099F06FC09AF0A8EC36F097C0E1F098C061
:1043E000E2F099C0E3F09AC0E4F0A0EC5CF0E1C028
:1043F0001EF2E2C01FF2E3C020F2E4C021F212007C
:10440000000E0101C06F000E0001FB6F4D0E040194
:104410007C19D8A4F7D3430E7D19D8B403D0F2D3B6
:104420000001FB2B0001FB51010D780EF324D96E26
:10443000040EF420DA6E2C0EDE18D8A4F1D7FB2B74
:10444000FB51010D780EF324D96E040EF420DA6EC0
:104450002C0EDE18D8A4F3D7FB2BFB51010D780EE0
:10446000F324D96E040EF420DA6EDF500101C06F20
:10447000410EC019D8A405D00201AC810101CD853F
:1044800007D00201AC910101CD9502D00001FB2BB8
:104490000001FB51010D780EF324D96E040EF420B7
:1044A000DA6E2C0EDE18D8A4F1D7FB2B000EFC6FB1
:1044B000030EFC6501D00CD0FC51010DC20EF3249B
:1044C000D96E020EF420DA6E780EDF6EFC2BF0D778
:1044D000780EFB25D96EDA6A040EDA22DF5002016B
:1044E000C26F0001FB51F16FF26B010EF127000E5C
:1044F000F223780EF125D96E040EF221DA6EDF5028
:104500000201C36FC20E00016C6F020E6D6F54EC9E
:1045100055F06CC0F3F06DC0F4F06EC0F5F06FC0F4
:10452000F6F0F3C060F0F4C061F0F5C062F0F6C0E0
:1045300063F0400E0001646F420E656F0F0E666FF0
:10454000000E676F0FEC6DF060C0ADF261C0AEF2AF
:1045500062C0AFF263C0B0F2020E0001FB27000E92
:10456000FC6F080EFC6501D00CD0FC51010DC20E91
:10457000F324D96E020EF420DA6E780EDF6EFC2B77
:10458000F0D7780EFB25D96EDA6A040EDA22DF50F6
:104590000201C26F0001FB51F16FF26B010EF127B6
:1045A000000EF223780EF125D96E040EF221DA6E98
:1045B000DF500201C36F0001FB51F16FF26B030E7C
:1045C000F127000EF223780EF125D96E040EF221A8
:1045D000DA6EDF500201C46F0001FB51F16FF26B24
:1045E000040EF127000EF223780EF125D96E040E89
:1045F000F221DA6EDF500201C56F0001FB51F16F4D
:10460000F26B050EF127000EF223780EF125D96E1C
:10461000040EF221DA6EDF500201C66F0001FB5179
:10462000F16FF26B060EF127000EF223780EF125E2
:10463000D96E040EF221DA6EDF500201C76F01015C
:10464000C3A122D00001FB51F16FF26B070EF127DD
:10465000000EF223780EF125D96E040EF221DA6EE7
:10466000DF500201C86F0001FB51F16FF26B080EC1
:10467000F127000EF223780EF125D96E040EF221F7
:10468000DA6EDF50020104D0300E0201C86F300E26
:10469000C96FC20E00016C6F020E6D6F54EC55F0C5
:1046A0006CC042F26DC043F26EC044F26FC045F27E
:1046B00042C260F043C261F044C262F045C263F09E
:1046C0003C0E0001646F000E656F000E666F000EF9
:1046D000676FFAEC5FF060C042F261C043F262C003
:1046E00044F263C045F202014251AD274351AE236B
:1046F0004451AF234551B02302D00001FB2B0001F0
:10470000FB51010D780EF324D96E040EF420DA6EFD
:104710002C0EDE18D8A4F1D7FB2BFB51010D780E1F
:10472000F324D96E040EF420DA6EDF500101C06F5D
:104730004E0EC019D8A403D00201AC9705D00201D7
:10474000AC8702D00001FB2B0001FB51010D780E5C
:10475000F324D96E040EF420DA6E2C0EDE18D8A4E1
:10476000F1D7FB2B000EFC6F040EFC6501D00CD0C2
:10477000FC51010DC20EF324D96E020EF420DA6E44
:10478000780EDF6EFC2BF0D7780EFB25D96EDA6A37
:10479000040EDA22DF500201C26F0001FB51F16FFB
:1047A000F26B010EF127000EF223780EF125D96E7F
:1047B000040EF221DA6EDF500201C36F0001FB51DB
:1047C000F16FF26B020EF127000EF223780EF12545
:1047D000D96E040EF221DA6EDF500201C46FC20EF0
:1047E00000016C6F020E6D6F54EC55F06CC0F3F06D
:1047F0006DC0F4F06EC0F5F06FC0F6F0F3C060F07D
:10480000F4C061F0F5C062F0F6C063F0400E000144
:10481000646F420E656F0F0E666F000E676F0FECD0
:104820006DF060C0B1F261C0B2F262C0B3F263C0B9
:10483000B4F2030E0001FB27000EFC6F080EFC65AE
:1048400001D00CD0FC51010DC20EF324D96E020E22
:10485000F420DA6E780EDF6EFC2BF0D7780EFB2595
:10486000D96EDA6A040EDA22DF500201C26F00014B
:10487000FB51F16FF26B010EF127000EF223780E5F
:10488000F125D96E040EF221DA6EDF500201C36FFA
:104890000001FB51F16FF26B030EF127000EF223C2
:1048A000780EF125D96E040EF221DA6EDF50020186
:1048B000C46F0001FB51F16FF26B040EF127000E83
:1048C000F223780EF125D96E040EF221DA6EDF5054
:1048D0000201C56F0001FB51F16FF26B050EF1276C
:1048E000000EF223780EF125D96E040EF221DA6E55
:1048F000DF500201C66F0001FB51F16FF26B060E33
:10490000F127000EF223780EF125D96E040EF22164
:10491000DA6EDF500201C76F0101C3A122D000018E
:10492000FB51F16FF26B070EF127000EF223780EA8
:10493000F125D96E040EF221DA6EDF500201C86F44
:104940000001FB51F16FF26B080EF127000EF2230C
:10495000780EF125D96E040EF221DA6EDF500201D5
:1049600004D0300E0201C86F300EC96FC20E0001B4
:104970006C6F020E6D6F54EC55F06CC042F26DC05E
:1049800043F26EC044F26FC045F242C260F043C2CF
:1049900061F044C262F045C263F03C0E0001646FF6
:1049A000000E656F000E666F000E676FFAEC5FF029
:1049B00060C042F261C043F262C044F263C045F29B
:1049C00002014251B1274351B2234451B32345510F
:1049D000B42302D00001FB2B0001FB51010D780E26
:1049E000F324D96E040EF420DA6E2C0EDE18D8A44F
:1049F000F1D7FB2BFB51010D780EF324D96E040E79
:104A0000F420DA6EDF500101C06F450EC019D8A442
:104A100003D00201AC9505D00201AC8502D00001A3
:104A2000FB2B0001FB51010D780EF324D96E040E0F
:104A3000F420DA6E2C0EDE18D8A4F1D7FB2BFB5134
:104A4000010D780EF324ED6F040EF420EE6F09ECE7
:104A500071F0EDC094F1EEC095F1EFC096F1F0C0A9
:104A600097F194C1ABF095C1ACF096C1ADF097C190
:104A7000AEF0000E0001AF6F000EB06F180EB16FF8
:104A8000430EB26F92EC50F00001D8B049D0000E46
:104A9000826F000E836FC80E846F420E856F94C1C3
:104AA0007EF095C17FF096C180F097C181F0FFEC58
:104AB00034F07EC0E1F07FC0E2F080C0E3F081C05E
:104AC000E4F0A0EC5CF0E1C0B7F2E2C0B8F294C14F
:104AD0007EF095C17FF096C180F097C181F0560EAF
:104AE0000001826F0E0E836FED0E846F3F0E856F97
:104AF000FFEC34F07EC094F17FC095F180C096F158
:104B000081C097F194C1E1F095C1E2F096C1E3F064
:104B100097C1E4F0A0EC5CF0E1C0B5F2E2C0B6F2FF
:104B20000101C5930201B65112E1140EB55DD8B072
:104B30000ED00101C5830201614B622B710E615DD4
:104B4000170E6259D8A015D00101C58112D00101FC
:104B5000C591000E0201626F000E616F000E3E6F84
:104B6000000E3F6F000E406F000E416F02D000013B
:104B7000FB2B0001FB51010D780EF324D96E040EBE
:104B8000F420DA6E2C0EDE18D8A4F1D7FB2BFB51E3
:104B9000010D780EF324ED6F040EF420EE6F09EC96
:104BA00071F0EDC094F1EEC095F1EFC096F1F0C058
:104BB00097F194C17EF095C17FF096C180F097C1C6
:104BC00081F0000E0001826F000E836FC80E846FAB
:104BD000420E856FFFEC34F07EC094F17FC095F1FA
:104BE00080C096F181C097F194C1E1F095C1E2F0E7
:104BF00096C1E3F097C1E4F0A0EC5CF0E1C0B9F23B
:104C0000E2C0BAF225B427BC89D027B687D001010B
:104C1000AB51AC11D8B405D0AB07D8A0AC072796E0
:104C20007DD0AFEC71F0000E0001FB6F01D0FB2BCB
:104C3000FB51010D780EF324D96E040EF420DA6EC8
:104C40002C0EDE18D8A4F3D7FB2B000E0101AC6F9D
:104C5000000EAB6F16D00001FB51010D780EF3244E
:104C6000D96E040EF420DA6ECE0E0101AB25E16E92
:104C7000020EAC21E26EDFCFE7FFAB4BAC2B0001A5
:104C8000FB2B0101AC5104E1040EAB5DD8A0E3D7CE
:104C9000CE0EAB25D96E020EAC21DA6E2C0EDF6E75
:104CA000AB4BAC2B000E0201C26F000E0001FB6F7C
:104CB00010D00001FB2BFB51010D780EF324D96EAF
:104CC000040EF420DA6E2C0EDE18D8A402D00201F5
:104CD000C22B090E0201C219D8A4EBD714D00001CF
:104CE000FB51010D780EF324D96E040EF420DA6E18
:104CF000CE0E0101AB25E16E020EAC21E26EDFCFDC
:104D0000E7FFAB4BAC2B0001FB2B0101AC5104E1E5
:104D10000B0EAB5DD8A0E3D7278612009FEC70F096
:104D20001200000E0001F36F0101BB51D8A432D173
:104D3000EBC084F1ECC085F1EDC086F1EEC087F1E7
:104D40000001EB51020112270001EC510201132373
:104D50000001ED51020114230001EE51020115235F
:104D600012C288F113C289F114C28AF115C28BF103
:104D70000001FA2B0DD0FA2BFA51040DC50EF324C5
:104D8000D96E030EF420DA6EDE6ADE6ADE6ADD6A50
:104D900001014C510001FA5DD8A0EDD7FA51040D84
:104DA000C50EF324D96E030EF420DA6E84C1DEFF43
:104DB00085C1DEFF86C1DEFF87C1DEFF12C2C5F3FB
:104DC00013C2C6F314C2C7F315C2C8F32682212A40
:104DD000000E0201126F000E136F000E146F000E12
:104DE000156F0001FA51040D000EF324D96E030E65
:104DF000F420DA6EDECFEFF0DECFF0F0DECFF1F0B0
:104E0000DECFF2F0EF1FF01FF11FF21FEF2B000EAD
:104E1000F023F123F223010184510001EF25010168
:104E2000806F85510001F0210101816F86510001E1
:104E3000F1210101826F87510001F2210101836F8D
:104E400000C3EFF001C3F0F002C3F1F003C3F2F0CE
:104E50000001EF1FF01FF11FF21FEF2B000EF023D8
:104E6000F123F223010188510001EF250D6E0101AC
:104E700089510001F0210E6E01018A510001F121DA
:104E80000F6E01018B510001F221106E0DC07CF1FB
:104E90000EC07DF10FC07EF110C07FF10301005103
:104EA0000101885D0301015101018959030102518A
:104EB00001018A590301035101018B59D8B023D054
:104EC000000E0001F36F1AD00001F351040DC50E5E
:104ED000F324D96E030EF420DA6EF351040D000EA4
:104EE000F324E16E030EF420E26EDECFE6FFDECFA8
:104EF000E6FFDECFE6FFDECFE6FFF32BF351010145
:104F00004C5DD8B0E1D702011A510101885D020160
:104F10001B510101895902011C5101018A590201E9
:104F20001D5101018B59D8B00AD088C11AF289C12C
:104F30001BF28AC11CF28BC11DF221C020F00201BC
:104F400016510101885D02011751010189590201C1
:104F5000185101018A590201195101018B59D8B028
:104F600013D088C116F289C117F28AC118F28BC119
:104F700019F259C25BF25AC25CF221C0B2F1000EC2
:104F800002015A6F000E596F000E0001FA6FACD08B
:104F9000000E12000001FA5101014C5DD8A0F8D7B3
:104FA000EBC084F1ECC085F1EDC086F1EEC087F175
:104FB0000001EB51020112270001EC510201132301
:104FC0000001ED51020114230001EE5102011523ED
:104FD0000001FA2BFA51040DC50EF324D96E030E0D
:104FE000F420DA6E84C1DEFF85C1DEFF86C1DEFFFC
:104FF00087C1DEFFFA51040D000EF324D96E030EB3
:10500000F420DA6EDECFEFF0DECFF0F0DECFF1F09D
:10501000DECFF2F0EF1FF01FF11FF21FEF2B000E9B
:10502000F023F123F223010184510001EF25010156
:10503000806F85510001F0210101816F86510001CF
:10504000F1210101826F87510001F2210101836F7B
:10505000000E7C6F000E7D6F000E7E6F000E7F6F66
:10506000010E0001F36F13D0F351040D000EF32471
:10507000D96E030EF420DA6EDE5001017C27DE507B
:105080007D23DE507E23DD507F230001F32BF3517F
:10509000FA5DD8B0E9D77CC1EFF07DC1F0F07EC1F8
:1050A000F1F07FC1F2F0EF1FF01FF11FF21FEF2BA5
:1050B000000EF023F123F223020112510001EF252B
:1050C00001017C6F020113510001F02101017D6F8C
:1050D000020114510001F12101017E6F02011551FD
:1050E0000001F22101017F6F0101BB51D8B4A3D0AF
:1050F00073D188C15BF189C15CF18AC15DF18BC15B
:105100005EF160D084C15BF185C15CF186C15DF167
:1051100087C15EF127D080C16CF081C16DF082C182
:105120006EF083C16FF0010E6AEC4AF06CC07EF045
:105130006DC07FF06EC080F06FC081F0CDEC6EF07E
:105140007EC0E1F07FC0E2F080C0E3F081C0E4F017
:10515000A0EC5CF0E1C05BF1E2C05CF1E3C05DF1AA
:10516000E4C05EF180C174F181C175F182C176F154
:1051700083C177F171D00DC06CF00EC06DF00FC01F
:105180006EF010C06FF0010E6AEC4AF06CC07EF059
:105190006DC07FF06EC080F06FC081F0CDEC6EF01E
:1051A0007EC0E1F07FC0E2F080C0E3F081C0E4F0B7
:1051B000A0EC5CF0E1C05BF1E2C05CF1E3C05DF14A
:1051C000E4C05EF10DC074F10EC075F10FC076F150
:1051D00010C077F141D07CC16CF07DC16DF07EC113
:1051E0006EF07FC16FF0010E6AEC4AF06CC07EF089
:1051F0006DC07FF06EC080F06FC081F0CDEC6EF0BE
:105200007EC0E1F07FC0E2F080C0E3F081C0E4F056
:10521000A0EC5CF0E1C05BF1E2C05CF1E3C05DF1E9
:10522000E4C05EF17CC174F17DC175F17EC176F19F
:105230007FC177F111D002019B51010AD8B459D72F
:10524000030AD8B45FD7010AD8B465D7070AD8B41F
:1052500092D7010AD8B4BFD7010177BF07D07751E1
:105260007611751108E17405D8B005D01F941F8818
:105270000E01E589E597010177BF0CD077517611D2
:10528000751103E17405D8A005D01F841F980E0185
:10529000E599E5871F8E000E0101B16FBDEC49F065
:1052A00018EC59F099D084C15BF185C15CF186C1DD
:1052B0005DF187C15EF127D080C16CF081C16DF0D6
:1052C00082C16EF083C16FF0010E6AEC4AF06CC0CF
:1052D0007EF06DC07FF06EC080F06FC081F0CDECCD
:1052E0006EF07EC0E1F07FC0E2F080C0E3F081C0EC
:1052F000E4F0A0EC5CF0E1C05BF1E2C05CF1E3C083
:105300005DF1E4C05EF180C178F181C179F182C1C3
:105310007AF183C17BF16ED00DC06CF00EC06DF0E0
:105320000FC06EF010C06FF0010E6AEC4AF06CC056
:105330007EF06DC07FF06EC080F06FC081F0CDEC6C
:105340006EF07EC0E1F07FC0E2F080C0E3F081C08B
:10535000E4F0A0EC5CF0E1C05BF1E2C05CF1E3C022
:105360005DF1E4C05EF10DC078F10EC079F10FC0BF
:105370007AF110C07BF13ED07CC16CF07DC16DF044
:105380007EC16EF07FC16FF0010E6AEC4AF06CC016
:105390007EF06DC07FF06EC080F06FC081F0CDEC0C
:1053A0006EF07EC0E1F07FC0E2F080C0E3F081C02B
:1053B000E4F0A0EC5CF0E1C05BF1E2C05CF1E3C0C2
:1053C0005DF1E4C05EF17CC178F17DC179F17EC10F
:1053D0007AF17FC17BF10ED002019A51010AD8B453
:1053E00062D7030AD8B468D7010AD8B495D7070A98
:1053F000D8B4C2D7BDEC49F092EC5FF004D00A0EED
:105400000101FE6F0DD00201A451040AD8B4F7D7F0
:10541000010AD8B4F4D704D00A0E0101FD6F08D0F8
:105420000201A851040AD8B4F7D7010AD8B4F4D7B6
:1054300078C160F079C161F07AC162F07BC163F03C
:1054400074C164F075C165F076C166F077C167F02C
:10545000010E0001686FC3EC69F001017BBF07D04A
:105460007B517A11791108E17805D8B005D01F96E3
:105470001F8A0E01E585E59301017BBF0CD07B51AE
:105480007A11791103E17805D8A005D01F861F9AFB
:105490000E01E595E5831F8C000E0101B16F010E31
:1054A000120000017D6F03D000017A4B7B2B000EB0
:1054B00000017A25D96E070E7B21DA6E2C0EDE18DC
:1054C000D8A4F2D77A4B7B2B40D2000E7A25D96E26
:1054D000070E7B21DA6EDF500201956F1200010E7C
:1054E0000201986F1200000E00017A25666F070E08
:1054F0007B21676F7EEC5DF0000166510201976FC2
:105500001200000E00017A25666F070E7B21676F7F
:105510007EEC5DF0000166510201A06F03D0000136
:105520007A4B7B2B000E00017A25D96E070E7B216A
:10553000DA6E2C0EDE18D8A4F2D77A4B7B2B000E35
:105540007A25666F070E7B21676F7EEC5DF066C083
:10555000A2F267C0A3F203D000017A4B7B2B000EAE
:1055600000017A25D96E070E7B21DA6E2C0EDE182B
:10557000D8A4F2D77A4B7B2B000E7A25666F070EE4
:105580007B21676F7EEC5DF0000166510201A16F27
:105590001200000E00017A25666F070E7B21676FEF
:1055A0007EEC5DF0000166510201A46F03D00001A2
:1055B0007A4B7B2B000E00017A25D96E070E7B21DA
:1055C000DA6E2C0EDE18D8A4F2D77A4B7B2B000EA5
:1055D0007A25666F070E7B21676F7EEC5DF066C0F3
:1055E000A6F267C0A7F203D000017A4B7B2B000E16
:1055F00000017A25D96E070E7B21DA6E2C0EDE189B
:10560000D8A4F2D77A4B7B2B000E7A25666F070E53
:105610007B21676F7EEC5DF0000166510201A56F92
:105620001200000E00017A25666F070E7B21676F5E
:105630007EEC5DF0000166510201A86F03D000010D
:105640007A4B7B2B000E00017A25D96E070E7B2149
:10565000DA6E2C0EDE18D8A4F2D77A4B7B2B000E14
:105660007A25666F070E7B21676F7EEC5DF066C062
:10567000AAF267C0ABF203D000017A4B7B2B000E7D
:1056800000017A25D96E070E7B21DA6E2C0EDE180A
:10569000D8A4F2D77A4B7B2B000E7A25666F070EC3
:1056A0007B21676F7EEC5DF0000166510201A96FFE
:1056B0001200000E00017A25666F070E7B21676FCE
:1056C0007EEC5DF00001665102019A6F1200000E3F
:1056D00000017A25666F070E7B21676F7EEC5DF017
:1056E0000001665102019B6F1200000E0001FC6F69
:1056F0000E0EFC6501D02AD0FC51020D530EF3248E
:10570000D96E030EF420DA6E000EDE6E000EDD6E32
:10571000FC51020D500EF324D96E040EF420DA6E03
:10572000000EDE6E000EDD6EFC51040D000EF32443
:10573000D96E040EF420DA6E000EDE6E000EDE6E00
:10574000000EDE6E000EDD6EFC2BD2D7000E0101C6
:105750004C6F000E00017A256C6F070E7B216D6F78
:1057600054EC55F06CC052F16DC053F16EC054F161
:105770006FC055F103D000017A4B7B2B000E000166
:105780007A25D96E070E7B21DA6E2C0EDE18D8A48E
:10579000F2D77A4B7B2B000E7A256C6F070E7B219C
:1057A0006D6F54EC55F06CC04EF16DC04FF16EC092
:1057B00050F16FC051F103D000017A4B7B2B000EEA
:1057C00000017A25D96E070E7B21DA6E2C0EDE18C9
:1057D000D8A4F2D77A4B7B2B000E7A25666F070E82
:1057E0007B21676F7EEC5DF00001665101014C6F1B
:1057F000000E0001FC6F48D07A4B7B2B000E7A25FF
:10580000D96E070E7B21DA6E2C0EDE18D8A4F4D7E1
:105810007A4B7B2B000E7A25666F070E7B21676F14
:105820007EEC5DF00001FC51020D530EF324D96EA5
:10583000030EF420DA6E66C0DEFF67C0DDFF02D023
:105840007A4B7B2B000E7A25D96E070E7B21DA6E00
:105850002C0EDE18D8A4F4D77A4B7B2B000E7A25B9
:10586000666F070E7B21676F7EEC5DF00001FC51D7
:10587000020D500EF324D96E040EF420DA6E66C0C9
:10588000DEFF67C0DDFFFC2B01014C510001FC5D18
:10589000D8B003D0B3D77A4B7B2B000E7A25D96EC4
:1058A000070E7B21DA6E2A0EDE18D8A4F4D77A0709
:1058B000D8A07B07020E01014D6F000E00017A2572
:1058C000D96E070E7B21DA6E310EDE18D8A41200D5
:1058D000010E01014D6F1200000E00017A25666F66
:1058E000070E7B21676F7EEC5DF0000166510201BF
:1058F0009C6F03D000017A4B7B2B000E00017A25B0
:10590000D96E070E7B21DA6E2C0EDE18D8A4F2D7E2
:105910007A4B7B2B000E7A25666F070E7B21676F13
:105920007EEC5DF066C09DF267C09EF21200000E34
:1059300000017A25666F070E7B21676F7EEC5DF0B4
:105940000001665102019F6F120000017D51000AA3
:10595000D8B4BBD5020AD8B4C2D5010AD8B4C3D5CD
:10596000070AD8B4CED5010AD8B413D6030AD8B4DE
:1059700058D6010AD8B49DD60F0AD8B4A8D6010AC1
:10598000D8B4B3D6030AD8B4A7D7060AD8A412004D
:10599000CED7470E03017619D8A412D0500E77192E
:1059A000D8A40ED0430E7819D8A40AD04F0E791976
:1059B000D8A406D04E0E7A19D8A402D0040E120034
:1059C000470E7619D8A412D0450E7719D8A40ED058
:1059D000440E7819D8A40AD0410E7919D8A406D05B
:1059E000540E7A19D8A402D0050E1200470E76196B
:1059F000D8A412D0450E7719D8A40ED0430E78192A
:105A0000D8A40AD04E0E7919D8A406D0460E7A1919
:105A1000D8A402D0060E1200530E7619D8A412D0C4
:105A2000450E7719D8A40ED0430E7819D8A40AD001
:105A30004E0E7919D8A406D0460E7A19D8A402D0F1
:105A4000070E1200470E7619D8A412D0450E77190A
:105A5000D8A40ED0430E7819D8A40AD04C0E7919C8
:105A6000D8A406D04F0E7A19D8A402D0080E12007E
:105A7000530E7619D8A412D0450E7719D8A40ED09B
:105A8000430E7819D8A40AD04C0E7919D8A406D0A0
:105A9000520E7A19D8A402D00A0E1200530E7619AB
:105AA000D8A412D0450E7719D8A40ED0430E781979
:105AB000D8A40AD0410E7919D8A406D04C0E7A1970
:105AC000D8A402D0130E1200470E7619D8A412D013
:105AD000450E7719D8A40ED04D0E7819D8A40AD047
:105AE000450E7919D8A406D04D0E7A19D8A402D043
:105AF0000B0E1200470E7619D8A412D0450E771956
:105B0000D8A40ED04D0E7819D8A40AD0450E791914
:105B1000D8A406D0540E7A19D8A402D0200E1200B0
:105B2000470E7619D8A412D0450E7719D8A40ED0F6
:105B3000430E7819D8A40AD0540E7919D8A406D0E7
:105B4000450E7A19D8A402D0210E1200470E7619FC
:105B5000D8A412D0450E7719D8A40ED0410E7819CA
:105B6000D8A40AD0440E7919D8A406D0530E7A19B5
:105B7000D8A402D00E0E1200470E7619D8A412D067
:105B8000450E7719D8A40ED0520E7819D8A40AD091
:105B9000410E7919D8A406D0570E7A19D8A402D08C
:105BA000100E1200470E7619D8A412D0450E7719A0
:105BB000D8A40ED0560E7819D8A40AD0450E79195B
:105BC000D8A406D0520E7A19D8A402D0140E12000E
:105BD000530E7619D8A412D0450E7719D8A40ED03A
:105BE000560E7819D8A40AD0450E7919D8A406D033
:105BF000520E7A19D8A402D0230E1200530E761931
:105C0000D8A412D0450E7719D8A40ED0550E781905
:105C1000D8A40AD0500E7919D8A406D04C0E7A19FF
:105C2000D8A402D0120E1200530E7619D8A412D0A6
:105C3000450E7719D8A40ED0430E7819D8A40AD0EF
:105C40004C0E7919D8A406D04D0E7A19D8A402D0DA
:105C50001A0E1200530E7619D8A412D0450E7719D9
:105C6000D8A40ED0430E7819D8A40AD04C0E7919B6
:105C7000D8A406D0540E7A19D8A402D01F0E120050
:105C8000470E7619D8A412D0450E7719D8A40ED095
:105C90004D0E7819D8A40AD0560E7919D8A406D07A
:105CA000540E7A19D8A402D0250E1200470E761988
:105CB000D8A412D0450E7719D8A40ED0500E78195A
:105CC000D8A40AD0490E7919D8A406D0530E7A194F
:105CD000D8A402D0260E1200530E7619D8A412D0E2
:105CE000450E7719D8A40ED0500E7819D8A40AD032
:105CF000490E7919D8A406D0530E7A19D8A402D027
:105D0000270E1200530E7619D8A412D0450E77191B
:105D1000D8A40ED0500E7819D8A40AD0490E7919FB
:105D2000D8A406D0300E7A19D8A402D0280E1200BA
:105D3000530E7619D8A412D0450E7719D8A40ED0D8
:105D4000500E7819D8A40AD0490E7919D8A406D0D3
:105D5000310E7A19D8A402D0290E1200530E7619EA
:105D6000D8A412D0450E7719D8A40ED0500E7819A9
:105D7000D8A40AD0490E7919D8A406D0320E7A19BF
:105D8000D8A402D02A0E1200530E7619D8A412D02D
:105D9000450E7719D8A40ED0500E7819D8A40AD081
:105DA000490E7919D8A406D0330E7A19D8A402D096
:105DB0002B0E1200530E7619D8A412D0450E771967
:105DC000D8A40ED0500E7819D8A40AD0490E79194B
:105DD000D8A406D0340E7A19D8A402D02C0E120002
:105DE000530E7619D8A412D0450E7719D8A40ED028
:105DF000500E7819D8A40AD0490E7919D8A406D023
:105E0000350E7A19D8A402D02D0E1200530E761931
:105E1000D8A412D0450E7719D8A40ED0500E7819F8
:105E2000D8A40AD0490E7919D8A406D0360E7A190A
:105E3000D8A402D02E0E1200530E7619D8A412D078
:105E4000450E7719D8A40ED0500E7819D8A40AD0D0
:105E5000490E7919D8A406D0370E7A19D8A402D0E1
:105E60002F0E12005FEC6FF0000E12000001E351E4
:105E7000E411D8B40CD0E3C0D9FFE4C0DAFFE1C02C
:105E8000DEFFE2C0DDFF03D00001E14BE22BE1C009
:105E9000D9FFE2C0DAFFDF50E66FE651CCEC70F0DC
:105EA000D8B0F2D7000E0001E76F2D0EE619D8A486
:105EB00003D0010EE76F04D02B0EE619D8A402D050
:105EC000E14BE22B000EE66F000EE96F000EEA6F69
:105ED000000EEB6F000EEC6F000EE86FE7B90AD012
:105EE000E1C0D9FFE2C0DAFF2E0EDE18D8A402D03E
:105EF000E7893ED0E1C0D9FFE2C0DAFFDF508DEC88
:105F000071F0D8A038D00001E783090EE619D8B4A3
:105F10002DD0E7B9E807E62BE9C060F0EAC061F0F0
:105F2000EBC062F0ECC063F00A0E646F000E656FA8
:105F3000000E666F000E676F0FEC6DF060C0E9F049
:105F400061C0EAF062C0EBF063C0ECF0E1C0D9FFE1
:105F5000E2C0DAFFDF500001E56FD00EE527E55122
:105F6000E927000EEA23EB23EC2302D0E7A9E82B74
:105F7000E14BE22BB3D7000E0001E66FE1C0D9FF81
:105F8000E2C0DAFF650EDE18D8B408D0E1C0D9FF50
:105F9000E2C0DAFF450EDE18D8A462D0E14BE22B56
:105FA000E1C0D9FFE2C0DAFF2D0EDE18D8A402D07E
:105FB000E78708D0E1C0D9FFE2C0DAFF2B0EDE1878
:105FC000D8A402D0E14BE22BE1C0D9FFE2C0DAFF56
:105FD000300EDE18D8B4F6D7E1C0D9FFE2C0DAFF40
:105FE000DF508DEC71F0D8A038D0E1C0D9FFE2C00D
:105FF000DAFFDF50D00F0001E66FE14BE22BE1C08A
:10600000D9FFE2C0DAFFDF508DEC71F0D8A025D0C7
:10601000E1C0D9FFE2C0DAFFDF500001E56FE651D1
:106020000A0DF350E525D00FE66FE14BE22BE1C0FE
:10603000D9FFE2C0DAFFDF508DEC71F0D8A00DD0AF
:10604000E1C0D9FFE2C0DAFFDF500001E56FE651A1
:106050000A0DF350E525D00FE66F0001E7B7E66DB6
:10606000E651E827E351E411D8A4E7A308D0E3C040
:10607000D9FFE4C0DAFFE1C0DEFFE2C0DDFFE9C026
:106080006CF0EAC06DF0EBC06EF0ECC06FF0010E8A
:106090006AEC4AF06CC0E9F06DC0EAF06EC0EBF05B
:1060A0006FC0ECF00001E951EA11EB11EC11D8A43A
:1060B00009D0000EE16F000EE26F000EE36F000EDC
:1060C000E46F1200E8AF6DD0E86D1DD0E9C0C8F0F4
:1060D000EAC0C9F0EBC0CAF0ECC0CBF0F90ECC6F4F
:1060E000020ECD6F150ECE6F500ECF6F28EC3BF029
:1060F000C8C0E9F0C9C0EAF0CAC0EBF0CBC0ECF010
:10610000F60E0001E827E851800A760FD8A01DD0CE
:10611000DDD7E9C0C8F0EAC0C9F0EBC0CAF0ECC0F6
:10612000CBF0000ECC6F000ECD6F200ECE6F410E67
:10613000CF6F28EC3BF0C8C0E9F0C9C0EAF0CAC094
:10614000EBF0CBC0ECF00001E807E851D8A4E1D7B0
:10615000E9C0ABF0EAC0ACF0EBC0ADF0ECC0AEF023
:10616000000EAF6F000EB06F800EB16F000EB26FF9
:1061700092EC50F00001D8B083D0E7A109D0000E16
:10618000E16F000EE26F800EE36F800EE46F12008D
:10619000000EE16F000EE26F800EE36F000EE46F01
:1061A0001200E851800A7F0FD8B01ED069D0E9C034
:1061B0007EF0EAC07FF0EBC080F0ECC081F0F90E19
:1061C000826F020E836F150E846F500E856FFFEC89
:1061D00034F07EC0E9F07FC0EAF080C0EBF081C00F
:1061E000ECF0F60E0001E8270A0EE861E0D71CD0BB
:1061F000E9C07EF0EAC07FF0EBC080F0ECC081F037
:10620000000E826F000E836F200E846F410E856F2B
:10621000FFEC34F07EC0E9F07FC0EAF080C0EBF024
:1062200081C0ECF00001E807E851D8A4E1D7FF0EE7
:10623000AB6FFF0EAC6F7F0EAD6F7F0EAE6FE9C020
:10624000AFF0EAC0B0F0EBC0B1F0ECC0B2F092EC4D
:1062500050F00001D8B014D0E7A109D0000EE16FD2
:10626000000EE26F800EE36F800EE46F1200000EEE
:10627000E16F000EE26F800EE36F000EE46F12001C
:10628000E7A112D0E9C07AF0EAC07BF0EBC07CF065
:10629000ECC07DF011EC70F07AC0E9F07BC0EAF060
:1062A0007CC0EBF07DC0ECF0E9C0E1F0EAC0E2F0C8
:1062B000EBC0E3F0ECC0E4F01200000E0001946FBC
:1062C000000E936F000E926F000E916F000E906F94
:1062D000000E8F6F000E606F070E616F000E636F10
:1062E0006269020E656F000E646F29EC70F0000E9B
:1062F0000001606F050E616F000E636F6269020E30
:10630000656F000E646F29EC70F094EC6FF0000E76
:1063100000016C6F070E6D6FD5EC6AF0000E000186
:10632000926F000E916F000E946F000E936F020E2D
:10633000945DD8B03CD0000E9325D96E070E942101
:10634000DA6E240EDE18D8A41FD0010E93258C6FB0
:10635000000E94218D6F000E8C25D96E070E8D21B5
:10636000DA6E390EDE18D8B403D00ED0934B942BCE
:10637000000E9325D96E070E9421DA6E0A0EDE18F0
:10638000D8A4F4D7934B942B000E9325D96E070E07
:106390009421DA6E000E9125E16E050E9221E26ED7
:1063A000DFCFE7FF914B922B934B942BC0D7000E7E
:1063B000946F000E936F02D0934B942B000E932595
:1063C000D96E050E9421DA6EDE28D8B40FD0010EF6
:1063D00093258C6F000E94218D6F000E8C25D96E45
:1063E000050E8D21DA6EDE28D8A4E6D7000E93259F
:1063F000D96E050E9421DA6E0A0EDF6E934B942B44
:10640000000E9325D96E050E9421DA6E240EDF6EF0
:10641000934B942B000E9325D96E050E9421DA6EC2
:10642000390EDF6E934B942B000E9325D96E050E1B
:106430009421DA6E2C0EDF6E934B942B000E932575
:10644000766F050E9421776F940E786F150E796F25
:1064500052C17AF053C17BF054C17CF055C17DF03C
:1064600016EC3FF003D00001934B942B000E00017B
:106470009325D96E050E9421DA6EDF50D8A4F3D798
:10648000000E9325D96E050E9421DA6E2C0EDF6E68
:10649000934B942B000E9325766F050E9421776F06
:1064A000940E786F150E796F4EC17AF04FC17BF064
:1064B00050C17CF051C17DF016EC3FF003D00001DB
:1064C000934B942B000E00019325D96E050E942159
:1064D000DA6EDF50D8A4F3D7000E9325D96E050EDF
:1064E0009421DA6E2C0EDF6E934B942B000E9325C5
:1064F000D96E050E9421DA6E01014C51300FDF6E1A
:106500000001934B942B000E9325D96E050E942118
:10651000DA6E2C0EDF6E934B942B000E9325766F64
:10652000050E9421776F980E786F150E796F53C30F
:106530007AF054C37BF016EC3FF003D00001934B8C
:10654000942B000E00019325D96E050E9421DA6E6E
:10655000DF50D8A4F3D7000E9325D96E050E9421F1
:10656000DA6E2C0EDF6E934B942B000E9325766F14
:10657000050E9421776F980E786F150E796F50C4C1
:106580007AF051C47BF016EC3FF003D00001934B3E
:10659000942B000E00019325D96E050E9421DA6E1E
:1065A000DF50D8A4F3D7000E9325D96E050E9421A1
:1065B000DA6E2C0EDF6E934B942B000E9325766FC4
:1065C000050E9421776F9B0E786F150E796F520E22
:1065D0007A6F150E7B6F16EC3FF003D00001934BE2
:1065E000942B000E00019325D96E050E9421DA6ECE
:1065F000DF50D8A4F3D7000E9325D96E050E942151
:10660000DA6E2C0EDF6E934B942B01014D05D8A44E
:1066100009D0000E00019325D96E050E9421DA6E83
:10662000310E08D0000E00019325D96E050E94217D
:10663000DA6E320EDF6E934B942B000E9325D96EDB
:10664000050E9421DA6E2C0EDF6E934B942B000E08
:106650009325D96E050E9421DA6E2A0EDF6E934BC8
:10666000942B000E9325D96E050E9421DA6E0D0E33
:10667000DF6E934B942B000E9325D96E050E94215B
:10668000DA6E0A0EDF6E934B942B94EC6FF035ECC0
:106690006AF0000E0001676F050E686F85EC69F007
:1066A000B6EC67F0120027A082D044C148F145C182
:1066B00049F146C14AF147C14BF170C172F171C154
:1066C00073F16AC16CF16BC16DF104C208F205C2CD
:1066D00009F206C20AF207C20BF240C144F141C1FD
:1066E00045F142C146F143C147F16EC170F16FC13E
:1066F00071F168C16AF169C16BF100C204F201C2B3
:1067000005F202C206F203C207F200EC22F021EE0B
:106710004EF0DECFF7F0DDCFF8F00001F71FF81FE5
:10672000F74BF82B0201AD510001F72501016E6F07
:106730000201AE510001F82101016F6F21EE52F00C
:10674000DECFF7F0DDCFF8F00001F71FF81FF74BB1
:10675000F82B0201B1510001F7250101686F020118
:10676000B2510001F8210101696F2EC260F02FC201
:1067700061F030C262F031C263F0640E0001646FF8
:10678000000E656F000E666F000E676F0FEC6DF008
:1067900060C000F261C001F262C002F263C003F2A5
:1067A000000E0101CF6FCF8B2790020E1200010166
:1067B000BCA120D0BC9142EC4EF00101FC51D8A408
:1067C00015D0A4EC58F097EC66F00001F96FF95180
:1067D000D8B410D0000E02013E6F000E3F6F000EC5
:1067E000406F000E416F0001F95112002496FC0722
:1067F0008F8EC48386B427BC1BD0278C0101C8A10F
:1068000015D0060ED36ED350700B600AD8A4FBD7F8
:10681000010E656E010ED36E0A0ECFEC71F0010110
:10682000C891CA68000ECC6EE10ECB6E030E12004A
:1068300027BC86B411D0320ECFEC71F086B403D0F1
:10684000279C090E1200000E02013E6F000E3F6FE2
:10685000000E406F000E416F86A45AD0200E2D18F6
:10686000D8A456D0020E0101CC19D8A451D0000EE4
:1068700000016B6F070E6C6F080E6D6F8EEC64F08D
:106880000009D8B43CD02B500101A727000EA82343
:10689000000E296E14D02950010D000EF324D96E7C
:1068A000070EF420DA6E750E0101A925E16E030EC4
:1068B000AA21E26EDFCFE7FFA94BAA2B292A295094
:1068C0000001F76FF86B0101A7510001F75D0101AD
:1068D000A8510001F859D8A0DED70101A85104E160
:1068E000070EA75DD8A00BD0000EA86F000EA76FF3
:1068F000000EAA6F000EA96FC9EC2CF01200000E5A
:1069000002013E6F000E3F6F000E406F000E416FA0
:106910000101C2AB0FD0000ECF6FCF89C29B000E1A
:1069200002013E6F000E3F6F000E406F000E416F80
:106930000F0E120027A403D02794010E1200C8B135
:106940000CD0A45104E19B0EA35DD8A012D0000E80
:10695000A46F000EA36F240E1200080EA35D070E95
:10696000A459D8A006D0000EA46F000EA36F240E69
:106970001200130EB66504D0000EB66F1D0E120085
:106980003B0EB56504D0000EB56F1E0E1200040E4E
:10699000C76504D0000EC76F0C0E120002014151F2
:1069A00007E1FA0E3E5D450E3F59010E4059D8B041
:1069B00056EC5EF0B00E02016B5D040E6C59D8A06F
:1069C00006D0000E6C6F000E6B6F310E1200185067
:1069D00007E11528EF0E16581F0E1758D8A002D041
:1069E0000D0E120084A409D00101C28F000ECF6FDA
:1069F000C2BFCF87C29F110E1200000E120000010D
:106A00008151800B8A6F81518125906F80BF908169
:106A10009051D8B40DD09029D8A408D0000E7E6F24
:106A2000000E7F6F000E806F000E816F808F08D088
:106A3000000E7E6F000E7F6F000E806F000E816F64
:106A40008551800B8A1B855185258F6F84BF8F816F
:106A50008F51D8B40DD08F29D8A408D0000E826FE2
:106A6000000E836F000E846F000E856F848F08D038
:106A7000000E826F000E836F000E846F000E856F14
:106A80008F51D8B403D09051D8A409D0000E7E6F96
:106A9000000E7F6F000E806F000E816F1200845118
:106AA0007E03F3CF95F0F4CF96F095518B6F8C6BFE
:106AB0008D6B8E6B9651916F926B936B946B835130
:106AC0007F03F3CF95F0F4CF96F095518B27000E0E
:106AD0008C238D238E2396519127000E922393238E
:106AE000942382518003F3CF95F0F4CF96F0955123
:106AF0008B27000E8C238D238E2396519127000E19
:106B00009223932394238DC08EF08CC08DF08BC084
:106B10008CF08B6B82517F03F3CF95F0F4CF96F01E
:106B200095518B2796518C23000E8D23000E8E23BA
:106B300083517E03F3CF95F0F4CF96F095518B27D8
:106B400096518C23000E8D23000E8E238DC08EF067
:106B50008CC08DF08BC08CF08B6B82517E03F3CF99
:106B600095F0F4CF96F095518B2796518C23000E1B
:106B70008D23000E8E2384517F03F3CF95F0F4CF45
:106B800096F09551912796519223000E9323000E73
:106B9000942383518003F3CF95F0F4CF96F0955171
:106BA000912796519223000E9323000E9423845133
:106BB0008003F3CF95F0F4CF96F09551866F965100
:106BC000876F886B896B88C089F087C088F086C022
:106BD00087F0866B865191278751922388519323A2
:106BE000895194238BC086F08CC087F08DC088F0CB
:106BF0008EC089F0190E05D0D89089338833873339
:106C00008633E82EF9D786519127875192238851F0
:106C10009323895194238DC08EF08CC08DF08BC04E
:106C20008CF08B6B8F5190C086F0876B8627000E9F
:106C30008723820E8625956FFF0E8721966F0FD0D2
:106C4000D89091379237933794378EBF9181D890EF
:106C50008B378C378D378E379507D8A0960793AF33
:106C6000EFD7000E8F6F8EAF16D0FF0E8B15866F8D
:106C7000FF0E8C15876FFF0E8D15886F7F0E8E159A
:106C8000896F8651871188118911D8A402D091A1EA
:106C900002D0010E8F6F8F51D8B41FD0010E9127F3
:106CA000000E92239323942394A117D091C086F0D1
:106CB00092C087F093C088F094C089F089358933F9
:106CC00088338733863386C091F087C092F088C0BE
:106CD00093F089C094F0954B962B96BF0DD09651AA
:106CE00003E19529D8A008D0000E916F000E926F95
:106CF000800E936F7F0E20D096BF05D096510EE187
:106D00009505D8B00BD0000E916F000E926F000E5B
:106D1000936F000E946F000E8A6F0FD095C090F0A5
:106D2000FF0E9117FF0E92177F0E9317000E941708
:106D300090B1938FD8909031946F8A51941391C0F1
:106D40007EF092C07FF093C080F094C081F012007A
:106D500000019A51800BA76F9A519A25A96F99BF8C
:106D6000A981A951D8B40DD0A929D8A408D0000E62
:106D7000976F000E986F000E996F000E9A6F998FA3
:106D800006D0000E976F000E986F000E996F000EE0
:106D90009A6F9E51800BA86FA751A819D8A4A78DF0
:106DA0009E519E25A86F9DBFA881A851D8B40DD033
:106DB000A829D8A408D0000E9B6F000E9C6F000E6F
:106DC0009D6F000E9E6F9D8F06D0000E9B6F000E74
:106DD0009C6F000E9D6F000E9E6FA951A85DD8B0EC
:106DE00022D0A7AD02D0800EA71BA9C0AAF0A8C0D0
:106DF000A9F0AAC0A8F097C0AAF09BC097F0AAC0BB
:106E00009BF098C0AAF09CC098F0AAC09CF099C0D2
:106E1000AAF09DC099F0AAC09DF09AC0AAF09EC0A9
:106E20009AF0AAC09EF0000EAA6FA9519F6FA06BA6
:106E30009F1FA01F9F4BA02BA851A16FA26B9F511A
:106E4000A127A051A223A2BF2CD0A25104E11A0E67
:106E5000A15DD8A026D09751981199119A11D8B454
:106E600002D0010E01D0000EAA6F000E976F000E27
:106E7000986F000E996F000E9A6FA8C0A9F015D0F8
:106E8000AAA105D0D890AA310109AA6F02D0D89042
:106E9000AA3397B1AA8F9A359A3399339833973397
:106EA000A92BA851A95DD8A0EBD7A7BD29D0A9517E
:106EB000D8A409D0000E976F000E986F000E996F3E
:106EC000000E9A6F12009B5197279C5198239D5159
:106ED00099239E519A239AA183D0AAA106D0D89033
:106EE000AA33AA510109AA6F02D0D890AA3397B148
:106EF000AA8F9A359A33993398339733A92B70D048
:106F00009B51975D9C5198599D5199599A51800A6E
:106F10009F6F9E51800A9F59D8B036D097C09FF07E
:106F200098C0A0F099C0A1F09AC0A2F09F1FA01F26
:106F3000A11FA21F9F2B000EA023A123A2239B51C0
:106F40009F25A36F9C51A021A46F9D51A121A56FE6
:106F50009E51A221A66FFF0EA325976FFF0EA421BD
:106F6000986FFF0EA521996FFF0EA6219A6F800ED4
:106F7000A71BAA6DAA51D8A40FD0010E9727000E07
:106F8000982399239A2308D09B51975F9C51985B33
:106F90009D51995B9E519A5B9751981199119A1145
:106FA000D8A41CD0AA51D8A419D0000E976F000EF7
:106FB000986F000E996F000E9A6F1200D890973755
:106FC000983799379A37AABF9781AAA102D0D8805B
:106FD00001D0D890AA37A951D8A4A90799AFEED764
:106FE000000EA86FAAAF0AD0AAC09FF07F0E9F170D
:106FF000D8A402D097A102D0010EA86FA851D8B48E
:1070000020D0010E9727000E982399239A239AA146
:1070100018D097C09FF098C0A0F099C0A1F09AC076
:10702000A2F0A235A233A133A0339F339FC097F0C3
:10703000A0C098F0A1C099F0A2C09AF0A929D8A444
:10704000A92BA929D8B403D0A951D8A40DD0000EDA
:10705000976F000E986F000E996F000E9A6FA951EE
:10706000D8A402D0000EA76FA9A102D0998F01D099
:10707000999FD890A9319A6FA7BF9A8F97C097F020
:1070800098C098F099C099F09AC09AF01200000E3A
:107090000001756F000E746F000E736F000E726F3B
:1070A000000E606F050E616F000E636F6269020E65
:1070B000656F000E646F29EC70F0000E0001606FC8
:1070C000070E616F000E636F6269020E656F000E3E
:1070D000646F29EC70F094EC6FF0000E00016C6F9F
:1070E000050E6D6FD5EC6AF0000E0001756F000E95
:1070F000746F020E755DD8B01200000E7425D96E43
:10710000050E7521DA6E240EDE18D8A447D0010EC4
:1071100074256F6F000E7521706F000E6F25D96E8C
:10712000050E7021DA6E300EDE18D8A437D0020EAC
:1071300074256F6F000E7521706F000E6F25D96E6C
:10714000050E7021DA6E2C0EDE18D8B413D026D0BE
:10715000000E7425D96E050E7521DA6E000E7225AB
:10716000E16E070E7321E26EDFCFE7FF744B752BE4
:10717000724B732B000E7425D96E050E7521DA6ED5
:107180000A0EDE18D8A4E4D7000E7225D96E070EB9
:107190007321DA6E0A0EDF6E724B732B000E7425AC
:1071A000D96E050E7521DA6E240EDE18D8A447D0EC
:1071B000010E74256F6F000E7521706F000E6F2524
:1071C000D96E050E7021DA6E310EDE18D8A437D0D4
:1071D000020E74256F6F000E7521706F000E6F2503
:1071E000D96E050E7021DA6E2C0EDE18D8B413D0CD
:1071F00026D0000E7425D96E050E7521DA6E000EAC
:107200007225E16E070E7321E26EDFCFE7FF744B4C
:10721000752B724B732B000E7425D96E050E7521DC
:10722000DA6E0A0EDE18D8A4E4D7000E7225D96EE5
:10723000070E7321DA6E0A0EDF6E724B732B000E8F
:107240007425D96E050E7521DA6E240EDE18D8A4C9
:1072500047D0010E74256F6F000E7521706F000E00
:107260006F25D96E050E7021DA6E320EDE18D8A4A5
:1072700037D0020E74256F6F000E7521706F000EEF
:107280006F25D96E050E7021DA6E2C0EDE18D8B47B
:1072900013D026D0000E7425D96E050E7521DA6E36
:1072A000000E7225E16E070E7321E26EDFCFE7FF5D
:1072B000744B752B724B732B000E7425D96E050E13
:1072C0007521DA6E0A0EDE18D8A4E4D7000E7225F6
:1072D000D96E070E7321DA6E0A0EDF6E724B732BB6
:1072E000000E7425D96E050E7521DA6E240EDE1897
:1072F000D8A447D0010E74256F6F000E7521706FF2
:10730000000E6F25D96E050E7021DA6E330EDE1871
:10731000D8A437D0020E74256F6F000E7521706FE0
:10732000000E6F25D96E050E7021DA6E2C0EDE1858
:10733000D8B413D026D0000E7425D96E050E752151
:10734000DA6E000E7225E16E070E7321E26EDFCF5A
:10735000E7FF744B752B724B732B000E7425D96E9F
:10736000050E7521DA6E0A0EDE18D8A4E4D7000ED9
:107370007225D96E070E7321DA6E0A0EDF6E724B1C
:10738000732B744B752BB5D60001AE51800BB36FC8
:10739000AE51AE25B96FADBFB981B9C0BEF0BF6BFC
:1073A000FF0EAB15C46FFF0EAC15C56F7F0EAD158C
:1073B000C66F000EAE15C76FBE51BF11D8B405D051
:1073C000C68FBE29BF11D8A408D0000EC46F000E0E
:1073D000C56F000EC66F000EC76FBE51BF11D8A497
:1073E00009D0000EAB6F000EAC6F000EAD6F000E3B
:1073F000AE6F1200B351D8B41AD0000EC06F000E99
:10740000C16F400EC26F000EC36F800EC213FF0E1D
:10741000C313000E0201586F210E576FC0C0ABF0AE
:10742000C1C0ACF0C2C0ADF0C3C0AEF012000001EC
:10743000BE29BF11D8A411D0000EC06F000EC16FBD
:10744000800EC26F7F0EC36FC0C0ABF0C1C0ACF086
:10745000C2C0ADF0C3C0AEF01200810EBE27FF0E59
:10746000BF23BE51010BB96FBF35BF33BE337F0E93
:10747000BE27000EBF23D890C435B56FC535B66F93
:10748000C635B76FC735B86F000EC46F000EC56F35
:10749000000EC66F000EC76F000EBA6F000EBB6FF6
:1074A000000EBC6F010EBD6FB951D8B405D0D89095
:1074B000B537B637B737B837000EB46F52D0BA51B8
:1074C000C413BB51C513BC51C613BD51C713C4511E
:1074D000B55DC551B659C651B759C751B859D8A0AD
:1074E00011D0C451B55FC551B65BC651B75BC7512A
:1074F000B85BBA51C427BB51C523BC51C623BD518B
:10750000C72314D0BAC0AFF0BBC0B0F0BCC0B1F05C
:10751000BDC0B2F0AF1FB01FB11FB21FAF51C41733
:10752000B051C517B151C617B251C717BAC0AFF0A5
:10753000BBC0B0F0BCC0B1F0BDC0B2F0D890B233A7
:10754000B133B033AF33AFC0BAF0B0C0BBF0B1C0ED
:10755000BCF0B2C0BDF0D890B537B637B737B83742
:10756000B42B180EB465ABD7C4C0AFF0C5C0B0F033
:10757000C6C0B1F0C7C0B2F0D890B233B133B033A7
:10758000AF33AFC0C4F0B0C0C5F0B1C0C6F0B2C038
:10759000C7F0010EC415BA6F000EC515BB6F000E03
:1075A000C615BC6F000EC715BD6FC4C0AFF0C5C017
:1075B000B0F0C6C0B1F0C7C0B2F0D890B233B133AA
:1075C000B033AF33AFC0C4F0B0C0C5F0B1C0C6F087
:1075D000B2C0C7F0BA51C427BB51C523BC51C623A2
:1075E000BD51C723C7A117D0C4C0AFF0C5C0B0F00C
:1075F000C6C0B1F0C7C0B2F0D890B233B133B03327
:10760000AF33AFC0C4F0B0C0C5F0B1C0C6F0B2C0B7
:10761000C7F0BE4BBF2BFF0EC415C06FFF0EC515C4
:10762000C16F7F0EC615C26F000EC715C36FBEC0F7
:10763000B9F0B9B1C28FD890B931C36FC39FC0C080
:10764000ABF0C1C0ACF0C2C0ADF0C3C0AEF0120030
:107650000001CB51800BD46FCB51CB25DF6FCABF5C
:10766000DF81DF51D8B40DD0DF29D8A408D0000EB7
:10767000C86F000EC96F000ECA6F000ECB6FCA8FA5
:1076800006D0000EC86F000EC96F000ECA6F000E44
:10769000CB6FCF51800BD41BCF51CF25E06FCEBF26
:1076A000E081E051D8B40DD0E029D8A408D0000E74
:1076B000CC6F000ECD6F000ECE6F000ECF6FCE8F51
:1076C00006D0000ECC6F000ECD6F000ECE6F000EF8
:1076D000CF6FCC51CD11CE11CF11D8A415D0000E43
:1076E000C86F000EC96F000ECA6F000ECB6F800E00
:1076F000CA137F0ECB13C8C0C8F0C9C0C9F0CAC036
:10770000CAF0CBC0CBF01200DF51D8A411D0000ECC
:10771000C86F000EC96F000ECA6F000ECB6FC8C0D5
:10772000C8F0C9C0C9F0CAC0CAF0CBC0CBF01200C3
:10773000E051D06FD16BD01FD11FD04BD12BDF5177
:10774000D26FD36BD051D227D151D3237F0ED22504
:10775000D96F000ED321DA6FC8C0D5F0C9C0D6F0FA
:10776000CAC0D7F0CBC0D8F0000EC86F000EC96FEA
:10777000000ECA6F000ECB6F000EDB6F000EDC6FC9
:10778000000EDD6F000EDE6F000EE06F28D0E051BE
:10779000D8B411D0D890D537D637D737D837D89076
:1077A000C837C937CA37CB37DEBFC881D890DB3777
:1077B000DC37DD37DE37CC51D55DCD51D659CE51D2
:1077C000D759CF51D859D8A009D0DE8DCC51D55F2B
:1077D000CD51D65BCE51D75BCF51D85BE02B190E84
:1077E000E065D5D7D551D611D711D811D8B411D05D
:1077F000DB810FD0D890C837C937CA37CB37DEBF47
:10780000C881D890DB37DC37DD37DE37D907D8A021
:10781000DA07CAAFEFD7000EE06FDEAF16D0FF0E6B
:10782000DB15D06FFF0EDC15D16FFF0EDD15D26FAB
:107830007F0EDE15D36FD051D111D211D311D8A440
:1078400002D0C8A102D0010EE06FE051D8B41FD021
:10785000010EC827000EC923CA23CB23CBA117D002
:10786000C8C0D0F0C9C0D1F0CAC0D2F0CBC0D3F0EC
:10787000D335D333D233D133D033D0C0C8F0D1C015
:10788000C9F0D2C0CAF0D3C0CBF0D94BDA2BDABFE3
:1078900010D0DA5103E1D929D8A00BD0000EDA6F4D
:1078A000D969000EC86F000EC96F000ECA6F000EB6
:1078B000CB6FDABF05D0DA5111E1D905D8B00ED0BF
:1078C000000EDA6F000ED96F000EC86F000EC96F80
:1078D000000ECA6F000ECB6F000ED46FD9C0DFF060
:1078E000DFA102D0CA8F01D0CA9FD890DF31CB6F01
:1078F000D451CB13C8C0C8F0C9C0C9F0CAC0CAF0BF
:10790000CBC0CBF01200000E0001786F000E776F35
:1079100014EC4BF06CC015F06DC016F06EC017F093
:107920006FC018F047EC38F0000E0201646F000ED3
:10793000636F000E0001606F050E616F000E636FD4
:10794000000E626F020E656F000E646F29EC70F01E
:10795000240E6AEC71F0000E0001786F000E776F54
:10796000785111E1020E775DD8B00DD0ED0E77257C
:10797000D96E020E7821DA6EDF506AEC71F00001E8
:10798000774B782BEDD72C0E6AEC71F0000E0001CE
:10799000786F000E776F785115E1020E775DD8B0E1
:1079A00011D0020E7725F66E140E7821F76EF86A64
:1079B000000EF8220800F5506AEC71F00001774BD8
:1079C000782BE9D72C0E6AEC71F0000E0001786F6D
:1079D000000E776F785111E1020E775DD8B00DD0AF
:1079E000EA0E7725D96E020E7821DA6EDF506AEC46
:1079F00071F00001774B782BEDD72A0E6AEC71F00D
:107A00000D0E6AEC71F00A0E6AEC71F0000E0001C6
:107A1000786F000E776F0CD0000E7725D96E070EA9
:107A20007821DA6EDF506AEC71F00001774B782B29
:107A3000000E7725D96E070E7821DA6EDE28D8A4DD
:107A4000EBD7240E6AEC71F0540E6AEC71F02C0E38
:107A50006AEC71F01DB018D0000E0001786F000EB6
:107A6000776F785135E10B0E775DD8B031D0CE0EFF
:107A70007725D96E020E7821DA6EDF506AEC71F04C
:107A80000001774B782BEDD7000E0001786F000EC8
:107A9000776F10D0840E7725F66E130E7821F76E6F
:107AA000F86A000EF8220800F5506AEC71F0000147
:107AB000774B782B840E7725F66E130E7821F76EB0
:107AC000F86A000EF8220800F5500009D8A4E2D7A1
:107AD0000D0E6AEC71F00A0E6AEC71F0000E0001F6
:107AE000786F000E776F10D0E00E7725F66E130ECC
:107AF0007821F76EF86A000EF8220800F5506AEC5B
:107B000071F00001774B782BE00E7725F66E130E9F
:107B10007821F76EF86A000EF8220800F550000987
:107B2000D8A4E2D70D0E6AEC71F00A0E6AEC71F07F
:107B3000240E6AEC71F02C0E6AEC71F022506AECA3
:107B400071F00D0E6AEC71F00A0E6AEC71F094ECB3
:107B50006FF0000E0001666F050E676F63C268F07C
:107B600064C269F06CEC6AF025822690279A25861B
:107B700027922788000E02012E6F000E2F6F000E35
:107B8000306F000E316F000E0101C66F000E000154
:107B9000606F070E616F000E636F000E626F020E62
:107BA000656F000E646F29EC70F012000101320560
:107BB000D8A40ED030511F0B0009D8A409D0048ED0
:107BC000030E3119D8A402D0010E01D0000EDD6FD2
:107BD0003251D8A4120030511F0B020AD8A412004F
:107BE00034510F0B0009D8B4120034510F0B436EFF
:107BF000030E43601200200E2D18D8A41200048E2C
:107C000034BF19D034510F0B436E4350020D0C0E8C
:107C1000F324D96E020EF420DA6EDECF47F0DDCF0A
:107C200048F034510F0B436E4350010D540EF324B2
:107C3000D96E020E18D034510F0B436E4350020D13
:107C4000070EF324D96E000EF420DA6EDECF47F073
:107C5000DDCF48F034510F0B436E4350010DA00EA1
:107C6000F324D96E010EF420DA6EDF50466E46B072
:107C700006D0FB0E4714476EFF0E481404D0040EC6
:107C80004710476E4850486E34BF0AD034510F0B2E
:107C9000436E4350020D0C0EF324D96E020E09D030
:107CA00034510F0B436E4350020D070EF324D96E6F
:107CB000000EF420DA6E47C0DEFF48C0DDFF030E81
:107CC0003119D8A42FD047C0D9FF48C0DAFFDFAEA2
:107CD0001CD034BF0DD034510F0B436E4350010DF7
:107CE000540EF324D96E020EF420DA6E02010CD089
:107CF000010134510F0B436E4350010DA00EF324CC
:107D0000D96E010EF420DA6EDF8247C0D9FF48C079
:107D1000DAFF000EDB8447C0D9FF48C0DAFF000E4F
:107D2000DB8E1200040E4718476E4850486E47C05D
:107D3000D9FF48C0DAFFDFAE1BD047C0D9FF48C02B
:107D4000DAFF7F0EDF1647C0D9FF48C0DAFF000E0A
:107D5000DB8C000E3C6E050E3B6E47C03DF048C00C
:107D60003EF0000E406E020E3F6EFDEC69F006D054
:107D700047C0D9FF48C0DAFF000EDB8C040E47185D
:107D8000476E4850486E46B206D047C0D9FF48C03B
:107D9000DAFFDFAE32D0010134BF0DD034510F0B0A
:107DA000436E4350010D540EF324D96E020EF4209D
:107DB000DA6E02010CD0010134510F0B436E4350B7
:107DC000010DA00EF324D96E010EF420DA6EDF92BD
:107DD00047C0D9FF48C0DAFF3B0EDF16000E3C6EED
:107DE000050E3B6E47C03DF048C03EF0000E406EB1
:107DF000020E3F6EFDEC69F006D047C0D9FF48C0C7
:107E0000DAFF3B0EDF16010134510F0B436E435076
:107E1000010DFF0EF324446E0D0EF420456E44C098
:107E2000D9FF45C0DAFFFE0EDF1612007A0E000100
:107E3000856F000E866F12D1250E8B19D8B409D02C
:107E400076C0D9FF77C0DAFF8BC0DFFF764B772B88
:107E500005D1000E826F34D0828932D085C0D9FF1F
:107E600086C0DAFFDECF83F0DDCF84F0020E8527F7
:107E7000000E862383518411D8A416D0630E836F1D
:107E8000150E846F11D083C0F6FF84C0F7FF000E7B
:107E9000F86E76C0D9FF77C0DAFF0800F5CFDFFFB4
:107EA000834B842B764B772B83C0F6FF84C0F7FF80
:107EB000000EF86E0800F5500009D8B4CFD0E3D713
:107EC00078C0F6FF79C0F7FF784B792B000EF86E7B
:107ED0000800F5CF8BF08B51000AD8B4CDD0640ADE
:107EE000D8B40AD00D0AD8B407D0050AD8B4B4D78C
:107EF0001F0AD8B4B3D7B2D082A90ED085C0D9FF9B
:107F000086C0DAFFDECF87F0DECF88F0DECF89F0E3
:107F1000DECF8AF0040E0ED085C0D9FF86C0DAFF0E
:107F2000DECF87F0DDCF88F0000E88BFFF0E896FAF
:107F30008A6F020E8527000E86238AAF0AD0030EB1
:107F400082138A1F891F881F876D000E882389234B
:107F50008A23010E8B6F0A0E8B19D8B41BD08B515C
:107F6000040D2A0EF324F66E130EF420F76EF86A51
:107F7000000EF8220900F550875D0900F550885978
:107F80000900F55089590900F5508A59D8A002D046
:107F90008B2BE1D782C07EF0030E7E17D8B408D0B9
:107FA00076C0D9FF77C0DAFF2D0EDF6E764B772BC8
:107FB0008B51806F816B80BF810748D080C07EF07D
:107FC00081C07FF0D8907E377F37D8907E377F375B
:107FD0002A0E7E25F66E130E7F21F76EF86A000ECC
:107FE000F8220900F5CF64F00900F5CF65F009002B
:107FF000F5CF66F00A00F5CF67F087C060F088C063
:1080000061F089C062F08AC063F081EC68F060C002
:108010006DF061C06EF062C06FF063C070F00A0E68
:108020000001716F000E726F000E736F000E746F9F
:10803000A1EC6AF000016D51300F8B6F76C0D9FF53
:1080400077C0DAFF8BC0DFFF764B772B8007D8A095
:1080500081078029B3E18129D8A4B0D778C0F6FF81
:1080600079C0F7FF784B792B000EF86E0800F5CF3A
:108070008BF08B51D8A4E0D676C0D9FF77C0DAFF59
:10808000000EDF6E1200000E0001826F000E816F85
:10809000000E606F070E616F000E636F6269020E63
:1080A000656F000E646F29EC70F094EC6FF0000EB9
:1080B00000016C6F070E6D6FD5EC6AF00009D8A453
:1080C0005ED0000E00018125606F070E8221616F76
:1080D000210E626F150E636F000E656F0B0E646FDD
:1080E0006CEC6BF00B0E00018127000E8223000E5A
:1080F0008125606F070E8221616F430E626F150E3E
:10810000636F000E656F020E646F6CEC6BF0020E15
:1081100000018127000E8223000E8125606F070E6B
:108120008221616FE10E626F140E636F000E656F46
:10813000110E646F6CEC6BF0110E00018127000EC4
:108140008223000E8125606F070E8221616F430E2E
:10815000626F150E636F000E656F020E646F6CEC3C
:108160006BF0020E00018127000E822394EC6FF069
:10817000000E0001676F070E686F85EC69F0460E10
:108180000201956F280E966F2788000E976F000EDC
:10819000986F000E01014D6F000E02019B6F000EE3
:1081A0009A6F000E9C6F000E9E6F000E9D6F000E6A
:1081B0009F6F000EA16F000EA06F000EA36F000E48
:1081C000A26F000EA56F000EA46F000EA76F000E29
:1081D000A66F000EA96F000EA86F000EAB6F000E09
:1081E000AA6F000E01014C6F000E0001826F000E9D
:1081F000816F020E825DD8B028D0000E8125D96E25
:10820000070E8221DA6E240EDE18D8A41BD0010ED0
:1082100081257E6F000E82217F6F000E7E25666FA6
:10822000070E7F21676F7EEC5DF000016651806F65
:1082300081C07AF082C07BF0805151EC2AF00001BD
:10824000814B822B814B822BD4D702019751D8A42A
:1082500003D035EC6AF015D0030E0101BF19D8A484
:1082600005D0BF80BF92BF84BF96BF98060EBF19CE
:10827000D8A405D0BF90BF82BF94BF96BF98B6EC7C
:1082800067F00E0E226E02019751D8B402D0020E92
:1082900022269851D8B402D0090E2226000E5E6F15
:1082A000960E5D6F01014D05D8A405D0010E0201A7
:1082B0005E6F2C0E5D6F279625901200000E000158
:1082C000786F35EC6AF000C570F00F0E0001701782
:1082D00070C000F50101CFA707D000C570F0400EB7
:1082E0000001701370C000F50101CFAB07D000C5CD
:1082F00070F0200E0001701370C000F50101CFA9CD
:1083000007D000C570F0100E0001701370C000F5AA
:10831000000E0001776F000E786F0BD07851010DC1
:10832000000EF324D96E050EF420DA6EDF50771BB1
:10833000782BFF0E706FFF0E716F2250726F736B90
:1083400070517227715173237851746F756B72512C
:10835000745D7551800A766F7351800A7659D8A082
:10836000DDD77851010D000EF324D96E050EF420EF
:10837000DA6E77C0DFFF25B67CD022C070F0716B5B
:10838000726B736B7051155E7151165A7251175A98
:108390007351185A000E0101CE6F000E0001786F64
:1083A00021D07851010D000EF324D96E070EF42070
:1083B000DA6E78511524626F000E1620636F000E7E
:1083C0001720646F000E1820656F7AEC6FF00001C3
:1083D000716FDE507119D8B403D0010E0101CE6F58
:1083E0000001782B2250785DD8A0DBD70101CE5157
:1083F000D8B439D0320E0001606F070E616F000EE5
:10840000636F000E626F000E656F200E646F29ECC3
:1084100070F015C066F016C067F017C068F018C09D
:1084200069F0320E00016A6F070E6B6F22C06CF0AC
:108430006D6B3BEC6BF022501526000E16221722B6
:10844000182215C066F016C067F017C068F018C093
:1084500069F0000E00016A6F070E6B6F22C06CF0AE
:108460006D6B3BEC6BF022501526000E1622172286
:10847000182215C066F016C067F017C068F018C063
:1084800069F0000E00016A6F050E6B6F22C06CF080
:108490006D6B3BEC6BF0000E0001786F13D07851E0
:1084A000010D000EF324D96E050EF420DA6E78511A
:1084B000010D000EF324E16E070EF420E26EDFCF13
:1084C000E7FF782B2250785DD8A0E9D722501526F7
:1084D000000E16221722182226902596B6EC67F079
:1084E000120002019751D8A405D0000E666F000E4D
:1084F000656F02D0D2EC55F065C28AF266C28BF28B
:1085000002019751D8B40BD06551595D66515A5943
:10851000D8B00FD065C259F266C25AF20AD0B5512E
:10852000595DB6515A59D8B004D0B5C259F2B6C245
:108530005AF21DB015D09805D8A412D034C38CF2CD
:1085400035C38DF236C38EF237C38FF238C390F243
:1085500039C391F23AC392F23BC393F23CC394F213
:1085600027A209D027920E01E885E883E8878B943B
:10857000010EFFEC4FF00201AC9327A823D027AAED
:108580000DD00E01E895E893E897020EFFEC4FF04E
:108590008B84278227980201AC83279A9651360D47
:1085A0008651F35C8751F458D8B00CD00E01E89591
:1085B000E893E8978B94020EFFEC4FF02782279800
:1085C0000201AC83ACC27DF21DA032D07D81020ECF
:1085D0007E6F000E7F6F000E806F000E816F030EA6
:1085E000826F000E836F000E846F000E856F000E89
:1085F000876F866986C2B5F287C2B6F2000E896FB0
:10860000040E886F9805D8A42BD034C38CF235C3E0
:108610008DF236C38EF237C38FF238C390F239C36E
:1086200091F23AC392F23BC393F23CC394F218D056
:10863000B1C282F2B2C283F2B3C284F2B4C285F292
:10864000ADC27EF2AEC27FF2AFC280F2B0C281F2A2
:10865000B7C286F2B8C287F2B9C288F2BAC289F24A
:10866000000E646F000E636F000E0001ED6F0C0EC4
:10867000ED6501D00FD0ED51010DF3500201F4254D
:10868000D96EF450F521DA6EDF506AEC71F000011A
:10869000ED2BEDD702019751D8B416D0000E000192
:1086A000ED6F010EED6501D00FD0ED51010DF350CE
:1086B0000201F025D96EF450F121DA6EDF506AEC38
:1086C00071F00001ED2BEDD702019805D8A416D06A
:1086D000000E0001ED6F080EED6501D00FD0ED51D9
:1086E000010DF3500201F225D96EF450F321DA6E38
:1086F000DF506AEC71F00001ED2BEDD726801200FF
:108700008D908D922050D8B4120027B203D0010E64
:10871000FFEC4FF02950D8A44CD0010E296E205008
:108720008CEC6EF000C35BF101C35CF102C35DF140
:1087300003C35EF1BDEC49F018EC59F0000E0D6E6C
:10874000000E0E6E000E0F6E000E106E000E010178
:108750005B6F000E5C6F000E5D6F000E5E6FBDEC18
:1087600049F092EC5FF00DC078F10EC079F10FC0C6
:108770007AF110C07BF10DC074F10EC075F10FC01D
:1087800076F110C077F178C160F079C161F07AC1FB
:1087900062F07BC163F074C164F075C165F076C1AD
:1087A00066F077C167F0010E0001686FC3EC69F0F5
:1087B0001200000E296E0101B251D8B4120002015C
:1087C0009751D8B407D05BC272F05CC273F0ADECC5
:1087D0006EF004D002015B516BEC6EF016C25BF1DF
:1087E00017C25CF118C25DF119C25EF1BDEC49F02F
:1087F00018EC59F000C3EBF001C3ECF002C3EDF04C
:1088000003C3EEF00001EB1FEC1FED1FEE1FEB2B7F
:10881000000EEC23ED23EE23020116510001EB259F
:108820000D6E020117510001EC210E6E020118516C
:108830000001ED210F6E020119510001EE21106EB1
:108840000DC06CF00EC06DF00FC06EF010C06FF078
:10885000010E6AEC4AF06CC07EF06DC07FF06EC015
:1088600080F06FC081F0CDEC6EF07EC0E1F07FC093
:10887000E2F080C0E3F081C0E4F0A0EC5CF0E1C085
:108880005BF1E2C05CF1E3C05DF1E4C05EF1BDEC20
:1088900049F092EC5FF00DC078F10EC079F10FC095
:1088A0007AF110C07BF10DC074F10EC075F10FC0EC
:1088B00076F110C077F178C160F079C161F07AC1CA
:1088C00062F07BC163F074C164F075C165F076C17C
:1088D00066F077C167F0010E0001686FC3EC69F0C4
:1088E0001200000E0001766FC50E746F030E756FD7
:1088F00035EC6AF001019F5108E1CC0E9C5DFF0E42
:108900009D591F0E9E59D8A007D026922598F9ECA4
:108910006FF0B6EC67F0120025B885D0340E9C5F7E
:10892000000E9D5B9E5B9F5B000ECE6F000E0001F4
:10893000766F330E766501D02FD07651706F716BE4
:10894000800E7027000E7123000E7025D96E070E61
:108950007121DA6E765101019C250001626F000ED3
:1089600001019D210001636F000E01019E210001A4
:10897000646F000E01019F210001656F7AEC6FF0BA
:108980000001736FDE507319D8B403D0010E0101DA
:10899000CE6F0001762BCDD70101CE51D8B43CD09B
:1089A000800E0001606F070E616F000E636F000E96
:1089B000626F000E656F340E646F29EC70F09CC11D
:1089C00066F09DC167F09EC168F09FC169F0800E9E
:1089D00000016A6F070E6B6F000E6D6F340E6C6FC7
:1089E0003BEC6BF0340E01019C27000E9D239E236F
:1089F0009F239CC166F09DC167F09EC168F09FC136
:108A000069F074C06AF075C06BF0000E00016D6F04
:108A1000340E6C6F3BEC6BF0340E01019C27000EA2
:108A20009D239E239F239CC166F09DC167F09EC13C
:108A300068F09FC169F074C06AF075C06BF0000EF9
:108A400000016D6F340E6C6F3BEC6BF0000E00019B
:108A5000766F330E766501D019D07651010DF35043
:108A60007425D96EF4507521DA6E7651706F716B82
:108A7000800E7027000E7123000E7025E16E070E28
:108A80007121E26EDFCFE7FF762BE3D7340E0101D1
:108A90009C27000E9D239E239F2326922598F9EC68
:108AA0006FF0B6EC67F01200000E00016D6F000E63
:108AB0006C6F240E0F012E6F2E95900E2F6F2F8945
:108AC000000E2D6F2D97670E2B6F000E2C6F2A5105
:108AD000618AA98A2A510E01E8971DA205D01DECD2
:108AE00071F00E01E88712008F80239645EC71F03B
:108AF0000F012F89000E00016D6F000E6C6F6D511C
:108B00000EE10A0E6C5DD8B00AD0050E626F150E2C
:108B1000636F28EC46F000016C4B6D2BF0D71DEC19
:108B200071F00F012A51FA0ECFEC71F0FA0ECFEC72
:108B300071F0FA0ECFEC71F0FA0ECFEC71F0FA0E84
:108B4000CFEC71F0FA0ECFEC71F0FA0ECFEC71F0C1
:108B5000FA0ECFEC71F023A6C9D7000E00016D6F9D
:108B6000000E6C6F6D510BE1030E6C5DD8B007D039
:108B7000FA0ECFEC71F000016C4B6D2BF3D71DECAE
:108B800071F0000E00016D6F000E6C6F6D5129E1E8
:108B9000320E6C5DD8B025D023960101C39123908D
:108BA00023A6FED723B6A8EC47F023B01AD00101C4
:108BB000C3A113D0C7EC6FF00E01E8872796E897A2
:108BC000E893E895FA0ECFEC71F0FA0ECFEC71F065
:108BD0000E01E887E883E885120000016C4B6D2BDD
:108BE000D5D7FA0ECFEC71F0FA0ECFEC71F0B20ED1
:108BF0000001626F140E636F28EC46F023B6A8ECF8
:108C000047F023A4F4D7140E0001626F150E636FB2
:108C100028EC46F023B6A8EC47F023A2F4D70E01C7
:108C2000E8872796E599E595E597E593FA0ECFEC69
:108C300071F0FA0ECFEC71F0FA0ECFEC71F0FA0E83
:108C4000CFEC71F00E01E589E585E587E58312003B
:108C5000000E00016B6F240E53EC72F0000E000149
:108C6000616F0A0E606FF7EC71F0000E00016A6F21
:108C700030D06A51010D62C064F063C065F0F350FA
:108C80006427F450652364C0F6FF65C0F7FF000E4B
:108C9000F86E0800F5506B1B6A51010D62C064F05C
:108CA00063C065F0F3506427F450652364C0F6FF99
:108CB00065C0F7FF000EF86E0800F55053EC72F037
:108CC000000E0001616F0A0E606FF7EC71F0000199
:108CD0006A2B6A51010D62C064F063C065F0F35005
:108CE0006427F450652364C0F6FF65C0F7FF000EEB
:108CF000F86E0800F5502A0AD8A4BBD72A0E53EC08
:108D000072F0000E0001616F0A0E606FF7EC71F0F7
:108D10006BC064F00001643B0F0E64170F0E641704
:108D20000A0E646109D06BC064F0643B0F0E6417D7
:108D30000F0E6417300E08D06BC064F0643B0F0E4A
:108D400064170F0E6417370E6425666F676B000E8D
:108D50006723665153EC72F0000E0001616F0A0E3A
:108D6000606FF7EC71F06BC064F00F0E00016417D8
:108D70000A0E646106D06BC064F00F0E6417300EEB
:108D800005D06BC064F00F0E6417370E6425686F52
:108D9000696B000E6923685153EC72F0000E0001FC
:108DA000616F0A0E606FF7EC71F00D0E53EC72F00C
:108DB000000E0001616F0A0E606FF7EC71F00A0E91
:108DC00053EC72F0000E0001616F0A0E606FF7EC59
:108DD00071F01200000E0E01476F000E466F000E7C
:108DE000456F939892909286929C929E93809392D4
:108DF000939493969398939A939C939EF18E000EDE
:108E0000626E9490949294949488949A959095928A
:108E1000969096929684969E9784979A978C978E22
:108E200098909892988498869898989C989E998003
:108E3000998299849986998C998E9A949A869A8C1B
:108E40009A8E0F0154850E01E993E995E997E99906
:108E5000E99B0F0154930E01E691E693E695E697A0
:108E6000E699F89F669C200E2E6F400E166F300E0E
:108E7000156F220E1A6F440E2C6F668C000E0001C7
:108E8000606F000E616F000E0AEC6FF0240E0F0190
:108E90002E6F2E95900E2F6F2F89000E2D6F2D9710
:108EA000670E2B6F000E2C6F2A51CA68000ECC6E15
:108EB000E10ECB6E9F820469D280C19E0E01458F68
:108EC000478D000EC16E700EC06E000E8D6F000ECD
:108ED0008C6F0A0E8B6F0C0E8A6F000E896F000E5E
:108EE000886FC18E9E9CB60E0F01536F900EBE6EA2
:108EF000BF80BF92BF84BF96BF98A6906180000ECE
:108F0000AA6ECD86CD9ECD9CCD82CD8ACD88000E19
:108F1000CF6E000ECE6ECD80619261949D809D8259
:108F2000B780D08EA98AF28CF28E0E01E885E88394
:108F3000E887E583E587E585E5890F015485389F56
:108F4000379F548B8F8035EC6AF0B6EC67F01200D7
:108F50004B0E04017C19D8A45DD0300E7D19D8A425
:108F600059D0300E7E19D8A455D0310E7F19D8A40F
:108F700051D0330E8119D8A417D0310E8219D8A43C
:108F800013D0340E8319D8A40FD0330E8519D8A46A
:108F90000BD0330E8719D8A407D0360E8819D8A461
:108FA00003D0238423961200320E8119D8A417D03F
:108FB000320E8219D8A413D0300E8319D8A40FD042
:108FC000330E8519D8A40BD0330E8719D8A407D037
:108FD000300E8819D8A403D0238223961200310EB4
:108FE0008119D8A417D0360E8219D8A413D0310E07
:108FF0008319D8A40FD0330E8519D8A40BD0330E03
:109000008719D8A407D0360E8819D8A403D023888E
:10901000239612004B0E7C19D8A42AD0300E7D194D
:10902000D8A426D0310E7E19D8A422D0300E7F19B4
:10903000D8A41ED0300E8119D8A40BD0300E8219BE
:10904000D8A407D0310E8319D8A403D0238C23963B
:109050001200300E8119D8A40BD0300E8219D8A47A
:1090600007D0320E8319D8A403D0238E2396120082
:10907000470E7919D8A40DD0500E7A19D8A409D06A
:10908000520E7B19D8A405D00101C39127802396E5
:109090001200470E04017919D8A412004E0E7A1955
:1090A000D8A41200520E7B19D8A4120027900101F7
:1090B000C381239612000001F46F0001F4514AECC1
:1090C0006EF00001F451040DC50EF324D96E030EA9
:1090D000F420DA6EDECFECF0DECFEDF0DECFEEF096
:1090E000DECFEFF0F451040D000EF324D96E030E21
:1090F000F420DA6EDECFF0F0DECFF1F0DECFF2F06A
:10910000DECFF3F0F01FF11FF21FF31FF02B000E64
:10911000F123F223F323EC51F0250101806F0001CC
:10912000ED51F1210101816F0001EE51F2210101A8
:10913000826F0001EF51F3210101836F00C3ECF056
:1091400001C3EDF002C3EEF003C3EFF00001EC1F2A
:10915000ED1FEE1FEF1FEC2B000EED23EE23EF2390
:109160000301C5510001EC250D6E0301C65100013C
:10917000ED210E6E0301C7510001EE210F6E0301B8
:10918000C8510001EF21106EEB05D8A410D0F451A6
:10919000040DC50EF324D96E030EF420DA6EDECF73
:1091A0005BF1DECF5CF1DECF5DF1DECF5EF1EB5146
:1091B000D8A408D080C15BF181C15CF182C15DF1AE
:1091C00083C15EF1BDEC49F092EC5FF080C178F1B3
:1091D00081C179F182C17AF183C17BF10DC074F153
:1091E0000EC075F10FC076F110C077F178C160F054
:1091F00079C161F07AC162F07BC163F074C164F03F
:1092000075C165F076C166F077C167F0010E0001A7
:10921000686FC3EC69F01200A098020171517211DD
:10922000D8B408D071C2D9FF72C2DAFFDFAE02D063
:10923000A0881200030E2A18D8A402D0000E2A6EAD
:109240002A50D8A402D0A0881200020E2A18D8A44E
:1092500013D0010E0001606F000E616F000E626F8F
:10926000000E636F020E4CEC53F060C071F261C0EF
:1092700072F2030E2A6E7FD02A04D8A47CD0400E4E
:109280000101D26504D0400E00016C6F02D0D2C142
:109290006CF000016C5100080101D225D26FAE0EB6
:1092A00002014E6F090E4F6F6CC06BF00101D1517E
:1092B000D8B41ED03FD051C2F6FF52C2F7FF000E05
:1092C000F86E4EC2D9FF4FC2DAFF0D0EF76403D01D
:1092D0000800F55005D0F6CFE1FFF7CFE2FFE750E9
:1092E000DF6E02014E4B4F2B514B522B00016B078F
:1092F00000016B51D8B422D0DED751C2F6FF52C262
:10930000F7FF000EF86E4EC2D9FF4FC2DAFF0D0E06
:10931000F76403D00800F55005D0F6CFE1FFF7CF92
:10932000E2FFE750DF6E02014E4B4F2B514B522BA9
:1093300000016B0700016B51D8A4DFD70101D251A6
:10934000D8A409D0400E00016C19D8A402D0020E96
:1093500001D0030E2A6E010E0001606FAE0E616F28
:10936000090E626F6CC063F0020E4CEC53F060C0EB
:1093700071F261C072F2A0881200000E0001CC6F81
:10938000000ECD6F7A0ECE6F440ECF6F5BC16CF0C6
:109390005CC16DF05DC16EF05EC16FF0010E6AECF4
:1093A0004AF06CC07EF06DC07FF06EC080F06FC080
:1093B00081F0CDEC6EF07EC0C8F07FC0C9F080C0F7
:1093C000CAF081C0CBF028EC3BF0C8C0E1F0C9C0C6
:1093D000E2F0CAC0E3F0CBC0E4F0A0EC5CF0E1C086
:1093E00058F1E2C059F158C160F059C161F0000173
:1093F000626B636BE80E646F030E656F000E666F41
:10940000000E676F0FEC6DF060C06CF061C06DF026
:1094100062C06EF063C06FF0010E6AEC4AF06CC07F
:109420007AF06DC07BF06EC07CF06FC07DF011EC07
:1094300070F07AC09BF07BC09CF07CC09DF07DC03A
:109440009EF05BC16CF05CC16DF05DC16EF05EC101
:109450006FF0010E6AEC4AF06CC07EF06DC07FF0D8
:109460006EC080F06FC081F0CDEC6EF07EC097F0E2
:109470007FC098F080C099F081C09AF0A8EC36F0D7
:1094800097C0E1F098C0E2F099C0E3F09AC0E4F030
:10949000A0EC5CF0E1C056F1E2C057F158C160F0B9
:1094A00059C161F0000E0001636F3C0E626F66EC03
:1094B0006DF00001605101015A6F5A513C0DF31ECD
:1094C000F41EF34AF42A5851F324586F5951F420EA
:1094D000596F12000001746F00017451D8A46FAF6E
:1094E0001AD06CC070F06DC071F06EC072F06FC0B9
:1094F00073F0701F711F721F731F702B000E71238A
:109500007223732370C076F071C077F072C078F068
:1095100073C079F008D06CC076F06DC077F06EC083
:1095200078F06FC079F06C516D116E116F11D8A485
:1095300009D0000E6C6F000E6D6F000E6E6F000E86
:109540006F6F1200960E756F06D0752BD890793319
:10955000783377337633000E7615706F000E7715FB
:10956000716F000E7815726FFE0E7915736F705162
:10957000711172117311D8B40DD0E7D7752B010E8C
:109580007627000E772378237923D89079337833A0
:1095900077337633000E7615706F000E7715716F86
:1095A000000E7815726FFF0E7915736F705171117F
:1095B00072117311D8B407D0E1D77507D8907637F8
:1095C00077377837793778BF03D0020E7561F5D7D2
:1095D00075B108D0FF0E7617FF0E77177F0E78173C
:1095E000FF0E7917D890753375C070F0716B726B80
:1095F000736B70C073F0726B716B706B705176131C
:109600007151771372517813735179137451D8A42F
:109610006FAF01D0798F76C06CF077C06DF078C0F5
:109620006EF079C06FF01200000E116E200E126EF7
:10963000000E136E000E146EFF0E0201326FEF0E5D
:10964000336F1F0E346F000E356F000E0001606F18
:10965000050E616F000E636F000E626F020E656F84
:10966000000E646F29EC70F074D011C062F012C06B
:1096700063F013C064F014C065F0000E0001676F62
:10968000100E666F000E686F050E696F9CEC6BF034
:1096900000C5E8FFFF0AD8A454D001C5E8FFFF0ABF
:1096A000D8A44FD002C5E8FFFF0AD8A44AD003C50A
:1096B000E8FFFF0AD8A445D004C5E8FFFF0AD8A4F4
:1096C00040D005C5E8FFFF0AD8A43BD006C5E8FF97
:1096D000FF0AD8A436D007C5E8FFFF0AD8A431D0C6
:1096E00008C5E8FFFF0AD8A42CD009C5E8FFFF0A87
:1096F000D8A427D00AC5E8FFFF0AD8A422D00BC5FA
:10970000E8FFFF0AD8A41DD00CC5E8FFFF0AD8A4C3
:1097100018D00DC5E8FFFF0AD8A413D00EC5E8FF86
:10972000FF0AD8A40ED00FC5E8FFFF0AD8A409D0BD
:1097300011C06CF012C06DF013C06EF014C06FF069
:109740001200000E1126020E1222000E1322000E2D
:10975000142202013251115C335112583451135802
:1097600035511458D8A081D711C06CF012C06DF0DB
:1097700013C06EF014C06FF012002D04D8B475BA87
:1097800007D0000E786E0E0110811089020E2D6E2A
:1097900078A406D00E0110A503D0789443EC6FF0A6
:1097A00075A202D0A198120078A009D00E0110A1D4
:1097B00006D00AEC4DF0A088040E2D6E789078A8A3
:1097C00004D00E0110B959EC70F078AC1CD00E0129
:1097D00010AD0ED0000E3C6E730E3B6E000E3D6E53
:1097E000000E3E6E000E406E010E3F6EFDEC69F005
:1097F000789C9EEC71F00101D951D8A4D907D951B8
:10980000D8B4C7EC60F078AA04D00E0110BB28ECE5
:109810006EF078A212D00E0110A30FD07F0E3C6E16
:109820003B68000E3D6E000E3E6E000E406E010E57
:109830003F6EFDEC69F0000E776E040E2D6002D0D5
:10984000A19812000E0110A73ED0000E4A6E030E22
:109850004A6401D038D078A636D076CF2EF02E309C
:10986000E832E8320F0B0101DB6F78962EB40AD094
:10987000DB51010D540EF324D96E020EF420DA6E82
:10988000020109D00101DB51010DA00EF324D96EB4
:10989000010EF420DA6EDF700101DB51D8A403D091
:1098A000DBEC64F00ED0000E3C6E720E3B6E2E0EA2
:1098B0003D6E000E3E6E000E406E000E3F6EFDECE3
:1098C00069F04A2AC4D7A19812000101BB69000EB1
:1098D0000001FA6F000E216E000EEB6F0C0EEB65AF
:1098E00001D00ED0EB51040DC50EF324D96E030E3A
:1098F000F420DA6EDE6ADE6ADE6ADD6AEB2BEED712
:10990000000E0201126F000E136F000E146F000E96
:10991000156F000E0101846F000E856F000E866FBB
:10992000000E876F000E886F000E896F000E8A6F21
:10993000000E8B6F000E806F000E816F000E826F25
:10994000000E836F000E0D6E000E0E6E000E0F6E79
:10995000000E106E000E7C6F000E7D6F000E7E6F8D
:10996000000E7F6F000E786F000E796F000E7A6F19
:10997000000E7B6F000E746F000E756F000E766F19
:10998000000E776F010EFFEC4FF00E01E887E885BF
:10999000E883000E0101B26F000E02015C6F000E41
:1099A0005B6FC00E1A6F270E1B6F090E1C6F000E27
:1099B0001D6FC00E166F270E176F090E186F000E61
:1099C000196F000E01015B6F000E5C6F000E5D6F82
:1099D000000E5E6F000E746F000E756F000E766FD6
:1099E000000E776F000E786F000E796F000E7A6FA1
:1099F000000E7B6FBDEC49F018EC59F092EC5FF073
:109A0000000E0201BE6F000EBF6F000EC06F000E91
:109A1000C16F1200A098000E776E000E786E000ED7
:109A20000D01FF6F000E2F6E0E0E306E000E326EA7
:109A3000000E316E000E346E020E336EB6EC70F016
:109A4000160E0E01116F9F0E0F6F7B0E106F000E22
:109A5000376E0B0E376401D00ED03750040D000E58
:109A6000F324D96E010EF420DA6EDE6ADE6ADE6A55
:109A7000DD6A372AEED7758C000E746E7598759C6A
:109A80007896000E046E000E0101626F000E646F86
:109A9000000E636F78B6F4D7010ED76F010ED66F44
:109AA000000ED56F000ED46F000EDC6F000E376E07
:109AB000020E376401D02ED03750020D070EF3246A
:109AC000D96E000EF420DA6E000EDE6E000EDD6E32
:109AD0003750020D0C0EF324D96E020EF420DA6E0C
:109AE000000EDE6E000EDD6E3750010DA00EF32469
:109AF000D96E010EF420DA6E000EDF6E3750010DC4
:109B0000540EF324D96E020EF420DA6E000EDF6ECE
:109B1000372ACED7080E076E010E086E160E0D01FD
:109B2000FF6F010E0101036F300E026F080E016F0F
:109B3000040E006F008F000EDF6F000E02014A6FEF
:109B4000000E4B6F000E4C6F000E4D6F000E0101AA
:109B5000D36F000E2D6E1200800E01013019D8A4B3
:109B60001200C00E046E82D0F30E016E140E026E4F
:109B7000000E066E120E056E12003251D8A442D0AD
:109B80003251020D050EF324F66E140EF420F76E1A
:109B9000F86A000EF8220900F5CF01F00A00F5CFAF
:109BA00002F0020E01242F6E000E0220306E2FC034
:109BB000F6FF30C0F7FF000EF86E0D0EF76403D00D
:109BC0000800F55005D0F6CFE1FFF7CFE2FFE750F0
:109BD000056E030E01242F6E000E0220306E2FC082
:109BE000F6FF30C0F7FF000EF86E0D0EF76403D0DD
:109BF0000800F55005D0F6CFE1FFF7CFE2FFE750C0
:109C0000066E1200000E046E1200030E0101326196
:109C100027D03251020DFC0EF324F66E130EF42001
:109C2000F76EF86A000EF8220900F5CF01F00A007D
:109C3000F5CF02F001C0F6FF02C0F7FF000EF86E8C
:109C40000D0EF76403D00800F55005D0F6CFE1FF04
:109C5000F7CFE2FFE7502F6E2F50056E066A120015
:109C6000000E046E1200000E046E1200010133514A
:109C7000010AD8B479D7030AD8B47FD7010AD8B477
:109C8000C4D7F1D70101C289C18E080EBD6F090E7C
:109C9000BD6501D047D0BD51010DBC0EF324F66E59
:109CA000130EF420F76EF86A000EF8220800F5CFC4
:109CB00086FEBD51010DBC0EF324F66E130EF4208A
:109CC000F76EF86A000EF8220800F5CF87FEC18E05
:109CD000C082050E0DEC72F0C0A0FED7C3CF69F0B4
:109CE00000016A6B69516A6F696BC250691369C080
:109CF00067F06AC068F0D89068336733D8906833EB
:109D000067330101BD51020D3E0EF324D96E030EDF
:109D1000F420DA6E00016751DE266851DD22010170
:109D2000BD2BB5D7C19E0301522B080E5219D8A4E2
:109D30003BD0000E00016A6F000E696F6A512FE17F
:109D40000A0E695DD8B02BD0340E6925D96E030E8A
:109D50006A21DA6ED8906935E16E6A35E26E3E0EA0
:109D6000E126030EE222E6CF60F0E5CF61F052C3B8
:109D700062F0636B66EC6DF000016051DF6ED890AD
:109D80006935D96E6A35DA6E3E0ED926030EDA22AF
:109D9000000EDE6E000EDD6E694B6A2BCFD7000E13
:109DA0000301526F3DC3C1F10101C2991200000EBF
:109DB0000001626F000E616F31D0B5C261F0B6C2B2
:109DC00062F03DD08AC261F08BC262F038D021C00F
:109DD00061F00001626B33D0000E0201A76F140E18
:109DE000A66F01017FBF2BD07F517E117D110BE14A
:109DF0007C05D8A024D007D0000EA76F140EA66F44
:109E000001017FAF1CD0000E0001626F0A0E616F6E
:109E1000000E0201A76F000EA66F11D00201A4511F
:109E2000010AD8B4CAD7030AD8B4CCD7010AD8B427
:109E3000CED7070AD8B4E0D7010AD8B4CDD70201EB
:109E4000A6510001615D0201A75100016259D8B01D
:109E500007D00A0E0101FE6F0E01E8838D921200F9
:109E60000201A505D8A404D00E01E8938D8212004A
:109E7000020E0201A519D8A427D00101FE51D8B4C1
:109E800023D00E01E8A302D0010E01D0000EFF0A7C
:109E90000001606F60470E01E85100016019FD0B81
:109EA00060190E01E86F0101FE078DA202D0010EBC
:109EB00001D0000EFF0A0001606F60478D506019ED
:109EC000FD0B60198D6E1200000E0101FE6F0E0178
:109ED000E8838D921200000E0001626F000E616F28
:109EE00031D0B5C261F0B6C262F03DD08AC261F035
:109EF0008BC262F038D021C061F00001626B33D0B8
:109F0000000E0201AB6F140EAA6F01017FBF2BD0B0
:109F10007F517E117D110BE17C05D8A024D007D0A4
:109F2000000EAB6F140EAA6F01017FAF1CD0000EA4
:109F30000001626F0A0E616F000E0201AB6F000E2E
:109F4000AA6F11D00201A851010AD8B4CAD7030AD6
:109F5000D8B4CCD7010AD8B4CED7070AD8B4E0D742
:109F6000010AD8B4CDD70201AA510001615D0201F6
:109F7000AB5100016259D8B007D00A0E0101FD6F44
:109F80000E01E8858D9012000201A905D8A404D025
:109F90000E01E8958D801200020E0201A919D8A4C5
:109FA00027D00101FD51D8B423D00E01E8A502D07D
:109FB000010E01D0000EFF0A0001606F604760478C
:109FC0000E01E85100016019FB0B60190E01E86FEA
:109FD0000101FD078DA002D0010E01D0000EFF0A85
:109FE0000001606F8D506019FE0B60198D6E1200BC
:109FF000000E0101FD6F0E01E8858D901200000139
:10A00000616F84D01FAC12000101B12B140EB11985
:10A01000D8A416D00E01E585E5831FB6E5951FBAD5
:10A02000E5931F9C000E0101B16F1FAE12000E01DF
:10A03000E589E5871FB4E5991FB8E5971F9E1200D3
:10A040001FA613D00E01E5A502D0010E01D0000E0F
:10A05000FF0A0001606F604760470E01E551000193
:10A060006019FB0B60190E01E56F1FAA12D00E01DB
:10A07000E5A302D0010E01D0000EFF0A0001606FBF
:10A0800060470E01E55100016019FD0B60190E01DA
:10A09000E56F1FAE12001FA412D00E01E5A902D079
:10A0A000010E01D0000EFF0A0001606F603B0E013F
:10A0B000E55100016019EF0B60190E01E56F1FA853
:10A0C00012000E01E5A702D0010E01D0000EFF0A1A
:10A0D0000001606F6047604760470E01E551000175
:10A0E0006019F70B60190E01E56F12000E01E5858E
:10A0F000E583E589E5871F941F961F981F9A120034
:10A100000E01E595E593E599E5971200000161518F
:10A11000000AD8B477D7010AD8B4E8D7030AD8A47C
:10A120001200EED7000E0001AB15B36F000EAC1598
:10A13000B46F800EAD15B56F7F0EAE15B66FB3510F
:10A14000B411B511B611D8A408D0000EAB6F000E33
:10A15000AC6F000EAD6F000EAE6F000EAF15B36F9B
:10A16000000EB015B46F800EB115B56F7F0EB2152D
:10A17000B66FB351B411B511B611D8A408D0000E02
:10A18000AF6F000EB06F000EB16F000EB26FAEAFCA
:10A190001DD0ABC0B3F0ACC0B4F0ADC0B5F0AEC034
:10A1A000B6F0B31FB41FB51FB61FB32B000EB423F8
:10A1B000B523B623000EB325AB6F000EB421AC6FF0
:10A1C000000EB521AD6F800EB621AE6FB2AF1DD0BF
:10A1D000AFC0B3F0B0C0B4F0B1C0B5F0B2C0B6F02B
:10A1E000B31FB41FB51FB61FB32B000EB423B52386
:10A1F000B623000EB325AF6F000EB421B06F000E72
:10A20000B521B16F800EB621B26F000EAB1B000EF0
:10A21000AC1B000EAD1B800EAE1B000EAF1B000E64
:10A22000B01B000EB11B800EB21BAF51AB5DB05125
:10A23000AC59B151AD59B251AE59D8B002D0D89045
:10A240001200D88012000001F06F0001F051D8B464
:10A250001200F05161EC60F00001F0518CEC6EF0F6
:10A26000C5C35BF1C6C35CF1C7C35DF1C8C35EF192
:10A27000BDEC49F018EC59F000C3ECF001C3EDF06F
:10A2800002C3EEF003C3EFF00001EC1FED1FEE1F61
:10A29000EF1FEC2B000EED23EE23EF230301C5513E
:10A2A0000001EC250D6E0301C6510001ED210E6E7B
:10A2B0000301C7510001EE210F6E0301C8510001D7
:10A2C000EF21106E0DC06CF00EC06DF00FC06EF07F
:10A2D00010C06FF0010E6AEC4AF06CC07EF06DC0E9
:10A2E0007FF06EC080F06FC081F0CDEC6EF07EC06C
:10A2F000E1F07FC0E2F080C0E3F081C0E4F0A0ECC8
:10A300005CF0E1C05BF1E2C05CF1E3C05DF1E4C090
:10A310005EF1BDEC49F092EC5FF00DC078F10EC03B
:10A3200079F10FC07AF110C07BF10DC074F10EC04D
:10A3300075F10FC076F110C077F178C160F079C186
:10A3400061F07AC162F07BC163F074C164F075C1E1
:10A3500065F076C166F077C167F0010E0001686FA5
:10A36000C3EC69F012000001606F0E01929F9A9F8A
:10A37000A29FAA9FAA9DA29D9A9D929D080E000150
:10A3800060655DD0080E606F5AD00E01929F9A9F53
:10A39000A29FAA9FAA9DA29D9A9D929D12000E0126
:10A3A000928F9A9FA29FAA9FAA9DA29D9A9D929DDD
:10A3B00012000E01928F9A8FA29FAA9FAA9DA29D22
:10A3C0009A9D929D12000E01928F9A8FA28FAA9F42
:10A3D000AA9DA29D9A9D929D12000E01928F9A8F26
:10A3E000A28FAA8FAA9DA29D9A9D929D12000E01F6
:10A3F000928F9A8FA28FAA8FAA8DA29D9A9D929DCD
:10A4000012000E01928F9A8FA28FAA8FAA8DA28D11
:10A410009A9D929D12000E01928F9A8FA28FAA8F01
:10A42000AA8DA28D9A8D929D12000E01928F9A8F05
:10A43000A28FAA8FAA8DA28D9A8D928D12000001F3
:10A440006051000AD8B4A1D7010AD8B4A8D7030A2A
:10A45000D8B4AFD7010AD8B4B6D7070AD8B4BDD795
:10A46000010AD8B4C4D7030AD8B4CBD7010AD8B4E8
:10A47000D2D70F0AD8A41200D8D7000E116EF00E52
:10A48000126E1F0E136E000E146EFF0E0201326F5D
:10A49000FF0E336F1F0E346F000E356F750E000107
:10A4A000606F030E616F000E636F000E626F000E2F
:10A4B000656F500E646F29EC70F053D011C062F0DC
:10A4C00012C063F013C064F014C065F0000E000108
:10A4D000676F100E666F750E686F030E696F9CECE8
:10A4E0006BF003017529D8A436D07629D8A433D0CF
:10A4F0007729D8A430D07829D8A42DD07929D8A408
:10A500002AD07A29D8A427D07B29D8A424D07C2982
:10A51000D8A421D07D29D8A41ED07E29D8A41BD0B0
:10A520007F29D8A418D08029D8A415D08129D8A4EF
:10A5300012D08229D8A40FD08329D8A40CD0842982
:10A54000D8A409D011C06CF012C06DF013C06EF029
:10A5500014C06FF01200340E1126000E12221322C6
:10A56000142202013251115C3351125834511358E4
:10A5700035511458D8A0A2D711C06CF012C06DF09C
:10A5800013C06EF014C06FF0120020EE01F01B50EB
:10A59000D9261C50DA22DF50306E30500101635D45
:10A5A000000E6459D8A063C130F03050635F000ED4
:10A5B000645B000E2F6E11D02F50010D380EF32466
:10A5C000D96E010EF420DA6E5FC1E1FF60C1E2FFD7
:10A5D000DFCFE7FF5F4B602B2F2A30502F5CD8A0D6
:10A5E000EBD763516411D8B432D020EE01F019508A
:10A5F000D9261A50DA22080EDF6E20EE02F019502A
:10A60000D9261A50DA22380EDE6E010EDD6E1BC01E
:10A61000D9FF1CC0DAFFDFBC0DD019C0D9FF1AC0AA
:10A62000DAFF480EDF6E19C0D9FF1AC0DAFF000E3C
:10A63000DB8E120019C0D9FF1AC0DAFF080EDF6ED8
:10A6400019C0D9FF1AC0DAFF000EDB8E120020EE0F
:10A6500001F01950D9261A50DA22080EDF6E20EECA
:10A6600002F01950D9261A50DA22300EDE6E010E91
:10A67000DD6E19C0D9FF1AC0DAFF040EDF6E19C0F3
:10A68000D9FF1AC0DAFF000EDB8E629FD851D8A422
:10A690001200C7EC60F012000001686F0001605109
:10A6A000D8B407D06851020D070EF324D96E000EFE
:10A6B00006D06851020D0C0EF324D96E020EF42060
:10A6C000DA6EDECF69F0DDCF6AF069516A11D8A485
:10A6D00005D0000E606F000E616F120020EE02F0D8
:10A6E0006951D9266A51DA2261C0DEFF62C0DDFFFE
:10A6F00020EE01F06951D9266A51DA2263C0DFFFEA
:10A7000069C0D9FF6AC0DAFF400EDF1669C0D9FF01
:10A710006AC0DAFF000EDB8669C0D9FF6AC0DAFFC3
:10A72000000EDB8E6051D8B418D06851020D070EB0
:10A73000F324D96E000EF420DA6EDECF64F0DDCFA4
:10A7400065F0040E6419666F6551676F6851020DFC
:10A75000070EF324D96E000E17D06851020D0C0EAF
:10A76000F324D96E020EF420DA6EDECF64F0DDCF72
:10A7700065F0040E6419666F6551676F6851020DCC
:10A780000C0EF324D96E020EF420DA6E66C0DEFFE2
:10A7900067C0DDFF69C060F06AC061F01200000EA2
:10A7A0000E018E6F000E8F6F000E906F000E916F76
:10A7B000000E926F000E936F000E946F000E956F57
:10A7C000000E966F000E976F000E986F000E996F37
:10A7D000000E9A6F000E9B6F000E9C6F000E9D6F17
:10A7E000000E9E6F000E9F6F000EA06F000EA16FF7
:10A7F000000EA26F000EA36F000EA46F000EA56FD7
:10A80000000EA66F000EA76F000EA86F000EA96FB6
:10A81000000EAA6F000EAB6F000EAC6F000EAD6F96
:10A82000000EAE6F000EAF6F000EB06F000EB16F76
:10A83000000EB26F000EB36F000EB46F000EB56F56
:10A84000000EB66F000EB76F000EB86F000EB96F36
:10A85000000EBA6F000EBB6F000EBC6F000EBD6F16
:10A86000000EBE6F000EBF6F000EC06F000EC16FF6
:10A87000000EC26F000EC36F000EC46F000EC56FD6
:10A88000000EC66F000EC76F000EC86F000EC96FB6
:10A89000000ECA6F000ECB6F000ECC6F000ECD6F96
:10A8A0001200000E0001726F000E716F000E606FDB
:10A8B000050E616F000E636F6269020E656F000E18
:10A8C000646F29EC70F0000E0001606F070E616F7D
:10A8D000000E636F6269020E656F000E646F29ECF3
:10A8E00070F0000E0101AA6F000EA96F000EA86F94
:10A8F000000EA76F37D03BEC72F0000E00016B6FBB
:10A90000070E6C6F400E6D6F8EEC64F00009D8B4CA
:10A9100029D02BC0A7F10101A86B000E296E14D01D
:10A920002950010D000EF324D96E070EF420DA6EC3
:10A93000000E0101A925E16E050EAA21E26EDFCF0E
:10A94000E7FFA94BAA2B292A295000016F6F706BD2
:10A950000101A75100016F5D0101A851000170596B
:10A96000D8A0DED70101A929010EAA59D8A0C3D7C2
:10A97000010E0001726F71690BD0000E7125D96E46
:10A98000050E7221DA6EFF0EDF6E7107D8A0720716
:10A99000000E7125D96E050E7221DA6E2A0EDE18B0
:10A9A000D8B41200EAD7376E2F50D8B407D037503A
:10A9B000020D070EF324D96E000E06D03750020D9B
:10A9C0000C0EF324D96E020EF420DA6EDECF38F0CE
:10A9D000DDCF39F038503910D8A405D0000E2F6ED5
:10A9E000000E306E120020EE02F03850D926395099
:10A9F000DA2230C0DEFF31C0DDFF20EE01F038503A
:10AA0000D9263950DA2232C0DFFF38C0D9FF39C029
:10AA1000DAFF400EDF1638C0D9FF39C0DAFF000E6A
:10AA2000DB8638C0D9FF39C0DAFF000EDB8E2F502D
:10AA3000D8B418D03750020D070EF324D96E000E8B
:10AA4000F420DA6EDECF33F0DDCF34F0040E3318AD
:10AA5000356E3450366E3750020D070EF324D96E22
:10AA6000000E17D03750020D0C0EF324D96E020ED3
:10AA7000F420DA6EDECF33F0DDCF34F0040E33187D
:10AA8000356E3450366E3750020D0C0EF324D96EED
:10AA9000020EF420DA6E35C0DEFF36C0DDFF38C0AE
:10AAA0002FF039C030F012006CC0D9FF6DC0DAFF52
:10AAB000DF500001796F6C4B6D2B200E7919D8B4E3
:10AAC000F3D7090E7919D8B4EFD7000E756F000EC1
:10AAD000766F000E776F000E786F000E746F2D0E7C
:10AAE0007919D8A402D0742B29D02B0E7919D8A4A7
:10AAF0002DD024D075C060F076C061F077C062F0D0
:10AB000078C063F00A0E0001646F000E656F000EDE
:10AB1000666F000E676F0FEC6DF079C070F0D00EAD
:10AB20000001702770516025756F000E6121766FEE
:10AB3000000E6221776F000E6321786F6CC0D9FF21
:10AB40006DC0DAFFDF50796F6C4B6D2B79518DEC56
:10AB500071F0D8B0CFD700017451D8B41AD075C0F5
:10AB600070F076C071F077C072F078C073F0701F2B
:10AB7000711F721F731F702B000E712372237323BA
:10AB800070C06CF071C06DF072C06EF073C06FF089
:10AB9000120075C06CF076C06DF077C06EF078C0B2
:10ABA0006FF012000101C2B31200C2B171D0000EE9
:10ABB000A66F000EA56FA65124E1080EA55DD8B0C2
:10ABC00020D0300E0001EB6F040EEC6FD890010125
:10ABD000A535D96EA635DA6ED890D936DA360001A9
:10ABE000EB51D926EC51DA22DE5002013A27DE5031
:10ABF0003B23DE503C23DD503D230101A54BA62B1A
:10AC0000DAD7020197510001606F616B626B636B71
:10AC10003AC264F03BC265F03CC266F03DC267F0E8
:10AC20000FEC6DF060C06CF061C06DF062C06EF052
:10AC300063C06FF0000E6AEC4AF06CC0CCF06DC0DF
:10AC4000CDF06EC0CEF06FC0CFF0C00E0001C86F67
:10AC5000E10EC96F640ECA6F4E0ECB6F28EC3BF04D
:10AC6000C8C0E1F0C9C0E2F0CAC0E3F0CBC0E4F074
:10AC7000A0EC5CF0E1C065F2E2C066F2000E0201F9
:10AC80003A6F000E3B6F000E3C6F000E3D6F1200DE
:10AC9000000E0201666F000E656F1200759804BE0B
:10ACA0003AD0010162AF0CD0020E2C6ED451D8B450
:10ACB00027EC65F0000E0101D66F000ED76F120071
:10ACC00020EE01F01950D9261A50DA22080EDF6E54
:10ACD00020EE02F01950D9261A50DA22300EDE6E1C
:10ACE000010EDD6E19C0D9FF1AC0DAFF0C0EDF6E3F
:10ACF00019C0D9FF1AC0DAFF000EDB8E07C0D9FFDA
:10AD000008C0DAFF040EDF6E07C0D9FF08C0DAFF03
:10AD1000000EDB8E1200010130AF11D0010E2C6E3F
:10AD2000D551D8B427EC65F0000E0101D66F000EA6
:10AD3000D76FD851D8A41200C7EC60F01200020EF1
:10AD40002C6E20EE01F01950D9261A50DA22080E86
:10AD5000DF6E20EE02F01950D9261A50DA22300E9A
:10AD6000DE6E010EDD6E19C0D9FF1AC0DAFF040EC7
:10AD7000DF6E19C0D9FF1AC0DAFF000EDB8E000E9D
:10AD80000101D66F000ED76FD851D8A41200C7ECBE
:10AD900060F012000001606F0E01AC9BA49B9C9BB5
:10ADA000949B9B91AB91A39148D00E01AC8BA48B4B
:10ADB0009C8B948B9B81AB8112000E01A48B9C8B8E
:10ADC00012000E01AC8BA48B948B9B81A38112008B
:10ADD0000E01AC8BA48B9C8B948BA38112000E0173
:10ADE000A48B9C8BAB81A38112000E01AC8B9C8B3E
:10ADF000948BAB81A38112000E01AC8B9C8B948B46
:10AE00009B81AB81A38112000E01AC8BA48B9C8B28
:10AE100012000E01AC8BA48B9C8B948B9B81AB811D
:10AE2000A38112000E01AC8BA48B9C8B948BAB8105
:10AE3000A38112000E01A381120000016051000ADB
:10AE4000D8B4B3D7010AD8B4B8D7030AD8B4B9D79D
:10AE5000010AD8B4BDD7070AD8B4C1D7010AD8B4FB
:10AE6000C4D7030AD8B4C8D7010AD8B4CDD70F0ABB
:10AE7000D8B4CFD7010AD8B4D5D7030AD8A41200C2
:10AE8000D9D70001606F0E01AB93A3939B9393936B
:10AE90009D9FAD9FA59F48D00E01AB83A3839B834D
:10AEA00093839D8FAD8F12000E01A3839B831200AD
:10AEB0000E01AB83A38393839D8FA58F12000E0198
:10AEC000AB83A3839B839383A58F12000E01A3837F
:10AED0009B83AD8FA58F12000E01AB839B83938361
:10AEE000AD8FA58F12000E01AB839B8393839D8F43
:10AEF000AD8FA58F12000E01AB83A3839B8312003D
:10AF00000E01AB83A3839B8393839D8FAD8FA58F0E
:10AF100012000E01AB83A3839B839383AD8FA58F18
:10AF200012000E01A58F120000016051000AD8B472
:10AF3000B3D7010AD8B4B8D7030AD8B4B9D7010A2D
:10AF4000D8B4BDD7070AD8B4C1D7010AD8B4C4D77A
:10AF5000030AD8B4C8D7010AD8B4CDD70F0AD8B4D9
:10AF6000CFD7010AD8B4D5D7030AD8A41200D9D7AD
:10AF70000001606F0E01A6959E9596958E95969709
:10AF8000A6979E9748D00E01A6859E8596858E85AC
:10AF90009687A68712000E019E85968512000E01E7
:10AFA000A6859E858E8596879E8712000E01A685B2
:10AFB0009E8596858E859E8712000E019E859685BC
:10AFC000A6879E8712000E01A68596858E85A68788
:10AFD0009E8712000E01A68596858E859687A68788
:10AFE0009E8712000E01A6859E85968512000E0191
:10AFF000A6859E8596858E859687A6879E87120054
:10B000000E01A6859E8596858E85A6879E87120051
:10B010000E019E87120000016051000AD8B4B3D718
:10B02000010AD8B4B8D7030AD8B4B9D7010AD8B43A
:10B03000BDD7070AD8B4C1D7010AD8B4C4D7030A08
:10B04000D8B4C8D7010AD8B4CDD70F0AD8B4CFD74F
:10B05000010AD8B4D5D7030AD8A41200D9D7000E54
:10B060000001686F000E0301526F25902592259410
:10B07000259A2796279027920101C29B0201AC9145
:10B08000AC93000EB66F000EB56F000EB86F000ED9
:10B09000B76F000EBA6F000EB96F000EAD6F000EE5
:10B0A000AE6F000EAF6F000EB06F000EB16F000EEE
:10B0B000B26F000EB36F000EB46F000E0101CB6FC4
:10B0C000000E0201666F000E656F279C2784000E3C
:10B0D0000001606F050E616F000E636F000E626FFE
:10B0E000020E656F000E646F29EC70F0000E000117
:10B0F000606F070E616F000E636F000E626F020ECD
:10B10000656F000E646F29EC70F0000E0101BF6FD7
:10B11000000E02012E6F000E2F6F000E306F000E1A
:10B12000316F000E0101A46F000EA36F000E02012B
:10B130003E6F000E3F6F000E406F000E416F010129
:10B14000CD91CD93CD9512000101C495C491C493C6
:10B1500086A403D08F9EC4851200800E03013C6537
:10B160000ED00101C48102015F516011D8A402D048
:10B170008F9E08D05F07D8A060078F8E03D08F8E78
:10B180000101C4830101C8B11200870EC16101D061
:10B19000CD817A0EC1611200010EFFEC4FF00E015D
:10B1A000E887E883E8850101CD81CD93CD95CFEC8B
:10B1B00053F0000E0101A66F000EA56FA65135E1F8
:10B1C0000A0EA55DD8B031D0CDA102D0010E01D0BC
:10B1D000000EFF0A0001626F0101CD5100016219EA
:10B1E000FE0B62190101CD6FCDA302D0010E01D07B
:10B1F000000EFF0A0001626F62470101CD5100019C
:10B200006219FD0B62190101CD6FF5EC70F0000EB3
:10B210000101A46F000EA36FA45104E1640EA35DAD
:10B22000D8A0FAD7A54BA62BC9D756EC5EF01200D2
:10B23000F00E0001AB6F7B0EAC6F120EAD6F490EBE
:10B24000AE6F5BC16CF05CC16DF05DC16EF05EC154
:10B250006FF0010E6AEC4AF06CC07EF06DC07FF0BA
:10B260006EC080F06FC081F0CDEC6EF07EC0AFF0AC
:10B270007FC0B0F080C0B1F081C0B2F092EC50F06D
:10B280000001D8A030D056C160F057C161F0000E67
:10B29000636F640E626F66EC6DF000016051DCEC70
:10B2A0005AF058C160F059C161F0000E0001636F9F
:10B2B0000A0E626F66EC6DF000016051B76FB75116
:10B2C000FAEC59F00001B7510A0DF35000080101E2
:10B2D00058250001B76FB75189EC59F001015A5157
:10B2E0006BEC5AF012D00A0E0001B76FB7516BEC3D
:10B2F0005AF00001B751FAEC59F00001B75189EC4E
:10B3000059F00001B751DCEC5AF00E018F8D908599
:10B3100012000001606F0E01949D9C9DA49DAC9D48
:10B32000AC9F9C9FA49F45D00E01948D9C8DA48DB5
:10B33000AC8DAC8F9C8F12000E019C8DA48D1200E1
:10B340000E01948D9C8DAC8DAC8FA48F12000E01DC
:10B35000948D9C8DA48DAC8DA48F12000E019C8DBC
:10B36000A48D9C8FA48F12000E01948DA48DAC8DA2
:10B370009C8FA48F12000E01948DA48DAC8DAC8F88
:10B380009C8FA48F12000E01948D9C8DA48D1200B1
:10B390000E01948D9C8DA48DAC8DAC8F9C8FA48F51
:10B3A00012000E01948D9C8DA48DAC8D9C8FA48F6A
:10B3B000120000016051000AD8B4B6D7010AD8B40F
:10B3C000BBD7030AD8B4BCD7010AD8B4C0D7070A80
:10B3D000D8B4C4D7010AD8B4C7D7030AD8B4CBD7D6
:10B3E000010AD8B4D0D70F0AD8B4D2D7010AD8A44A
:10B3F0001200D7D70001606F0E018F9F979F9F9F0C
:10B40000A79FA79D979D9F9D45D00E018F8F978FDA
:10B410009F8FA78FA78D978D12000E01978F9F8FFB
:10B4200012000E018F8F978FA78FA78D9F8D12000F
:10B430000E018F8F978F9F8FA78F9F8D12000E0108
:10B44000978F9F8F978D9F8D12000E018F8F9F8FEB
:10B45000A78F978D9F8D12000E018F8F9F8FA78FC3
:10B46000A78D978D9F8D12000E018F8F978F9F8FC5
:10B4700012000E018F8F978F9F8FA78FA78D978DAB
:10B480009F8D12000E018F8F978F9F8FA78F978DA3
:10B490009F8D120000016051000AD8B4B6D7010A8E
:10B4A000D8B4BBD7030AD8B4BCD7010AD8B4C0D724
:10B4B000070AD8B4C4D7010AD8B4C7D7030AD8B486
:10B4C000CBD7010AD8B4D0D70F0AD8B4D2D7010A43
:10B4D000D8A41200D7D70001606F0E0195919D91FD
:10B4E000A591AD91A9979997A19745D00E01958106
:10B4F0009D81A581AD81A987998712000E019D814B
:10B50000A58112000E0195819D81AD81A987A1873A
:10B5100012000E0195819D81A581AD81A187120048
:10B520000E019D81A5819987A18712000E01958149
:10B53000A581AD819987A18712000E019581A58112
:10B54000AD81A9879987A18712000E0195819D8100
:10B55000A58112000E0195819D81A581AD81A987EC
:10B560009987A18712000E0195819D81A581AD81EA
:10B570009987A187120000016051000AD8B4B6D79C
:10B58000010AD8B4BBD7030AD8B4BCD7010AD8B4CF
:10B59000C0D7070AD8B4C4D7010AD8B4C7D7030A9A
:10B5A000D8B4CBD7010AD8B4D0D70F0AD8B4D2D7E1
:10B5B000010AD8A41200D7D70001606F0E01909B3A
:10B5C000989BA09BA89BA8959895A09545D00E0107
:10B5D000908B988BA08BA88BA885988512000E0164
:10B5E000988BA08B12000E01908B988BA88BA8854E
:10B5F000A08512000E01908B988BA08BA88BA08544
:10B6000012000E01988BA08B9885A08512000E0168
:10B61000908BA08BA88B9885A08512000E01908B33
:10B62000A08BA88BA8859885A08512000E01908B11
:10B63000988BA08B12000E01908B988BA08BA88BFF
:10B64000A8859885A08512000E01908B988BA08B01
:10B65000A88B9885A085120000016051000AD8B41B
:10B66000B6D7010AD8B4BBD7030AD8B4BCD7010AED
:10B67000D8B4C0D7070AD8B4C4D7010AD8B4C7D73A
:10B68000030AD8B4CBD7010AD8B4D0D70F0AD8B49C
:10B69000D2D7010AD8A41200D7D70001606F0E01DB
:10B6A000A69B9E9B969B8E9B9D9DAD9DA59D45D0EB
:10B6B0000E01A68B9E8B968B8E8B9D8DAD8D120071
:10B6C0000E019E8B968B12000E01A68B9E8B8E8B8D
:10B6D0009D8DA58D12000E01A68B9E8B968B8E8B59
:10B6E000A58D12000E019E8B968BAD8DA58D12003F
:10B6F0000E01A68B968B8E8BAD8DA58D12000E0143
:10B70000A68B968B8E8B9D8DAD8DA58D12000E0117
:10B71000A68B9E8B968B12000E01A68B9E8B968B12
:10B720008E8B9D8DAD8DA58D12000E01A68B9E8BEF
:10B73000968B8E8BAD8DA58D120000016051000A95
:10B74000D8B4B6D7010AD8B4BBD7030AD8B4BCD78B
:10B75000010AD8B4C0D7070AD8B4C4D7010AD8B4EC
:10B76000C7D7030AD8B4CBD7010AD8B4D0D70F0AA9
:10B77000D8B4D2D7010AD8A41200D7D70001606F7D
:10B780000E01A69D9E9D969D8E9D969FA69F9E9F17
:10B7900045D00E01A68D9E8D968D8E8D968FA68F8F
:10B7A00012000E019E8D968D12000E01A68D9E8DAB
:10B7B0008E8D968F9E8F12000E01A68D9E8D968D7A
:10B7C0008E8D9E8F12000E019E8D968DA68F9E8F60
:10B7D00012000E01A68D968D8E8DA68F9E8F120063
:10B7E0000E01A68D968D8E8D968FA68F9E8F120040
:10B7F0000E01A68D9E8D968D12000E01A68D9E8D3A
:10B80000968D8E8D968FA68F9E8F12000E01A68D1F
:10B810009E8D968D8E8DA68F9E8F12000001605199
:10B82000000AD8B4B6D7010AD8B4BBD7030AD8B433
:10B83000BCD7010AD8B4C0D7070AD8B4C4D7010A04
:10B84000D8B4C7D7030AD8B4CBD7010AD8B4D0D755
:10B850000F0AD8B4D2D7010AD8A41200D7D7000152
:10B86000606F0E01AA91A2919A9192919A93AA93D4
:10B87000A29345D00E01AA81A2819A8192819A83D6
:10B88000AA8312000E01A2819A8112000E01AA81E0
:10B89000A28192819A83A28312000E01AA81A281C1
:10B8A0009A819281A28312000E01A2819A81AA83B9
:10B8B000A28312000E01AA819A819281AA83A28397
:10B8C00012000E01AA819A8192819A83AA83A2838F
:10B8D00012000E01AA81A2819A8112000E01AA8192
:10B8E000A2819A8192819A83AA83A28312000E0177
:10B8F000AA81A2819A819281AA83A2831200000167
:10B900006051000AD8B4B6D7010AD8B4BBD7030A2D
:10B91000D8B4BCD7010AD8B4C0D7070AD8B4C4D7A2
:10B92000010AD8B4C7D7030AD8B4CBD7010AD8B410
:10B93000D0D70F0AD8B4D2D7010AD8A41200D7D7CB
:10B940000001E335E435EA6FEA51D8A409D0000ECE
:10B95000E16F000EE26F000EE36F000EE46F120065
:10B96000E1C0E5F0E2C0E6F0E3C0E7F0E4C0E8F0F3
:10B97000200E05D0D890E833E733E633E533E82EE0
:10B98000F9D7E551E96FE38FFF0EE117FF0EE217DC
:10B99000FF0EE317000EE417960EEA5FEAAF16D02B
:10B9A000EA51800A970FD8B009D0000EE16F000E5F
:10B9B000E26F000EE36F000EE46F1200D890E433E4
:10B9C000E333E233E133EA3FF9D715D01F0EEA65DE
:10B9D0000FD0000EE16F000EE26F000EE36F000E5D
:10B9E000E46F1200D890E137E237E337E437EA0733
:10B9F000EA51D8A4F7D7E951D8B408D0E41FE31F1F
:10BA0000E21FE16D000EE223E323E423E1C0E1F055
:10BA1000E2C0E2F0E3C0E3F0E4C0E4F01200048E20
:10BA2000000E2F6E0E0E306E000E326E000E316E56
:10BA3000000E346E020E336EB6EC70F0000E2F6EF8
:10BA4000010E306E000E326E000E316E000E346E3E
:10BA5000300E336EB6EC70F0758C000E436E020E35
:10BA6000436401D016D04350010DA00EF324D96ECB
:10BA7000010EF420DA6E000EDF6E4350010D540EFD
:10BA8000F324D96E020EF420DA6E000EDF6E432A24
:10BA9000E6D7E80E2F6E020E306E000E326E000EEC
:10BAA000316E000E346E020E336EB6EC70F0759C83
:10BAB000080E076E010E086E000E1B6E010E1C6E46
:10BAC0001BC019F01CC01AF032C1DFF10101DF51B7
:10BAD000D8A403D0100E2D6E1200000E3C6E010E85
:10BAE0003B6EDF0E3D6E010E3E6E000E406E010E8F
:10BAF0003F6EFDEC69F0200E2D6E120003D00001A8
:10BB0000664B672B66C0D9FF67C0DAFF200EDE18D0
:10BB1000D8B4F5D766C0D9FF67C0DAFF090EDE18C2
:10BB2000D8B4EDD7000E00016C6F000E6B6F000EE5
:10BB30006A6F66C0D9FF67C0DAFF2D0EDE18D8A481
:10BB400002D06A2B26D066C0D9FF67C0DAFF2B0E61
:10BB5000DE18D8A420D01DD06BC060F06CC061F09E
:10BB6000000E0001636F0A0E626F31EC71F066C067
:10BB7000D9FF67C0DAFFDF500001686F696B605161
:10BB8000682761516923D00E68256B6FFF0E69210C
:10BB90006C6F664B672B66C0D9FF67C0DAFFDF505A
:10BBA0008DEC71F0D8B0D8D700016A51D8B40DD05F
:10BBB0006BC068F06CC069F0681F691F684B692B27
:10BBC00068C066F069C067F012006BC066F06CC0B8
:10BBD00067F0120001013039E832030B0009D8A4E4
:10BBE000120042D0048E080E2D6E1200ACEC4DF007
:10BBF00012000FEC5DF01200DF0E016E010E026EFE
:10BC00000480010E056E048E1200F3EC63F0120046
:10BC1000D6EC3DF0120001013451010DE80EF32481
:10BC2000016E020EF420026E0480010E056E048E79
:10BC30001200048E3451010DE80EF324D96E020E69
:10BC4000F420DA6E32C1DFFF1200000E3C6E020EED
:10BC50003B6E000E3D6E000E3E6E000E406E000EFE
:10BC60003F6EFDEC69F0120001013151000AD8B4B9
:10BC7000CCD7010AD8B4CCD7020AD8B4C9D7060A9F
:10BC8000D8B4B0D7030AD8B4B1D7010AD8B4DDD735
:10BC90000F0AD8B4B1D7010AD8B4ABD7030AD8B4C5
:10BCA000BAD7010AD8B4C5D7070A1200010EFFECB3
:10BCB0004FF00101C4A31AD00E01E895E893E8976C
:10BCC00005EC69F00E01E885E883E8878F9E86B66B
:10BCD000FED7000E0101C66F0F0EC66501D006D05B
:10BCE000C80ECFEC71F00101C62BF6D7C4A112002B
:10BCF000010EFFEC4FF00E01E885E883E8978F9E78
:10BD000005EC69F0000E0101C66F130EC66501D087
:10BD100016D0000EA46F000EA36FA45104E1140E00
:10BD2000A35DD8A0FAD7C62BF0D7000EA46F000EE3
:10BD3000A36FA45104E1050EA35DD8A0FAD786B67F
:10BD40000BD0F3D7000EA46F000EA36FA45104E133
:10BD5000030EA35DD8A0FAD786B6F4D7000EC66F3F
:10BD6000040EC66501D01200000EA46F000EA36F72
:10BD7000A45104E1050EA35DD8A0FAD7C62BF0D7D5
:10BD8000010E0001F26FA5EC62F00001F06F000EF1
:10BD9000206EC00E0301006F270E016F090E026FA7
:10BDA000000E036F010E0001F26F0C0EF26501D060
:10BDB00012D0F251040D000EF324D96E030EF420BC
:10BDC000DA6E600EDE6EEA0EDE6E000EDE6E000EC5
:10BDD000DD6EF22BEAD7F051D8B41200010EF26FEB
:10BDE00033D0F25161EC60F003010051C55D0151A7
:10BDF000C6590251C7590351C859D8B023D0000EB3
:10BE00000001F16F0C0EF16501D01AD0F151040D53
:10BE1000C50EF324D96E030EF420DA6EF151040D31
:10BE2000000EF324E16E030EF420E26EDECFE6FF97
:10BE3000DECFE6FFDECFE6FFDECFE6FFF12BE2D777
:10BE4000F2C020F00001F22BF251F05DD8A01200F8
:10BE5000C8D7080E2F6E065011E1080E055CD8B049
:10BE60000DD005C02FF00101DE51D8A402D0010E83
:10BE700004D0DE05D8A402D0020EDE6F2F50055E7E
:10BE8000000E065A20EE01F00750D9260850DA229B
:10BE90002FC0DFFF380E0201736F010E746F04A014
:10BEA0001DD03CD001C0F6FF02C0F7FF000EF86EB7
:10BEB00073C2D9FF74C2DAFF0D0EF76403D0080015
:10BEC000F55005D0F6CFE1FFF7CFE2FFE750DF6E88
:10BED000014A022A0201734B742B2F062F50D8B44B
:10BEE0001200E0D701C0F6FF02C0F7FF000EF86EA7
:10BEF00073C2D9FF74C2DAFF0D0EF76403D00800D5
:10BF0000F55005D0F6CFE1FFF7CFE2FFE750DF6E47
:10BF1000014A022A0201734B742B2F062F50D8B40A
:10BF20001200E0D7000E0001AB6F5F0EAC6F6A0E1F
:10BF3000AD6F470EAE6F5BC16CF05CC16DF05DC163
:10BF40006EF05EC16FF0010E6AEC4AF06CC07EF0DC
:10BF50006DC07FF06EC080F06FC081F0CDEC6EF0F0
:10BF60007EC0AFF07FC0B0F080C0B1F081C0B2F051
:10BF700092EC50F00001D8A02CD056C160F057C10F
:10BF800061F0000E636F640E626F66EC6DF000018D
:10BF90006051CAEC56F058C160F059C161F0000E12
:10BFA0000001636F0A0E626F66EC6DF00001605174
:10BFB000B76FB751B8EC57F00001B7510A0DF35005
:10BFC0000008010158250001B76FB75141EC57F047
:10BFD0000ED00A0E0001B76FB751B8EC57F0000150
:10BFE000B75141EC57F00001B751CAEC56F00E01C1
:10BFF00093811200000E0001696F67AF0AD0671FBE
:10C00000661F651F646D000E652366236723010E9E
:10C01000696F63AF0AD0631F621F611F606D000EFE
:10C02000612362236323010E691B000E6A6F000EF9
:10C030006B6F000E6C6F000E6D6F645165116611B1
:10C040006711D8B42AD0010E686F06D0D890643733
:10C05000653766376737682B67AFF8D7D8906A3788
:10C060006B376C376D376451605D6551615966514E
:10C07000625967516359D8A009D06451605F655116
:10C08000615B6651625B6751635B6A81D89067331D
:10C09000663365336433682FE1D76951D8B408D06B
:10C0A0006D1F6C1F6B1F6A6D000E6B236C236D235D
:10C0B0006AC060F06BC061F06CC062F06DC063F08C
:10C0C00012000001EB6F0001EB07000E9B6F800E6A
:10C0D0009C6FFF0E9D6F490E9E6F000E826F000ECB
:10C0E000836F500E846F420E856FEB516C6F6D6BDA
:10C0F0006E6B6F6B000E6AEC4AF06CC07EF06DC028
:10C100007FF06EC080F06FC081F0FFEC34F07EC035
:10C1100097F07FC098F080C099F081C09AF0A8ECA9
:10C1200036F097C0E1F098C0E2F099C0E3F09AC011
:10C13000E4F0A0EC5CF0E1C011F0E2C012F0E3C06A
:10C1400013F0E4C014F011C062F012C063F013C029
:10C1500064F014C065F0000E0001676F340E666F66
:10C16000750E686F030E696F9CEC6BF0C50E0001D5
:10C17000606F030E616F750E626F030E636F000ECA
:10C18000656F340E646F6CEC6BF0010E12000101F0
:10C19000D751D8A41200010ED76FD651D8A41200DF
:10C1A000010ED66F020E2C18D8A415D020EE01F087
:10C1B0000750D9260850DA22000EDF6E07C0D9FFDB
:10C1C00008C0DAFF480EDF6E07C0D9FF08C0DAFFEB
:10C1D000000EDB8E12002C04D8A41200000EDA6FC1
:10C1E00020EE01F01B50D9261C50DA22080EDF6E1B
:10C1F00020EE02F01B50D9261C50DA22300EDE6EE3
:10C20000010EDD6E1BC0D9FF1CC0DAFF040EDF6E0D
:10C210001BC0D9FF1CC0DAFF000EDB8E010EDA6FE7
:10C2200020EE01F01950D9261A50DA22080EDF6EDE
:10C2300020EE02F01950D9261A50DA22300EDE6EA6
:10C24000010EDD6E19C0D9FF1AC0DAFF800EDF6E55
:10C2500012000001606F48D00E01AA81A68DA68B46
:10C26000A685AB83AC8B95818F8F948D908B1200BC
:10C270000E01A2819E8D9E8B9E85A383A48B9D81A2
:10C28000978F9C8D988B12000E019A81968D968BBC
:10C2900096859B839C8BA5819F8FA48DA08B12007C
:10C2A0000E0192818E8D8E8B8E859383948BAD81C2
:10C2B000A78FAC8DA88B12000E019A83968F9D8D4F
:10C2C00096879D8F9B81A987A78DAC8FA88512002B
:10C2D0000E01AA83A68FAD8DA687AD8FAB819987FE
:10C2E000978D9C8F9885120000016051000AD8B488
:10C2F000B3D7010AD8B4BCD7030AD8B4C5D7010A4A
:10C30000D8B4CED7070AD8B4D7D7010AD8A4120018
:10C31000DFD707C0D9FF08C0DAFF000EDFBC010E6F
:10C32000306E040E0718076E0850086E080E2D18A0
:10C33000D8A40BD0010132517F0B746E7450D8B465
:10C3400002D0100E01D0040E2D6E2C04D8A43BD0C8
:10C3500020EE02F00750D9260850DA22380EDE6EA1
:10C36000010EDD6E29EC5FF0020E0101DE19D8A48A
:10C370000DD007C0D9FF08C0DAFF040EDF6E07C07A
:10C38000D9FF08C0DAFF000EDB8E12003050D8A4AF
:10C390000DD007C0D9FF08C0DAFF480EDF6E07C016
:10C3A000D9FF08C0DAFF000EDB8E120007C0D9FFEC
:10C3B00008C0DAFF080EDF6E07C0D9FF08C0DAFF39
:10C3C000000EDB8E1200010162BF629F000E2C6E18
:10C3D000120055D022EEB5F0DECF67F0DDCF68F069
:10C3E0000001D89067376837D89067376837D8909A
:10C3F0006737683767C060F068C061F09DC262F05F
:10C400009EC263F066EC6DF000016051B3EC51F038
:10C410001200000E0001636F640E626F8AC260F04A
:10C420008BC261F066EC6DF00001D8906037613727
:10C43000D89060376137D8906037613760C069F055
:10C4400061C06AF0000E636F640E626F9DC260F09F
:10C450009EC261F066EC6DF060C06BF061C06CF084
:10C4600069C060F06AC061F06BC062F06CC063F0DC
:10C4700066EC6DF000016051B3EC51F01200020166
:10C480009C51010AD8B4A6D7030AD8A41200C1D778
:10C49000000E0001626F000E616F0FD0B5C261F037
:10C4A000B6C262F015D08AC261F08BC262F010D0C1
:10C4B00021C061F00001626B0BD00201A051010AA2
:10C4C000D8B4ECD7030AD8B4EED7010AD8B4F0D761
:10C4D0000201A2510001615D0201A35100016259F4
:10C4E000D8B006D00A0E0101FF6F0E01E8871200D6
:10C4F0000201A105D8A403D00E01E8971200020E94
:10C500000201A119D8A41BD00101FF51D8B417D042
:10C510000E01E8A702D0010E01D0000EFF0A0001B3
:10C52000606F6047604760470E01E8510001601985
:10C53000F70B60190E01E86F0101FF071200000EF2
:10C540000101FF6F0E01E88712003DEC52F06CC054
:10C55000ECF06DC0EDF06EC0EEF06FC0EFF0000ECD
:10C56000116EF00E126E1F0E136E000E146E11502F
:10C570000001EC190CE11250ED1909E11350EE190C
:10C5800006E11450EF19D8A402D0000E1200115089
:10C59000EC5F1250ED5B1350EE5B1450EF5B000E3E
:10C5A000CC6F000ECD6F500ECE6F420ECF6FECC031
:10C5B0006CF0EDC06DF0EEC06EF0EFC06FF0000EED
:10C5C0006AEC4AF06CC0C8F06DC0C9F06EC0CAF029
:10C5D0006FC0CBF028EC3BF0C8C0E1F0C9C0E2F07E
:10C5E000CAC0E3F0CBC0E4F0A0EC5CF00001E15184
:10C5F000EB6FEB511200000E0001706F14EC4BF06A
:10C600006CC032F26DC033F26EC034F26FC035F2DE
:10C61000000E116E200E126E000E136E000E146EC0
:10C6200031D011C062F012C063F013C064F014C0C6
:10C6300065F0000E0001676F100E666F000E686FE8
:10C64000050E696F9CEC6BF000C5E8FF240AD8A4C6
:10C6500011D001C5E8FF360AD8A40CD002C5E8FF06
:10C66000460AD8A407D003C5E8FF2C0AD8A402D0F4
:10C670000001702B000E1126020E1222000E132252
:10C68000000E142202013251115C33511258345100
:10C69000135835511458D8A0C4D700017051120056
:10C6A000010130511F0BE806D8A412003039E832DE
:10C6B000030BE806D8A412003451D8B434D03405A2
:10C6C000D8A4120030D0D90E016E020E026E000EF8
:10C6D000066E080E056E0480048E1200D90E016EDF
:10C6E000020E026E048E120036C163F137C164F18E
:10C6F000E10E5F6F020E606F000E656F000E666FD9
:10C70000000E676F628F1200E10E016E020E026E64
:10C71000000E066E070E056EC10E046E120032C1C9
:10C72000D0F1048E12003151000AD8B4CCD7010ADE
:10C73000D8B4D4D7210AD8B4D7D7010AD8B4E4D70B
:10C74000030AD8A41200EBD725BA1200000E01018B
:10C750005B6F000E5C6F000E5D6F000E5E6FBDECD8
:10C7600049F018EC59F0000E0D6E000E0E6E000E22
:10C770000F6E000E106E000E01015B6F000E5C6FFD
:10C78000000E5D6F000E5E6FBDEC49F092EC5FF045
:10C790000DC078F10EC079F10FC07AF110C07BF1B5
:10C7A0000DC074F10EC075F10FC076F110C077F1B5
:10C7B00078C160F079C161F07AC162F07BC163F049
:10C7C00074C164F075C165F076C166F077C167F039
:10C7D000010E0001686FC3EC69F027B21200010E70
:10C7E000FFEC4FF01200000E0101386F000E396FA0
:10C7F00033D0048EDD05D8A43AD0388338D0048EE7
:10C8000036D0048E34BF0AD034510F0B2F6E2F5008
:10C81000020D0C0EF324D96E020E09D034510F0B09
:10C820002F6E2F50020D070EF324D96E000EF42048
:10C83000DA6EDECF30F0DDCF31F030C0D9FF31C05D
:10C84000DAFFDFAE14D030C0D9FF31C0DAFFDFA489
:10C850000ED0010E386F0BD030511F0B000AD8B428
:10C86000C8D7010AD8B4CBD7030AD8B4CAD704AE04
:10C870001200380E016E010E026E0480020E056E6B
:10C880001200C60EF66EE40EF76E000EF86E02EEA3
:10C89000EAF010EE0EF00900F5CFEEFFE550E150A2
:10C8A000FAE11A0EF66EE50EF76E000EF86E01EE66
:10C8B000FCF010EE04F00900F5CFEEFFE550E1507A
:10C8C000FAE109EE00F0EE0EEE6AE806FDE104EE94
:10C8D00000F0F80EEE6AE806FDE103EE00F0F90E56
:10C8E000EE6AE806FDE102EE00F0EA0EEE6AE80606
:10C8F000FDE101EE40F0A00EEE6AE806FDE1000168
:10C90000FC6BFB6BFA6B00EE01F02E0EEE6AE80694
:10C91000FDE15D905D920001D0EF0AF0000E2B6EFC
:10C920000101AD51AE11D8B406D0ADC1D9FFAEC131
:10C93000DAFFDFBE3ED020EE01F0AD51D926AE5178
:10C94000DA2200016D51DE5CD8B00AD0010120EE80
:10C9500001F0AD51D926AE51DA22DF5000016D6FE2
:10C96000000E2B6E13D02B50010D6E0EF324D96EDA
:10C97000090EF420DA6E2B50010DF3506B25E16E99
:10C98000F4506C21E26EDFCFE7FF2B2A6D512B5C58
:10C99000D8A0E9D7000E606F6E0E616F090E626F4E
:10C9A000400E636F020E4CEC53F060C0ADF161C0FD
:10C9B000AEF12B5012002D0E0101D96F2EC049F09F
:10C9C000FD0E4916D8A43BD02EC049F0D89049326C
:10C9D0003F0E49164950040D000EF3241B6E010E44
:10C9E000F4201C6E1BC019F01CC01AF0040E19189C
:10C9F000196E1A501A6E1BC0D9FF1CC0DAFFDF3047
:10CA0000E8320F0B0D0AD8A417D0300E2F6E010E8E
:10CA1000306E20EE02F01B50D9261C50DA22DECFF9
:10CA200031F0DDCF32F0000E346E080E336E87EC3D
:10CA30006CF027EC67F012002AEC6CF012002E501C
:10CA4000FD0B040AD8A4120089EC61F01200000E5C
:10CA50000101D56F000ED46F020E2C18D8A41FD080
:10CA600020EE01F01950D9261A50DA22080EDF6E96
:10CA700020EE02F01950D9261A50DA22380EDE6E56
:10CA8000010EDD6E19C0D9FF1AC0DAFF480EDF6E45
:10CA900019C0D9FF1AC0DAFF000EDB8E1200055054
:10CAA000365D06503759D8B004D036C105F037C1CD
:10CAB00006F029EC5FF020EE02F00750D92608506E
:10CAC000DA22380EDE6E010EDD6E07C0D9FF08C017
:10CAD000DAFF480EDF6E07C0D9FF08C0DAFF000E8C
:10CAE000DB8E12001DA002D0010E12000201ACA1CB
:10CAF00019D025800101CD8502016F517011D8B484
:10CB00000CD06F07D8A0700725942796010E01015D
:10CB1000AC6F900EAB6F000E1200258427B60FD0BD
:10CB20002498F9D725900101CD95020E0201706F6E
:10CB3000580E6F6F259427962498000E1200460E0B
:10CB400002019519D8A402D0010E1200500E9519B9
:10CB5000D8A410D0B65104E1150EB55DD8A002D00E
:10CB6000010E120024A803D02498010E120024986C
:10CB7000000E1200000E1200346E000E356E010E13
:10CB8000366E2F50306E316AD89030363136345090
:10CB9000326E336AD89032363336D89032363336E6
:10CBA0003050322631503322D89032363336D89036
:10CBB00032363336325035263350362235C0D9FF1F
:10CBC00036C0DAFFDF9E2F50D8A407D03450020DB4
:10CBD0000C0EF324D96E020E06D03450020D070E4F
:10CBE000F324D96E000EF420DA6E35C0DEFF36C0B5
:10CBF000DDFF35C0D9FF36C0DAFFDF9C20EE04F040
:10CC00003550D9263650DA22DF8C12003CD0020192
:10CC1000B5516BEC6EF01200100E02018A5D270E0A
:10CC20008B59D8A016D08AC260F08BC261F0000E7A
:10CC30000001636F640E626F66EC6DF060C074F0AB
:10CC400061C075F074C072F075C073F0ADEC6EF039
:10CC500012008AC260F08BC261F0000E0001636FA7
:10CC60000A0E626F66EC6DF060C074F061C075F022
:10CC700074C072F075C073F0ADEC6EF0120021500C
:10CC80008CEC6EF0120002019F51010AD8B4BFD79C
:10CC9000030AD8B4C1D7010AD8A41200F0D7C0EC57
:10CCA0005EF02050D8B4120020508CEC6EF000C31F
:10CCB0005BF101C35CF102C35DF103C35EF1BDEC46
:10CCC00049F018EC59F0000E01015B6F000E5C6F2B
:10CCD000000E5D6F000E5E6FBDEC49F092EC5FF0F0
:10CCE000000E0101786F000E796F000E7A6F000E52
:10CCF0007B6F000E746F000E756F000E766F000E66
:10CD0000776F78C160F079C161F07AC162F07BC160
:10CD100063F074C164F075C165F076C166F077C1E7
:10CD200067F0010E0001686FC3EC69F0120088A67D
:10CD300086A602D0190E120088AE88BC02D0220E40
:10CD4000120088AE24B008D0190E17EC72F088BE1D
:10CD500003D02480150E120088AC24B208D0190E1E
:10CD600017EC72F088BC03D02482160E120088A63D
:10CD700024B408D0FA0E17EC72F088B603D02484DD
:10CD8000170E120086B624B608D0190E17EC72F0F2
:10CD900086A603D02486180E120088BE24A001D0D7
:10CDA000249088BC24A201D0249288B624A401D067
:10CDB000249486A624A601D02496000E1200000E0C
:10CDC0000001636F000E646F000E656F000E666FEA
:10CDD0007DEC72F0DEEC71F088EC72F0000E000178
:10CDE000636F200E646F000E656F000E666F6651F4
:10CDF0002BE16329EF0E64591F0E6559D8B024D07A
:10CE00008A94200E2AEC72F0000165512AEC72F02F
:10CE1000000164512AEC72F0000163512AEC72F0B7
:10CE20008A841E0ECFEC71F07DEC72F0DEEC71F0B6
:10CE300088EC72F0000E00016327100E6423000ED0
:10CE40006523000E6623D3D7DEEC71F01200000ECE
:10CE50000101DE6F000ED86F000ED56F000ED46F8B
:10CE6000000EDA6F000E2C6E07C0D9FF08C0DAFF83
:10CE70007F0EDF16040E0718076E0850086E07C0F5
:10CE8000D9FF08C0DAFF7F0EDF16040E0718076E01
:10CE90000850086E19C0D9FF1AC0DAFF7F0EDF16DE
:10CEA000000E046E000E066E000E056E000E626F20
:10CEB000000E646F000E636FEAEC5DF0000E3C6ED6
:10CEC000030E3B6E000E3D6E000E3E6E000E406E79
:10CED000000E3F6EFDEC69F04EEC56F012000101C1
:10CEE000C29BCA51D8B428D0CA510001606F616B8F
:10CEF000626B636BFF0E646FFF0E656F000E666FF3
:10CF0000000E676F0FEC6DF00201365100016025D5
:10CF10000201366F3751000161210201376F38512C
:10CF2000000162210201386F3951000163210201C1
:10CF3000396F000E0101CA6FCB51040D300EF3247E
:10CF4000D96E040EF420DA6E36C2DEFF37C2DEFF81
:10CF500038C2DEFF39C2DEFFCB2B080ECB19D8A4B6
:10CF600002D0000ECB6F000ECA6F12000201975163
:10CF7000D8B41200020E0101CC19D8B41200C00EB0
:10CF8000BE6E320E6AEC72F0320E6AEC72F0320E45
:10CF90006AEC72F0320E6AEC72F0320E6AEC72F0E9
:10CFA000320E6AEC72F0320E6AEC72F0320E6AECFB
:10CFB00072F0320E6AEC72F0320E6AEC72F0320EDF
:10CFC0006AEC72F0320E6AEC72F0320E6AEC72F0B9
:10CFD000320E6AEC72F0320E6AEC72F0320E6AECCB
:10CFE00072F0AE0E0F01536FA6900101C285320E92
:10CFF0006AEC72F0120014EC4BF06CC098F16DC04A
:10D0000099F16EC09AF16FC09BF1000E156E200E63
:10D01000166E000E176E000E186E02D03BEC72F00A
:10D020002A50D8B41DD0FAD73BEC72F02A50D8A4BD
:10D0300017D0E1EC70F0000E00016D6F050E6E6F01
:10D04000B5EC6CF0000E1526020E1622000E17220B
:10D05000000E182202D03BEC72F02A50D8A4FBD765
:10D0600001019851155C995116589A5117589B51C6
:10D070001858D8A0D9D771EC70F012006FC0D9FF42
:10D0800070C0DAFF300EDF6E00016F4B702B6FC087
:10D09000D9FF70C0DAFF300EDF6E6F4B702B6FC0A0
:10D0A000D9FF70C0DAFF300EDF6E6F4B702B6FC090
:10D0B000D9FF70C0DAFF000EDF6E6DC071F06DC079
:10D0C00060F06EC061F0000E636F0A0E626F66EC76
:10D0D0006DF060C06DF061C06EF000016D510A0D21
:10D0E000F350715F7151300F6F07D8A070076FC098
:10D0F000D9FF70C0DAFFDF6E6D516E11D8B4120027
:10D10000DCD7000E0001686F000E696F000E6A6FB9
:10D11000000E6B6F6451651166116711D8B42AD087
:10D12000010E6C6F06D0D890643765376637673765
:10D130006C2B67AFF8D7D890683769376A376B3789
:10D140006451605D65516159665162596751635917
:10D15000D8A009D06451605F6551615B6651625B24
:10D160006751635B6881D890673366336533643396
:10D170006C2FE1D768C060F069C061F06AC062F0EE
:10D180006BC063F01200FF0E0101986FEF0E996FF4
:10D190001F0E9A6F000E9B6F000E156E100E166E0E
:10D1A000000E176E000E186E02D03BEC72F02A5083
:10D1B000D8B41DD0FAD73BEC72F02A50D8A417D0BF
:10D1C000E1EC70F0000E00016D6F050E6E6FB5ECB6
:10D1D0006CF0000E1526020E1622000E1722000E0D
:10D1E000182202D03BEC72F02A50D8A4FBD70101E0
:10D1F0009851155C995116589A5117589B511858C7
:10D20000D8A0D9D771EC70F012000E018E698F6929
:10D21000906991699269936994699569966997692A
:10D22000986999699A699B699C699D699E699F69DA
:10D23000A069A169A269A369A469A569A669A7698A
:10D24000A869A969AA69AB69AC69AD69AE69AF693A
:10D25000B069B169B269B369B469B569B669B769EA
:10D26000B869B969BA69BB69BC69BD69BE69BF699A
:10D27000C069C169C269C369C469C569C669C7694A
:10D28000C869C969CA69CB69CC691200000E01017D
:10D29000596F000E586F000E576F000E566F000E3C
:10D2A0005A6F000E5B6F000E5C6F000E5D6F000E1C
:10D2B0005E6F000E8CEC6EF092EC5FF018EC59F0A3
:10D2C000000EB3EC51F0F5EC70F0010E0001606F50
:10D2D000000E616F000E626F000E636F010E646FCF
:10D2E000000E656F000E666F000E676F000E686FB0
:10D2F000C3EC69F00E01E885E883E887E587E589F6
:10D30000E583E5858D928D901200B7EC6DF0C80E27
:10D31000CFEC71F0C80ECFEC71F0C80ECFEC71F00D
:10D32000C80ECFEC71F0000E00016E6F000E6D6F35
:10D33000020E6E5DD8B01200DEEC71F07DEC72F082
:10D34000000E0001696F100E6A6F6DC06BF06EC049
:10D350006CF069516B276A516C236BC061F06CC033
:10D3600062F0636B646B6D516725D96E6E516821F5
:10D37000DA6EDF50656FE0EC6FF0DEEC71F000010B
:10D380006D4B6E2BD5D70E018E9F959D9197A89DC5
:10D3900000016805D8A4120063BF09D0635162116F
:10D3A000611103E16005D8A002D00E018E8F00014B
:10D3B00063BF07D063516211611105E16005D8B008
:10D3C00002D00E01958D000167BF09D0675166112B
:10D3D000651103E16405D8A002D00E019187000118
:10D3E00067BF07D067516611651106E16405D8B0C3
:10D3F00012000E01A88D120012000ED0010EBFEC1B
:10D4000071F01200020EBFEC71F0120009EC6BF02B
:10D41000120050EC63F012003BC041F03CC042F0FF
:10D420004250000AD8B404D07F0AD8A412001AD0FF
:10D430004150010AD8B4EAD7030AD8B41200010A4D
:10D44000D8B4E7D7060AD8B41200770AD8B41200C5
:10D45000010AD8B41200070AD8B4D4D7010AD8A454
:10D460001200CCD74150FF0A1200A60E0F01536FD5
:10D47000D00EBE6EA690320E6AEC72F0320E6AECDE
:10D4800072F0320E6AEC72F0320E6AEC72F0320E0A
:10D490006AEC72F0320E6AEC72F0320E6AEC72F0E4
:10D4A000320E6AEC72F0320E6AEC72F0320E6AECF6
:10D4B00072F0320E6AEC72F0320E6AEC72F0320EDA
:10D4C0006AEC72F0320E6AEC72F0320E6AEC72F0B4
:10D4D000320E6AEC72F01200000E00016B6F000E4B
:10D4E0006A6F20D0DEEC71F07DEC72F000016A51C1
:10D4F0001524616F6B511620626F000E1720636F49
:10D50000000E1820646F6A516625D96E6B51672131
:10D51000DA6EDF50656FE0EC6FF0DEEC71F0000169
:10D520006A4B6B2B68516A5D69516B59D8A0DAD789
:10D530006851152669511622000E1722000E182276
:10D54000120000017151721173117411D8B424D0FA
:10D55000010E756F06D0D8907137723773377437F4
:10D56000752B74AFF8D771516D5D72516E5973514F
:10D570006F5974517059D8A008D071516D5F7251B4
:10D580006E5B73516F5B7451705BD89074337333FF
:10D5900072337133752FE7D76DC06DF06EC06EF0CA
:10D5A0006FC06FF070C070F01200000E0001626F6B
:10D5B000100E636F000E646F000E656F020E676FD2
:10D5C000000E666F6CC068F06DC069F09CEC6BF08B
:10D5D0006CC0D9FF6DC0DAFF240EDE18D8A417D0B6
:10D5E000000120EE01F06C51D9266D51DA22300E87
:10D5F000DE18D8A40CD020EE02F06C51D9266D5163
:10D60000DA222C0EDE18D8A402D0010E1200000E71
:10D610001200000E0201E16F4B0EE26F000EE36F8D
:10D62000000EE46F000EE56F000EE66F080EE76F68
:10D63000000E2B6E1A0E376E010EECEC6EF01E0E05
:10D64000376E020EECEC6EF0000E2F6E6E0E306E2A
:10D65000090E316E400E326E020ED3EC54F02FC024
:10D66000ADF130C0AEF1000E0201716F000E726FAD
:10D67000000E2A6E1200000E00016F6F000E6E6F1A
:10D68000000E6F6F000E6E6F1CD07DEC72F000010B
:10D690006E516625616F6F516721626F000E6821C0
:10D6A000636F000E6921646F6E516A25D96E6F51E8
:10D6B0006B21DA6EDF50656FE0EC6FF000016E4BAE
:10D6C0006F2B6C516E5D6D516F59D8A0DED771EC28
:10D6D00072F0DEEC71F0120062C069F063C06AF0B3
:10D6E00060C067F061C068F01DD069C0F6FF6AC015
:10D6F000F7FF000EF86E0D0EF76403D00800F5502A
:10D7000005D0F6CFE1FFF7CFE2FFE7500001666FEB
:10D71000694B6A2B67C0D9FF68C0DAFF66C0DFFFBC
:10D72000674B682B00016407D8A065076429DDE119
:10D730006529D8B41200D9D7000E00016B6F000E16
:10D740006A6FC9508A94030E2AEC72F0000164518A
:10D750002AEC72F0000163512AEC72F00001625170
:10D760002AEC72F0000E00016B6F000E6A6F0CD095
:10D770006A516825D96E6B516921DA6E5BEC72F0E3
:10D78000DF6E00016A4B6B2B66516A5D67516B5906
:10D79000D8A0EED78A8412000001616F00016151A8
:10D7A0002FEC5CF000016151BEEC5BF000016151B7
:10D7B0004DEC5BF000016151B8EC57F00001615194
:10D7C00041EC57F000016151CAEC56F00001615183
:10D7D0006BEC5AF000016151FAEC59F00001615113
:10D7E00089EC59F000016151DCEC5AF00001615103
:10D7F000B3EC51F012002592000E0201646F000E8E
:10D80000636F000E0001606F050E616F000E636FA5
:10D81000000E626F020E656F000E646F29EC70F0EF
:10D82000000E0001606F070E616F000E636F000E47
:10D83000626F020E656F000E646F29EC70F014ECDD
:10D840004BF06CC015F06DC016F06EC017F06FC0D5
:10D8500018F01200020E2C18D8A403D0C5EC52F018
:10D860001200000E2C6E0101DA51D8A41FD020EE58
:10D8700001F01950D9261A50DA22080EDF6E20EE78
:10D8800002F01950D9261A50DA22300EDE6E010E3F
:10D89000DD6E19C0D9FF1AC0DAFF0C0EDF6E19C099
:10D8A000D9FF1AC0DAFF000EDB8E1200000EDA6F0D
:10D8B0001200000E156E000E166E000E176E000E92
:10D8C000186EE1EC70F005C5EDF206C5EEF208C584
:10D8D000EAF209C5EBF2410E0201EA19D8A41200DE
:10D8E0004B0EEB19D8A4120085AE08D0410EEA6F9A
:10D8F000520EEB6F060E0101BF6F12004B0E0201BC
:10D90000EA6F520EEB6F030E0101BF6F120031C0C0
:10D9100037F032C038F02FC035F030C036F01CD0B0
:10D9200037C0F6FF38C0F7FF000EF86E0D0EF76433
:10D9300003D00800F55005D0F6CFE1FFF7CFE2FFA6
:10D94000E750396E374A382A35C0D9FF36C0DAFF7A
:10D9500039C0DFFF354A362A3306D8A034063328CB
:10D96000DFE13428D8B41200DBD7000E0001706F5D
:10D97000000E6F6F02D03BEC72F02A50D8B41CD06E
:10D98000FAD73BEC72F02A50D8A416D000016F51A0
:10D990006D250201516F000170516E210201526F1D
:10D9A000400E0101D26F010ED16F010E2A6E400EA2
:10D9B00000016F27000E7023020E0001705DD8B0C9
:10D9C0001200DFD7000E0001706F000E6F6F000EA7
:10D9D0006C6F050E6D6FD5EC6AF01BD03BEC72F0EE
:10D9E0002A50D8A416D0000E00016F250201516FF5
:10D9F000050E000170210201526F080E0101D26F65
:10DA0000010ED16F010E2A6E080E00016F27000E65
:10DA10007023020E0001705DD8B01200DFD7000E37
:10DA20000001686F000E696F000E6A6F000E6B6F69
:10DA300060A108D0645168276551692366516A2343
:10DA400067516B23D8906437653766376737D8904E
:10DA5000633362336133603360516111621163116A
:10DA6000D8A4E6D768C060F069C061F06AC062F00F
:10DA70006BC063F01200A0982A50D8B402D0A088DE
:10DA80001200000E0001646F60C062F061C063F0BC
:10DA9000642B6429D8B40DD062C0F6FF63C0F7FFD1
:10DAA000624B632B000EF86E0800F5500009D8A4F5
:10DAB000EFD760C051F261C052F264C0D2F1000EE3
:10DAC0000101D16F010E2A6EA0881200000E000124
:10DAD000666F000E656F62516311D8B41CD0010EE1
:10DAE000646F04D0D89062376337642B63AFFAD782
:10DAF000D890653766376251605D63516159D8A02F
:10DB000005D06251605F6351615B6581D89063337A
:10DB10006233642FEDD765C060F066C061F012001B
:10DB2000A0982A50D8B402D0A0881200000E00019C
:10DB3000646F60C062F061C063F0642B6429D8B484
:10DB400009D062C0D9FF63C0DAFF624B632BDF509C
:10DB5000D8A4F3D760C051F261C052F264C0D2F1D0
:10DB6000010E0101D16F010E2A6EA0881200000E75
:10DB70000001636F100E646F000E656F000E666F1C
:10DB80007DEC72F0DEEC71F088EC72F08A94200E7D
:10DB90002AEC72F0000165512AEC72F00001645128
:10DBA0002AEC72F0000163512AEC72F08A84DEECF8
:10DBB00071F0780ECFEC71F01200000E0001636F6F
:10DBC000F00E646F1F0E656F000E666F7DEC72F0D5
:10DBD000DEEC71F088EC72F08A94200E2AEC72F080
:10DBE000000165512AEC72F0000164512AEC72F0D8
:10DBF000000163512AEC72F08A84DEEC71F0780E39
:10DC0000CFEC71F012000E01D28DD28FD08DD18762
:10DC1000D581CF8DCF8FD48FD48DD085D08BD48B21
:10DC2000D381D383D58FCE85CE87CE89CE8BD58D2C
:10DC3000CE8DCE8FD281D28305EC69F0800E0E019D
:10DC4000D76FF70ED66F020EDA6F830ED96F120000
:10DC50000D01FFA11DD01BC0D9FF1CC0DAFF800E33
:10DC6000DE18D8A414D007C0D9FF08C0DAFF840E8C
:10DC7000DE18D8A40CD01BC0D9FF1CC0DAFF0C0ED4
:10DC8000DF6E1BC0D9FF1CC0DAFF000EDB8EFF91D8
:10DC9000789A12000001726F72C06DF000016E6B15
:10DCA000C20E6F6F020E706F3EEC68F00201C2513F
:10DCB000D00F2FEC5CF00201C351D00FBEEC5BF033
:10DCC0000201C451D00F4DEC5BF00E01A6999E9954
:10DCD00096998E8912000001726F72C06DF000017A
:10DCE0006E6BC20E6F6F020E706F3EEC68F0020139
:10DCF000C251D00F2FEC5CF00201C351D00FBEEC2B
:10DD00005BF00201C451D00F4DEC5BF00E01A699FF
:10DD10009E8996998E9912000001726F72C06DF003
:10DD200000016E6BC20E6F6F020E706F3EEC68F0FA
:10DD30000201C251D00F2FEC5CF00201C351D00F91
:10DD4000BEEC5BF00201C451D00F4DEC5BF00E0154
:10DD5000A6999E9996898E99120072C06DF073C033
:10DD60006EF0C20E00016F6F020E706F3EEC68F035
:10DD70000201C251D00F2FEC5CF00201C351D00F51
:10DD8000BEEC5BF00201C451D00F4DEC5BF00E0114
:10DD9000A6899E9996998E991200000181AF13D0A1
:10DDA0007EC07AF07FC07BF080C07CF081C07DF0C7
:10DDB00011EC70F07AC07EF07BC07FF07CC080F008
:10DDC0007DC081F012007EC07EF07FC07FF080C0F9
:10DDD00080F081C081F012003A6E37A405D0000EA9
:10DDE0002F6E3A50BCEC65F037A205D0010E2F6EB5
:10DDF0003A50BCEC65F03A50010DFF0EF324386E3A
:10DE00000D0EF420396E38C0D9FF39C0DAFF37C0A3
:10DE1000DFFF12000001626F3F0EC716000EC66ED4
:10DE200000016251C6126151C71205D0C78C0DD0D6
:10DE3000C78CC6880AD06051000AD8B4F7D7020A46
:10DE4000D8B4F6D7010AD8B4F4D7C68A12003DEC8C
:10DE500052F06CC09CF16DC09DF16EC09EF16FC020
:10DE60009FF1C0EC5EF0259A000E0101B26F000E2A
:10DE700002015C6F000E5B6F000E216E25882692FA
:10DE8000F9EC6FF01200000E0101DC6F000E3C6E29
:10DE9000740E3B6E000E3D6E000E3E6E000E406E28
:10DEA000000E3F6EFDEC69F075920E01109501D0E9
:10DEB000789478B4FDD7000E0101D36F1200750E6F
:10DEC0000001606F030E616F000E636F000E626FE2
:10DED000000E656F500E646F29EC70F0000E0101AA
:10DEE000AA6F000EA96F000E296E000EA86F000E1B
:10DEF000A76F12000101AF69C9508A94030E2AEC82
:10DF000072F0000164512AEC72F0000163512AECB6
:10DF100072F0000162512AEC72F05BEC72F00101C8
:10DF2000AF6F8A84AF511200270E0001626F100E8E
:10DF3000616F03D06107D8A0620784B409D00101E2
:10DF4000C2AB27B005D0000161516211D8A4F2D74D
:10DF500084A41200320E17EC72F012002D50D8A4D7
:10DF60001200000E756E000E0E01106F160E116F6E
:10DF70009F0E0F6F7B0E106FD08EA288A088F28E3E
:10DF800001D0758675A6FDD7010E2D6E1200240EE8
:10DF90000F012E6F2E95900E2F6F2F89000E2D6F73
:10DFA0002D97100E2B6F000E2C6F2A51618AA98AB3
:10DFB0002A510E01E897A69A0A0ECFEC71F01200D2
:10DFC000C9508A94020E43EC72F00001635143EC95
:10DFD00072F00001625143EC72F00001615143ECB8
:10DFE00072F00001655143EC72F08A8421EC72F00A
:10DFF0001200000E0001606F0DD06051040DC50EBF
:10E00000F324D96E030EF420DA6EDE6ADE6ADE6A6D
:10E01000DD6A602B01014C510001605DD8B0120037
:10E02000ECD700017A517B117C117D11D8B408D056
:10E03000000E7A1B000E7B1B000E7C1B800E7D1BCE
:10E040007AC07AF07BC07BF07CC07CF07DC07DF034
:10E05000120060C066F061C067F009D066C0D9FFE9
:10E0600067C0DAFF62C0DFFF0001664B672B00016B
:10E070006407D8A065076429F1E16529D8B41200C6
:10E08000EDD77DEC72F0DEEC71F08A94600E2AEC34
:10E0900072F08A84780ECFEC71F0780ECFEC71F0CC
:10E0A000780ECFEC71F0780ECFEC71F0DEEC71F001
:10E0B00012000E01108578987582010E0101DC6F47
:10E0C000000ED36F000E3C6E750E3B6E000E3D6E63
:10E0D000000E3E6E000E406E000E3F6EFDEC69F0CD
:10E0E000120002D03BEC72F02A50D8A4FBD72A5081
:10E0F000D8A40AD06A0E0001606F150E616F3BEC68
:10E100006DF002D03BEC72F02A50D8B41200FAD76E
:10E11000000E0001626FCFEC53F0000E0001626F41
:10E12000050E626501D01200625129EC61F0640EA7
:10E13000CFEC71F0CFEC53F00001622BF1D7000E61
:10E140000001606F7F0E606501D00CD06051010D41
:10E15000780EF324D96E040EF420DA6E000EDF6E12
:10E16000602BF0D7000E0101C96F12002FC035F0EF
:10E1700030C036F008D035C0D9FF36C0DAFF31C024
:10E18000DFFF354A362A3306D8A034063328F3E1B8
:10E190003428D8B41200EFD70001626F010E0001DD
:10E1A000616F200E6219D8B408D00E0E626103D0E0
:10E1B000090E626102D0000E616F61C060F06031D3
:10E1C000120015C062F016C063F017C064F018C0EA
:10E1D00065F0020E0001676F000E666F000E686F3B
:10E1E000050E696F9CEC6BF012000E01909D989DDE
:10E1F000A09D0101CDA102D00E01908D0101CDA302
:10E2000002D00E01988D0101CDA512000E01A08D46
:10E210001200EDC0E1F0EEC0E2F0000E0001E36F8D
:10E22000000EE46F36EC2FF0E1C0EDF0E2C0EEF04E
:10E23000E3C0EFF0E4C0F0F01200240E0F012E6FE7
:10E240002E95900E2F6F2F89000E2D6F2D97100E8B
:10E250002B6F000E2C6F2A51A69A0A0ECFEC71F08C
:10E260001200000160516203F3CF64F0F4CF65F057
:10E2700060516303F350652761516203F3506527D2
:10E2800064C060F065C061F01200240E0F012E6FB3
:10E290002E95900E2F6F2F89000E2D6F2D97670EE4
:10E2A0002B6F000E2C6F2A510A0ECFEC71F012006A
:10E2B0000001606F05D0900E636E66BA1200FDD744
:10E2C00000016051000AD8B4F6D7010AD8B4120090
:10E2D000030A12000001606F020E0201645DD8B0F3
:10E2E00008D0000E6325D96E050E6421DA6E60C079
:10E2F000DFFF634B642B1200C95077EC72F0000E05
:10E30000EBEC71F07DEC72F0DEEC71F088EC72F009
:10E31000DEEC71F0DEEC71F012000001626F000EB5
:10E320000001616F3A0E626105D02F0E626502D066
:10E33000010E616F61C060F060311200010E0201D8
:10E340004A27000E4B234C234D230101DC51D8A456
:10E350001200D32BD351D8A41200D3691200CE0ED1
:10E360000001606F020E616F000E636F000E626F3E
:10E37000000E656F0B0E646F29EC70F012002F6EAB
:10E3800005D0900E636E66BA1200FDD72F50000ABA
:10E39000D8B4F7D7010AD8B41200030A120000015A
:10E3A000616F0D0E0001606FFB0EE82EFED7602F2F
:10E3B000FCD700D00001612FF4D71200640E0001D9
:10E3C000626F02EC72F002D002EC72F00001626F38
:10E3D00062A11200F9D70001626F8A94010E2AEC43
:10E3E00072F0000162512AEC72F08A84120004D0AB
:10E3F00000016007D8A06107000160516111D8B425
:10E400001200F6D78A94050E2AEC72F05BEC72F0DB
:10E410000101AF6F8A84AF5112000001606F030EDB
:10E42000E82EFED700F00001602FF9D7120000019E
:10E43000606FC80E00D0E82EFDD70001602FF9D71D
:10E440001200230E0001606F01D060076051D8B444
:10E450001200FBD70001616FC9CF60F061C0C9FF36
:10E46000C7B01200FDD72D0E0001626F150E636F4D
:10E4700028EC46F012001F0E2D64120075B2120037
:10E480000CEC49F012000001606FC95060C0C9FF78
:10E49000C7B01200FDD7360E0001626F150E636F14
:10E4A00028EC46F012000001606F0F012EA3FDD78B
:10E4B00060C029FF1200C9CF60F0000EC96EC7A06E
:10E4C000FED7C95012004848004141008A028C0220
:10E4D0007D02AC020001606F00F00001602FFCD7EC
:10E4E00012008A94040E2AEC72F08A8412008A9434
:10E4F000500E2AEC72F08A8412008A94060E2AECDE
:10E5000072F08A841200259A010EFFEC4FF012007F
:10E5100002EC72F00001626F1200100A0A0A120087
:020000040001F9
:10FFF000A0F509F010F0FFF7FBFEFBFC19F0F8F399
:00000001FF
